:020000040000FA
:1000000000040020990900002D0600007909000075
:1000100037060000410600004B060000000000000B
:10002000000000000000000000000000BD0900000A
:1000300055060000000000005F0600006906000091
:10004000730600007D060000870600009106000090
:100050009B060000A5060000AF060000B9060000E0
:10006000C3060000CD060000D7060000E106000030
:10007000EB060000F5060000FF060000090700007F
:10008000130700001D0700002707000031070000CC
:100090003B070000450700004F070000590700001C
:1000A000630700006D07000077070000810700006C
:1000B0008B070000950700009F070000A9070000BC
:1000C000B3070000BD070000C7070000D10700000C
:1000D000DB070000E5070000EF070000F90700005C
:1000E000030800000D0800001708000021080000A8
:1000F0002B080000350800003F08000049080000F8
:10010000530800001FB500F003F88DE80F001FBD75
:1001100000F038BC70B50B46010B184400F6FF70B8
:10012000040B4FF080500022090303692403406947
:1001300043431D1B104600F0E9F929462046BDE85F
:10014000704000F0E3B9F0B54FF6FF734FF4B475AB
:100150001A466E1E12E0A94201D3344600E00C4656
:10016000B1EB040130F8027B641E3B441A44F9D120
:100170009CB204EB134394B204EB12420029EAD17F
:1001800098B200EB134002EB124140EA0140F0BD8F
:10019000C34992B00446D1E90001CDE91001FF2224
:1001A0004021684600F094FB94E80F008DE80F00B2
:1001B000684610A902E004C841F8042D8842FAD12B
:1001C00010216846FFF7BFFF1090AA208DF8440069
:1001D00000F0FAF800F0DDF84FF01024A0691022CA
:1001E0006946803000F0DEF8A069082210A900F00E
:1001F000D9F800F0C2F870B504460068A94D072888
:1002000069D2DFE800F033041929561E2500D4E92D
:10021000026564682946304600F0FDF82A4621460A
:10022000304600F0BFF8AA002146304600F024FB1B
:10023000002800D0032070BD00F0D6FB4FF48050A2
:1002400007E0201D00F0C6F80028F4D100F0CCFB38
:1002500060682860002070BD241D94E807009200AB
:1002600000F00AFB0028F6D00E2070BD00F0BEF8AA
:100270000028FAD1D4E9010100EB81034FF080504E
:10028000026945696A43934209D84FF010225369C5
:1002900003EB81030169406941438B4201D9092085
:1002A00070BD5069401C01D10F2070BD2046FFF782
:1002B0006FFF00F09BF80028F7D1201D00F08AF8AE
:1002C0000028F2D160680028F0D100F07DF800F03D
:1002D00060F800F052F8072070BD10B50C461828E1
:1002E00002D00120086010BD2068FFF784FF206065
:1002F00010BD4FF01024A069401C05D0A569A66967
:1003000080353079AA2808D06069401C2DD06069FA
:100310000068401C29D060692CE010212846FFF7B6
:1003200012FF316881421CD1A16901F18002C03104
:1003300005E030B108CA51F8040D984201D10120FE
:1003400000E000208A42F4D158B1286810B1042896
:1003500003D0FEE7284600F070F85249686808604C
:1003600008E000F016F800F008F84FF4805001683B
:10037000491C01D000F012FBFEE7BFF34F8F4A4843
:1003800001684A4A01F4E06111430160BFF34F8FF5
:10039000FEE74FF010208169491C02D0806900F00F
:1003A0008CB870472DE9F04117460D4606460024EB
:1003B00006E03046296800F093F8641C2D1D361DB8
:1003C000BC42F6D3BDE8F0814FF0102080694FF4B5
:1003D00080519FE64FF080510A69496900684A439D
:1003E000824201D810207047002070474FF08050A3
:1003F0000169406941434FF01020826902F5805243
:10040000914201D2092070478069401C01D0002030
:1004100070470420704770B50C4605464FF480665F
:1004200008E0284600F049F8B44205D3A4F58064FA
:1004300005F58055002CF4D170BD4168044609B122
:10044000012600E000264FF010256869A26892009E
:1004500000F012FAF8B1A06881006869FFF75AFE4F
:10046000BEB16E694FF08050A56864680169426949
:100470005143A1420DD9016940694143A94208D9BC
:1004800029463046FFF7C7FF2A4621463046FFF788
:1004900089FFFFF772FFFFF797FFFFF77AFFF8E793
:1004A0000C0A0000000000200CED00E00400FA053A
:1004B000144801680029FCD07047134A02211160DA
:1004C00010490B68002BFCD00F4B1B1D18600868EF
:1004D0000028FCD00020106008680028FCD070477D
:1004E000094B10B501221A60064A1468002CFCD092
:1004F000016010680028FCD00020186010680028F7
:10050000FCD010BD00E4014004E5014070B50C468C
:10051000054600F073F810B900F07EF828B12146C6
:100520002846BDE8704000F007B821462846BDE8DF
:10053000704000F037B800007FB5002200920192B1
:10054000029203920A0B000B6946012302440AE05F
:10055000440900F01F0651F8245003FA06F635430B
:1005600041F82450401C8242F2D80D490868009A94
:1005700010430860081D0168019A1143016000F0F2
:100580003DF800280AD0064910310868029A104345
:100590000860091D0868039A104308607FBD0000C9
:1005A0000006004030B50F4C002200BF04EB0213E0
:1005B000D3F800582DB9D3F8045815B9D3F8085812
:1005C0001DB1521C082AF1D330BD082AFCD204EB1D
:1005D0000212C2F80008C3F804180220C3F8080881
:1005E00030BD000000E001404FF08050D0F83001F5
:1005F000082801D000207047012070474FF080503C
:10060000D0F83011062905D0D0F83001401C01D0B7
:1006100000207047012070474FF08050D0F8300123
:100620000A2801D0002070470120704708208F4918
:1006300009680958084710208C4909680958084773
:1006400014208A4909680958084718208749096809
:100650000958084730208549096809580847382053
:1006600082490968095808473C20804909680958A7
:10067000084740207D4909680958084744207B49BC
:1006800009680958084748207849096809580847FF
:100690004C20764909680958084750207349096871
:1006A00009580847542071490968095808475820D3
:1006B0006E490968095808475C206C49096809585F
:1006C0000847602069490968095808476420674954
:1006D00009680958084768206449096809580847A3
:1006E0006C20624909680958084770205F49096809
:1006F0000958084774205D49096809580847782057
:100700005A490968095808477C2058490968095816
:1007100008478020554909680958084784205349EB
:100720000968095808478820504909680958084746
:100730008C204E4909680958084790204B490968A0
:1007400009580847942049490968095808479820DA
:1007500046490968095808479C20444909680958CE
:100760000847A0204149096809580847A4203F4983
:10077000096809580847A8203C49096809580847EA
:10078000AC203A49096809580847B0203749096838
:1007900009580847B4203549096809580847B8205E
:1007A0003249096809580847BC2030490968095886
:1007B0000847C0202D49096809580847C4202B491B
:1007C000096809580847C82028490968095808478E
:1007D000CC202649096809580847D02023490968D0
:1007E00009580847D4202149096809580847D820E2
:1007F0001E49096809580847DC201C49096809583E
:100800000847E0201949096809580847E4201749B2
:10081000096809580847E820144909680958084731
:10082000EC201249096809580847F0200F49096867
:1008300009580847F4200D49096809580847F82065
:100840000A49096809580847FC20084909680958F5
:1008500008475FF480700549096809580847000097
:1008600003480449024A034B70470000000000207F
:10087000180A0000180A000040EA010310B59B079F
:100880000FD1042A0DD310C808C9121F9C42F8D0FA
:1008900020BA19BA884201D9012010BD4FF0FF30AB
:1008A00010BD1AB1D30703D0521C07E0002010BDC1
:1008B00010F8013B11F8014B1B1B07D110F8013B4D
:1008C00011F8014B1B1B01D1921EF1D1184610BD2E
:1008D00002F0FF0343EA032242EA024200F005B8B5
:1008E0007047704770474FF000020429C0F0128033
:1008F00010F0030C00F01B80CCF1040CBCF1020FD3
:1009000018BF00F8012BA8BF20F8022BA1EB0C01A7
:1009100000F00DB85FEAC17C24BF00F8012B00F89D
:10092000012B48BF00F8012B70474FF0000200B5C3
:10093000134694469646203922BFA0E80C50A0E802
:100940000C50B1F12001BFF4F7AF090728BFA0E8B0
:100950000C5048BF0CC05DF804EB890028BF40F87C
:10096000042B08BF704748BF20F8022B11F0804FBE
:1009700018BF00F8012B7047014B1B68DB68184754
:100980000000002009480A497047FFF7FBFFFFF706
:10099000B9FB00BD20BFFDE7064B1847064A1060B3
:1009A000016881F30888406800470000180A0000C9
:1009B000180A0000F3020000000000201EF0040FDF
:1009C0000CBFEFF30881EFF30981886902380078E2
:1009D000182803D100E00000074A1047074A1268B0
:1009E0002C3212681047000000B5054B1B68054A01
:1009F0009B58984700BD0000DB020000000000206B
:100A0000080A0000040000000010000000000000C0
:080A100000FFFFFF0090D0037E
:1010000010400020111400001914000031120000DB
:101010001D1400001F140000211400000000000037
:101020000000000000000000000000002314000089
:1010300025140000000000002714000029140000FF
:10104000191B00002B1400005D1E00002B14000073
:101050002B1400002B140000811700002B1400003B
:101060002B1400002B1400002B1400002B14000084
:101070002B1400002B1400002B1400002B14000074
:101080002B140000291B00002B1400002B1400005F
:101090002B1400002B1400002B1400002B14000054
:1010A0002B1400002B1400002B1400002B14000044
:1010B0002B1400002B1400000000000000000000B2
:1010C0002B1400002B1400002B1400002B14000024
:1010D0002B1400002B1400002B140000B51E000080
:1010E0002B1400002B1400002B1400000000000043
:1010F000000000002B140000000000002B14000072
:1011000000000000000000000000000000000000DF
:1011100000000000000000000000000000000000CF
:1011200000000000000000000000000000000000BF
:1011300000000000000000000000000000000000AF
:10114000000000000000000000000000000000009F
:10115000000000000000000000000000000000008F
:10116000000000000000000000000000000000007F
:10117000000000000000000000000000000000006F
:10118000000000000000000000000000000000005F
:10119000000000000000000000000000000000004F
:1011A000000000000000000000000000000000003F
:1011B000000000000000000000000000000000002F
:1011C000000000000000000000000000000000001F
:1011D000000000000000000000000000000000000F
:1011E00000000000000000000000000000000000FF
:1011F00000000000000000000000000000000000EF
:10120000DFF80CD000F070FA004800477D7D000048
:101210001040002000B583B002900091019244F28A
:10122000010071466A4601F045F803B000BD0000B8
:10123000094B1EF0040F1CBFEFF309801847EFF3B2
:1012400008800649064A884201D8904202D88D4655
:101250004FF0000018470000351900001040002032
:101260001020002030B450E8012F93B2C4892344E9
:101270008489A34228BF1B1B0489A34202BFBFF37A
:101280002F8F002007E0C3EA020340E80134002C5E
:10129000E9D14FF001000A6030BC704750E8012FDF
:1012A000C2EA024240E801210029F7D1704730B478
:1012B00050E8022F1FFAA2F3C488A34202BFBFF373
:1012C0002F8F00200DE0C48923448489A34228BFC6
:1012D0001B1BC2EA034340E80234002CE8D14FF064
:1012E00001000A6030BC704750E8022FC2EA224277
:1012F00040E802210029F7D17047034653E8022F46
:10130000D988B2EB324F4FF0000017BF92B241EADA
:10131000014142EA014104E05A68B2EB324F08BF92
:10132000012043E80212002AE8D1704730B4044695
:1013300054E8000F0D4644E80053002BF8D1156027
:1013400030BC704730B4044654E8000F40EA010551
:1013500044E80053002BF7D1156030BC704730B41F
:10136000044654E8000F00EA010544E80053002B4E
:10137000F7D1156030BC704730B4044654E8000F14
:1013800080EA010544E80053002BF7D1156030BC1A
:10139000704730B4044654E8000F00EB010544E800
:1013A0000053002BF7D1156030BC704730B40446B1
:1013B00054E8000FA0EB010544E80053002BF7D1DF
:1013C000156030BC704770B404464FF0000054E81C
:1013D000006F0D68AE4207BF44E80023012044E8D7
:1013E00000630E60002B1CBF0020F0E770BC70474C
:1013F00030B4044654E8000F88422CBF451A054615
:1014000044E80053002BF5D1156030BC7047000054
:101410000648804706480047FEE7FEE7FEE7FEE78E
:10142000FEE7FEE7FEE7FEE7FEE7FEE7811C0000C1
:10143000011200000048704790F30000A0F1410144
:10144000192900D8203070472DE9FE4399461546EA
:101450008846074601AC022942D3002D40D0002027
:101460000290A8F101004FF0FF36009022E000FB4F
:10147000057201FB057011464A469047002805DCBD
:1014800054F82600304444F8260013E060682A46E9
:1014900000FB057154F8040C00FB057007E00B78A5
:1014A00090F800C001F801CB00F8013B521E002A61
:1014B000F5D1764254F8040C61688842D7DC4B467B
:1014C0002A463846FFF7C0FF54F8040C4B46A8EBF9
:1014D0000001401C00FB05702A46491EFFF7B4FFBF
:1014E000BDE8FE8310B5431A934209D283188818C9
:1014F00003E010F8011D03F8011D521EF9D210BDC2
:1015000040EA01039B0703D009E008C9121F08C085
:10151000042AFAD203E011F8013B00F8013B521E05
:10152000F9D210BDD2B201E000F8012B491EFBD266
:1015300070470022F6E710B513460A4604461946DE
:10154000FFF7F0FF204610BD30B505462A460B4692
:1015500012F8010B13F8014B08B1A042F8D01CB1EE
:10156000002802D06D1CF1E7284630BDCAB2401EEB
:1015700010F8011F8A4202D00029F9D100207047DB
:10158000421C10F8011B0029FBD1801A704710B5CE
:10159000002200E0521C835C8C5CA34201D1002B32
:1015A000F8D1D8B2E1B2401A10BD034611F8012BB0
:1015B00000F8012B002AF9D11846704730B50546CE
:1015C0000020034600E05B1C934205D2EC5CC85C43
:1015D000201A01D1002CF6D130BD2DE9F0479146FB
:1015E0000F4680460446002614F8015B2DB1FFF734
:1015F00021FF0068405DC007F6D12B2D02D02D2DB4
:1016000018D0641E4A463946204600F01EF827B11D
:101610003968A14201D1C7F8008071054FF002047A
:101620000BD54042002803DD00F0AEFD0460A007AA
:10163000BDE8F08746F48066E4E70028F8DA00F0B9
:10164000A3FD04606FF00040F2E72DE9F05F8246F1
:101650000078002715468B460AF10104B946302868
:1016600001D09DB113E014F8010B0127782803D0B5
:10167000582801D045B10AE00DB1102D07D100273F
:10168000102514F8010B02E0082500E00A250026C9
:10169000B0460EE005FB080005FB06F1012701EB53
:1016A00010461FFA80F8B6F5803F00D3B94614F80B
:1016B000010B294600F02AF80028EBDABBF1000FF5
:1016C00005D00FB1641E00E05446CBF80040B9F1DC
:1016D000000F06D000F058FD02210160C81EBDE8D1
:1016E000F09F48EA0640FAE7064C074D06E0E0683E
:1016F00040F0010394E8070098471034AC42F6D359
:10170000FFF782FDB4110100D41101003A2800D284
:10171000303820F02002412A01D3A2F1370088425C
:1017200001D34FF0FF30704770B58C1810F8015B93
:1017300015F0070301D110F8013B2A1106D110F86A
:10174000012B03E010F8016B01F8016B5B1EF9D16E
:101750002B0705D40023521E0DD401F8013BFAE7F4
:1017600010F8013BCB1A921C03E013F8015B01F85F
:10177000015B521EF9D5A142D8D3002070BD0000F4
:101780002DE9F04F00268DB0DFF8A081B146049618
:101790004FF48075012437460596284609F0ECFB86
:1017A00038B1D8F80403204203D0284609F0DAFB08
:1017B00026432D1D64007F1CADB2082FEDD34FF4DE
:1017C000BE74204609F0D8FB48B1204609F0CAFB98
:1017D00046F0004604AA0221002009F08DFB544C7B
:1017E00016F0FF0F15D00127002537420DD008EB6A
:1017F0008501D1F81005D1F81015C0F3052054F873
:101800002520C1F3014102B190477F006D1C082DD6
:10181000EBD3002E7EDA0020CDF82890411E0DF18A
:10182000100B07AACDF82C9042F82010401C9146CE
:101830000228F9D300252E46A11911F8607F91F9ED
:10184000000027F0C008401C40D007A9404606F021
:101850003FFF40B34FEA971A404602F057FC54F856
:1018600020701FB1BAF1030F03D006E0BAF1030FE5
:101870002CD10AA9404606F033FF02A8CDF8088013
:1018800009F00AFB029900EB8100D0F8000704A9D7
:10189000C0F301400290404606F01AFF002802986B
:1018A00002D0022802D011E003280FD1BAF1030FB1
:1018B00008D10298022833D00221404609F0D4FA18
:1018C0006D1CEDB217B151464046B847761C042E48
:1018D000B2D3002D21D001AA0221002009F00CFB77
:1018E00000205A460DF1040152F8206051F82030D2
:1018F000B34217D000200AAE4FEA090351F8207016
:1019000042F8207056F8207043F82070401C0228DE
:10191000F4D300E001E0002D8CD10DB0BDE8F08FD4
:101920000321CAE7401C0228DED3F6E7006000402E
:10193000C81300201CB5814609F01AFF09F0B2FC5B
:101940000028FBD137484E460768374C01256068B0
:10195000002821D0208835A105EB0040B26909F0AC
:10196000CFFD6068002817D0D6E90201CDE900015B
:101970002088D6E9002305EB004032A109F0D8FD0C
:10198000606848B1F0690090D6E9042320883BA143
:1019900005EB004009F0C3FD2248001D00688007E8
:1019A00007D5606828B120883E4905EB004009F062
:1019B000A3FDDFF8F480002605FA06F038420AD0CD
:1019C00058F826203AB1606828B1208837A105EB85
:1019D000004009F095FD761C1A2EEDD338060AD585
:1019E000606840B10F480C300268208832A105EBD6
:1019F000004009F085FD38040AD5606840B1094807
:101A000010300268208834A105EB004009F078FD11
:101A10000448C8300068C00700D000BE484600F047
:101A200069F8000028ED00E08C0400204841524491
:101A3000204641554C542061742030782530385868
:101A400000000000202052303A2020307825303825
:101A500058202052313A2020307825303858202024
:101A600052323A2020307825303858202052333AEC
:101A700020203078253038580000000020205231D6
:101A8000323A2030782530385820204C523A2020E5
:101A900030782530385820205053523A203078255D
:101AA0003038580048FE0000E8010020436175739B
:101AB000653A2025732E00004D656D4D616E61679E
:101AC00065204661756C7420416464726573733A75
:101AD0002030782530385800427573204661756C87
:101AE0007420416464726573733A2030782530380D
:101AF00058000000BFF34F8F05480168054A01F404
:101B0000E06111430160BFF34F8F00BFFDE70000AC
:101B10000CED00E00400FA0510B50BF047F9BDE844
:101B200010400BF071B8000002490248091F096813
:101B300000680847E0010020044900EB400001EB89
:101B4000C000416D806D081A70470000881D00209C
:101B500000F064BA70B5064614460D46002001F048
:101B60001BFD22462946304600F006F804460020B8
:101B700001F040FD204670BD2DE9F0471B4D0746A2
:101B8000164628780C4608B900F048FA07EB4700DB
:101B900005EBC007A046D7E91595002448374D4509
:101BA00011D9B868441BB44200D334467868224641
:101BB00041194046FFF796FCB868361B2544A044FF
:101BC000A84200D10025A9EB0500B04200D206468C
:101BD0003EB17868324641194046FFF783FC3444F1
:101BE000354404B13D612046BDE8F087881D0020E2
:101BF00070B50B4B0646144618780D4608B900F030
:101C00000DFA002001F0C8FC22462946304600F0BB
:101C100009F80446002001F0EDFC204670BD0000EC
:101C2000881D002070B50E46144900EB400001EB02
:101C3000C0051446E86A183520B101280FD00228E3
:101C400005D113E0284600F01DFAA04201D200247D
:101C500011E022463146284600F061FA0BE02846A2
:101C600000F010FAA042F4D20446F2E731462846CA
:101C700000F028FA0446204670BD0000881D0020B0
:101C800030B54FF0805000228300D0F83011C3F8F7
:101C90000C21C3F81021624B1A60624B1B68624C26
:101CA0002360604B1B1D1B68241D23605D4B0833A4
:101CB0001B68241D23605B4B0C331B68241D2360B1
:101CC000584B10331B68241D2360564B14331B687C
:101CD000241D2360534B18331B68534C203423605E
:101CE000504B1C331B68241D23604E4B20331B6854
:101CF000241D23604B4B24331B68241D2360494B58
:101D000028331B68241D2360464B2C331B68241D7D
:101D10002360444B30331B68434C40342360414BB9
:101D200034331B68241D23603E4B38331B68241D4D
:101D300023603C4B3C331B68241D2360394B4033EC
:101D40001B68241D23600124082902D1D0F83431F6
:101D500013B1082904D006E0354B3449196005E079
:101D6000D0F8343113B1082904D006E0314BFB21FF
:101D7000196005E0D0F8343113B1082908D00EE01D
:101D800090F858322C48016863F30301016002E0C7
:101D9000D0F834311BB929494FF400700860284845
:101DA0000168C90702D06FF0010101602548016890
:101DB00041F470010160BFF34F8FBFF36F8F4FF09D
:101DC0001021D1F80002002803DBD1F8040200281A
:101DD00022DA1D4B1C601D480468002CFCD0122424
:101DE000C1F800420568002DFCD0C1F8044201682A
:101DF0000029FCD01A6001680029FCD0BFF34F8F86
:101E000010487C380168124A01F4E0611143016016
:101E1000BFF34F8F00BFFDE70F490E48086030BD8C
:101E2000380500400404001020C50040488103002C
:101E30008C56004018F50040E40E004040960240E9
:101E40000004004088ED00E004E5014000E40140AA
:101E50000400FA050090D0030803002010B5054CDB
:101E6000206818B904A12B2001F004FC2068BDE80B
:101E7000104000475C0100202E2E5C2E2E5C2E2E82
:101E80005C2E2E5C2E2E5C2E2E5C6D6F64756C6548
:101E9000735C6E7266785C647269766572735C738B
:101EA00072635C7072735C6E7266785F7072732EB0
:101EB000630000002DE9F05F5448D0F8045300247B
:101EC0002E464FF0010913E096FAA6F0B0FA80F71B
:101ED000B80000F5807080460AF098FD28B14046B1
:101EE0000AF09CFD09FA07F0044309FA07F086435B
:101EF000002EE9D108F0B4F8002869D0444AD0781F
:101F0000F0BBA00264D5434940F2A978C1F8008033
:101F1000081D036813F0FF0C02D0036803EA0C0CE1
:101F200040F2AA7AC1F800A0036813F0FF0301D0C1
:101F30000668334040F2AB7BC1F800B0066816F08B
:101F4000FF0601D007683E4040F2AC770F6007689B
:101F500017EA0C0709D0D2F810C04CEA070CC2F8F7
:101F600010C0C1F800800760076840F2AD770F60CD
:101F700007681F4009D0136943EA0743136100E073
:101F800026E0C1F800A00760036840F2AE730B6062
:101F9000036833400BD0DE0701D044F40004DE06B2
:101FA00001D544F00104C1F800B003600068106975
:101FB00030F0011102D005F080710C4310F0011FC8
:101FC00006D0690504D520F0011044F48064106146
:101FD000C4F3C05624F400044F46DFF83C8009E007
:101FE00094FAA4F0B0FA80F558F82500804707FA73
:101FF00005F08443002CF3D10CF010FA002E03D02E
:10200000BDE8F05F04F0D4BEBDE8F09F0070024070
:102010002C0100200078024018EB000010B5124C93
:1020200002202061606111A0A06104F17800E061EC
:102030004FF4007020620020A06260620BA1A164D6
:10204000E06204F51E71E1641021A065C4E914107A
:10205000E06509A1E01DFFF7A8FA08A12046FFF7F7
:10206000A4FA2020A07110BD881D00205465726D57
:10207000696E616C0000000052545400534547479C
:10208000455200000269C1688A4203D88068401A3C
:10209000104400E0501A401E70470000C11700EBCA
:1020A000D161074B4A1153F8222021F01F01411A38
:1020B00001208840024201D0012070470020704773
:1020C00000E100E02DE9F047C4681746894606465E
:1020D0004FF000083069A04201D9051B02E0B16849
:1020E000201A0D1AB0686D1E001BA84200D80546C4
:1020F000BD4200D33D4670682A4620444946FFF75A
:10210000F1F9B0687F1B2C44A844A944A04200D137
:102110000024F460002FDDD14046BDE8F0872DE9B2
:10212000F04104468846D4E90207C51BE1686068AF
:1021300016460844B54206D94146FFF7D3F9B81907
:10214000E060BDE8F0812A464146FFF7CBF9761BF7
:1021500008EB050132466068FFF7C4F9E660F0E776
:102160000FB4084B10B504A902AA039800F01FF899
:10217000044602A9002000F085F8204610BC5DF856
:1021800014FB000085220000004870470C0300206B
:1021900002E008C8121F08C1002AFAD17047704730
:1021A000002001E001C1121F002AFBD170472DE978
:1021B000F84F9946924688460546002706E02528AE
:1021C0000AD051464A4690476D1C7F1C287800284B
:1021D000F5D13846BDE8F88F002315F8011F1846E1
:1021E0002E2915D115F8011F04232A290DD06FF0CF
:1021F0002F022978A1F13004092C09D800EB8000C6
:1022000002EB400008446D1CF3E758F8040B6D1C0A
:102210002A78002ADDD0632A07D0732A0FD010460F
:1022200051464A4690477F1C2AE018F8042B8DF847
:10223000002000218DF801106E46012103E058F8BE
:10224000046B4FF0FF315A074FF0000401D409E04E
:10225000641C84420BDA8C42FADB325D002AF7D12F
:1022600005E0641C8C42FCDB305D0028F9D127447A
:1022700004E016F8010B51464A469047641EF8D216
:102280006D1CA3E70A68531C0B6010707047800731
:1022900001D00020704701207047C3688B4206D8E8
:1022A00011440069491E814201D801207047002075
:1022B000704700002DE9FE4315460F46804672B672
:1022C00009F056FA08F0EEFF0028FBD16FF48041C8
:1022D000224C18EB01004FF0010622D00128606863
:1022E00014D030B120883A4606EB00401CA109F01A
:1022F00007F921480068C00700D000BE2A4603B095
:1023000039464046BDE8F04300F064B80028F0D0FC
:1023100020882B8806EB004018A16A6809F0F7F8BE
:10232000E7E760680028E4D0A8680AF0DDF9034612
:10233000D5E90001CDE900100297208816A106EB2F
:102340000040AA6809F0FEF860680028D1D0208813
:102350001BA106EB004009F0CFF8CAE7F804002003
:10236000554E4B4E4F574E204641554C54206174AC
:102370002030782530385800F0ED00E041535345C7
:102380005254494F4E204641494C454420617420E7
:1023900025733A25750000004552524F522025758D
:1023A000205B25735D2061742025733A25750D0A25
:1023B00050432061743A203078253038780000008E
:1023C000456E64206F66206572726F722072657050
:1023D0006F72740008B501238DF800309DF800304D
:1023E000144B186059609A606FF48041401807D010
:1023F00001280FD1DA60D86800889861D86807E0B2
:102400001A611869806858611869006898611869CC
:102410004068D861186858689868D8681869586919
:102420009869D86972B600BF9DF800000028FBD1FA
:1024300062B608BD34140020014804F01EB9000043
:102440006C01002070B514460E46050004D10B49FE
:1024500040F2C51001F00EF93CB12868012EC460AD
:102460000AD000218160002070BD04494FF4E37060
:1024700001F000F9072070BD0121F3E788FB00009F
:1024800038B50E4808235822416800910C4900686D
:1024900005F019FF00280FD10A4A69460A4804F0DE
:1024A000F1F8040008D10121074804F0C2F90649F7
:1024B000012008390870204638BD0000BCEB000040
:1024C0005414002081D300006C01002070B5164622
:1024D0000D46040004D10C4940F2D51001F0CAF8B1
:1024E0000A48854201D9072070BD0948266104F0D9
:1024F000C4F828446060A06800B1A5602146BDE82A
:10250000704000200BF0A0BD88FB000017FCFF000E
:102510006C01002010B5040004D106494FF4F57099
:1025200001F0A8F8002021462076BDE810400120E7
:102530000BF08ABD88FB000070B50546064844686C
:1025400007E02946204601F05BFF204600F022FA12
:102550000446002CF5D170BD8C01002070B50A48EE
:1025600045680EE02E7A002405E02146284600F05A
:1025700015FE641CE4B2B442F7D3284600F00AFA10
:102580000546002DEED170BD8C0100202DE9F041F3
:102590000E4840F2AB67456814E02E7A00240BE049
:1025A00000222146284600F05DFE18B108A13846F9
:1025B00001F060F8641CE4B2B442F1D3284600F0A4
:1025C000E9F90546002DE8D1BDE8F0818C01002035
:1025D0002E2E5C2E2E5C2E2E5C2E2E5C2E2E5C2E35
:1025E0002E5C636F6D706F6E656E74735C6C696288
:1025F0007261726965735C757362645C6170705F4F
:10260000757362642E63000070B50646094806259E
:1026100044680AE03146204601F0F2FE05460628ED
:1026200005D1204600F0B6F90446002CF2D1284628
:1026300070BD00008C0100202DE9FC4115460F0003
:10264000064604D11E494FF47C7001F013F8304661
:1026500001F09AF80446007DC00715D0002000F074
:102660009BFFE06E98B1A84200D805462A4638463E
:10267000A16EFEF737FFE06E401BE066A06E656757
:102680002844A066002405E00820BDE8FC81A0697C
:1026900028B11124002000F0ADFF2046F5E7C4E981
:1026A0000675304603F0CFFF06498969CDE900146D
:1026B000694600F0A3FB0400ECD19224EAE7000095
:1026C00014FC00001CEC000010B501F05DF8406F38
:1026D00010BDFEB515460E46044601F055F8007DC6
:1026E00010F0010F0AD0204603F0A4FF002100964D
:1026F000CDE90151694600F0CDFBFEBD0820FEBDCD
:10270000F8B5040004D138A140F2EF4000F0B2FF68
:10271000606820B934A14FF49E6000F0ABFF6068A0
:10272000006820B930A140F2F14000F0A3FF20681A
:10273000006820B12CA140F2F24000F09BFF07F0AE
:102740001BFE10B907F022FE20B927A140F2F64087
:1027500000F090FF00250FE0002705E0007800F072
:1027600061FB08B11120F8BD3946781CC7B230466C
:1027700000F0C0F80028F1D12946681CC5B22046F7
:1027800000F0E0F80600E7D100250DE0002703E0A7
:102790000078214600F04CFB3946781CC7B2304621
:1027A00000F0A8F80028F3D12946681CC5B22046DD
:1027B00000F0C8F80600E9D1194D40F21C5607E0B8
:1027C000A04203D108A1304600F054FF28680568F4
:1027D00028680028F4D113482C60694640690090AD
:1027E000204601F00DFEF8BD2E2E5C2E2E5C2E2E06
:1027F0005C2E2E5C2E2E5C2E2E5C636F6D706F6EC9
:10280000656E74735C6C69627261726965735C7524
:102810007362645C6170705F757362642E63000044
:1028200090010020D0EB00002DE9F04F87B04FF071
:1028300000081D46934689460446DDF840A04646FA
:10284000CDF80C8000E0761C606801230022476808
:10285000214603A8B8470028F5D140468DF80080EE
:102860000027B84601903BE0606801236A46D0F833
:1028700004C0214601A8E0476068012305AAD0F8FA
:1028800004C0214601A8E0479DF8141049451AD11B
:10289000D84514D19DF80000CAF8000005F8010BD6
:1028A0006A1C85F8009060689DF8003021464568F4
:1028B00001A89B1EA847002007B0BDE8F08F08F1D3
:1028C000010000F0FF0860689DF800300022D0F899
:1028D00004C0214601A89B1EE0479DF80000074464
:1028E000B742C1D30520E7E70148406870470000C0
:1028F0008C01002070B50D46040004D106494FF448
:102900008E7000F0B7FE6078A84201D8002070BD3C
:10291000A0782044284470BDD0FB000070B50D465F
:10292000040004D106494FF48E7000F0A3FE6078D5
:10293000A84201D8002070BDA0782044284470BD72
:10294000D0FB000070B50D46040003D10649E92014
:1029500000F090FE207AA84201D8002070BD05EB5F
:1029600045000934204470BDD0FB000070B50D4611
:10297000040003D10649E92000F07CFE207AA84239
:1029800001D8002070BD05EB45000934204470BD1E
:10299000D0FB000010B5040004D104494FF4F970D5
:1029A00000F068FE2068006810BD000004310000DF
:1029B00010B5040004D104A14FF4F97000F05AFEE0
:1029C0002068006810BD00002E2E5C2E2E5C2E2E7E
:1029D0005C2E2E5C2E2E5C2E2E5C636F6D706F6EE7
:1029E000656E74735C6C69627261726965735C7543
:1029F0007362645C6170705F757362642E6800005E
:102A000002484078002800D0012070478C01002047
:102A10002DE9F041484E0D460246097806243078EB
:102A200001270F2964D2DFE801F063080C0E632050
:102A30004863636363252D363F0003200BF0F4FBEE
:102A400056E0002454E03C48001D05F07EFC28B10F
:102A50003A480760BFF36F8FBFF34F8F307800287D
:102A6000EFD137A140F20B4009E0104600F0A4F886
:102A700004463DE00028E4D031A140F2164000F0C9
:102A8000F9FDDEE7012804D02DA140F21C4000F042
:102A9000F1FD002005E03948006810F0010F0AD070
:102AA00002200BF0C1FBCCE7022804D224A14FF492
:102AB000866000F0DFFD0120F3E7E878032817D0F7
:102AC000A87830B1802804D01DA140F23E4000F02B
:102AD000D1FD1949E87808310A6832B100230B604A
:102AE00049689047040006D000E00E2407F0A8FCD7
:102AF0002046BDE8F0810BF08FFB28B1A8780028B4
:102B0000F6D107F060FCF3E71D480078082810D1E3
:102B10001B48001D007800070BD1194808300078C9
:102B200010F0F00F05D116480C30007810F0F00FBF
:102B3000DED007F045FCDBE7AC0100205C70024012
:102B40002E2E5C2E2E5C2E2E5C2E2E5C2E2E5C2EBF
:102B50002E5C636F6D706F6E656E74735C6C696212
:102B60007261726965735C757362645C6170705FD9
:102B7000757362645F636F72652E63003804004092
:102B8000E00F00F0024A0146D2E9000210470000BF
:102B9000F414002070B50C46054607F00BFCA84263
:102BA00001D0102070BD0348D4E90012C0E9021220
:102BB000002070BDAC0100207FB5054605208DF8D2
:102BC000000006240DF1010007F012FC0BF024FBBD
:102BD0002949002008609DF8010010F01F0006D070
:102BE00001280FD0022826D0032833D106E06946F9
:102BF00028460AF073FD044606282AD16846FFF7E6
:102C000003FD25E09DF8050003A900F007FB050082
:102C100008D06A469DF80C1000F0BCFA044606285D
:102C200002D016E0102415E06A469DF80C102846E4
:102C30000AF0AEFE0CE09DF80500010705D06946DC
:102C400000F080F80446062803D168460AF0F0FD3B
:102C5000044624B107F0F4FB04B0204670BD0BF02D
:102C6000DBFA30B107F0A6FB0028F5D107F0ABFB8B
:102C7000F2E707F0A5FBEFE7B4010020FEB5C0883E
:102C800014460E46A04201D2054600E01546844295
:102C900007D2802007F00AF8B4FBF0F100FB1140E6
:102CA00068B100200096CDE90150002000F074FCCE
:102CB0006946802000F0EEF8040002D006E0012012
:102CC000F0E705498020FFF765FF0446002000F08B
:102CD00091FC2046FEBD00004CEC000008B14021F4
:102CE00001600148704700004815002010B507F04A
:102CF00055FB20B104A140F26F3000F0BBFCBDE8F1
:102D0000104006F0D5BD00002E2E5C2E2E5C2E2E1F
:102D10005C2E2E5C2E2E5C2E2E5C636F6D706F6EA3
:102D2000656E74735C6C69627261726965735C75FF
:102D30007362645C6170705F757362642E6300001F
:102D400006F0F8BD10B50C46010600F00F02092A86
:102D500008D200F009F8006820B12146BDE8104013
:102D600001F04EBB102010BD10B5010600F00F049D
:102D700008D5092C04D309A140F2611000F07AFCB7
:102D8000144808E0092C04D304A140F2671000F0B5
:102D900071FC1048483000EBC40010BD2E2E5C2E94
:102DA0002E5C2E2E5C2E2E5C2E2E5C2E2E5C636FE7
:102DB0006D706F6E656E74735C6C6962726172695E
:102DC00065735C757362645C6170705F7573626477
:102DD0002E630000AC14002010B5044600F00F0074
:102DE000082805D2204606F089FE204606F0E2FFBC
:102DF0002046BDE8104006F0A5BE000070B50C46A8
:102E0000054606F0EFFE18B105480078022801D00B
:102E1000082070BD21462846BDE8704006F0EABE95
:102E20008C01002010B5FFF79FFF006810BD000067
:102E300070B50D460646FFF797FF0446056015B1CD
:102E40006868006808E00EB1802E04D103A140F24A
:102E50008B1000F00FFC0020606070BD2E2E5C2EE9
:102E60002E5C2E2E5C2E2E5C2E2E5C2E2E5C636F26
:102E70006D706F6E656E74735C6C6962726172699D
:102E800065735C757362645C6170705F75736264B6
:102E90002E63000070B50C46054606F0A3FE18B17F
:102EA00005480078022801D0082070BD2146284638
:102EB000BDE8704007F00EB88C0100200149096898
:102EC000084700003C15002070B57D4C0546606841
:102ED00020B97CA140F2C33000F0CCFB03F0F6F93E
:102EE000072804D277A140F2CA3000F0C3FB28784B
:102EF000092872D007DC16D2DFE800F07085A98CB3
:102F000096B2B715DA00812814D006DC0A28F0D072
:102F10000F28EED0802806D13CE082281FD08328DD
:102F200043D084284AD0BDE8704066A140F2AB404F
:102F300000F0A0BB7148FFF725FE7048FFF7FCFAD0
:102F40000D200BF041FCA06810B96D48007A00B16B
:102F5000012007F079FAFFF701FB012073E0FFF78A
:102F6000FDFA07F0C7FA00200AF0C4FE6348401CCF
:102F7000FFF7E2FA6148401CFFF704FE0E200BF059
:102F800023FC207800F0EEFA00283BD0BDE870402A
:102F900006F00EBB2078052803D0062803D00728AA
:102FA00030D102204FE008204DE02078032829D1BD
:102FB00007F0EAFA002825D0042044E0207803280E
:102FC00005D107F0E1FA10B104200AF093FE07F0F2
:102FD000ABFB002816D0062035E06AE000200BF09D
:102FE000F3FBA46840F20E260AE02946204601F0D1
:102FF00007FA1CB943A1304600F03CFB2068446846
:10300000002CF2D170BDFFF7A9FA02200AF072FE7F
:10301000012003E005200AF06DFE03200BF0D4FB35
:103020002846FFF7AFFD46E003200BF0CDFB334809
:10303000801CFFF7A7FD3148801CFFF77DFA207840
:103040000628AED10720BDE870400AF053BE032029
:103050000AF050FE02200BF0B7FB2846FFF76CFA8F
:103060002846BDE87040FFF78DBDA878FFF77CFECD
:103070000446006820B913A140F2874000F0FAFA34
:10308000606820B90FA14FF4916000F0F3FAD4E921
:103090000002294690470028B4D0A8780107B1D093
:1030A00000F00F010829ADD2BDE8704006F050BE17
:1030B00008200BF089FB2846BDE87040FFF73CBABA
:1030C0008C0100202E2E5C2E2E5C2E2E5C2E2E5C73
:1030D0002E2E5C2E2E5C636F6D706F6E656E74733A
:1030E0005C6C69627261726965735C757362645C61
:1030F0006170705F757362642E630000E1EB000025
:103100003C1500202E2E5C2E2E5C2E2E5C2E2E5C6E
:103110002E2E5C2E2E5C636F6D706F6E656E7473F9
:103120005C6C69627261726965735C757362645C20
:103130006170705F757362642E680000FFF7BEBE39
:1031400010B520B104A140F2272000F093FABDE8A9
:1031500010400F48FFF7B2BE2E2E5C2E2E5C2E2E96
:103160005C2E2E5C2E2E5C2E2E5C636F6D706F6E4F
:10317000656E74735C6C69627261726965735C75AB
:103180007362645C6170705F757362642E630000CB
:10319000D0EB0000114601F033B9000070B50446D1
:1031A00040680D46C2680AB120469047207AA8427E
:1031B00004D20CA140F2BF2000F05CFA2946204660
:1031C000FFF7C0FB05464678002408E02146284664
:1031D000FFF790FB007806F061FC641CE4B2B44297
:1031E000F4D370BD2E2E5C2E2E5C2E2E5C2E2E5C0B
:1031F0002E2E5C2E2E5C636F6D706F6E656E747319
:103200005C6C69627261726965735C757362645C3F
:103210006170705F757362642E6300002DE9F04188
:1032200080460F480E46456816E02F7A00240DE0D0
:1032300021462846FFF786FB0178414504D106B1B7
:1032400034702846BDE8F081641CE4B2BC42EFD380
:103250002846FFF79FFB0546002DE6D10020F1E749
:103260008C01002070B50446406815460E46836800
:103270001BB120469847062809D1207AB04204D2D3
:103280000E494FF4287000F0F5F90DB1072070BD1C
:1032900031462046FFF756FB05464678002408E0F5
:1032A00021462846FFF726FB0078FFF795FD641CB2
:1032B000E4B2B442F4D3002070BD0000E431000059
:1032C000034600205A681269002A01D018461047A8
:1032D000704700002DE9F843044606F017FA20B9BC
:1032E0002FA14FF4367000F0C5F93B4807F002F803
:1032F000002850D139490870486088604821384812
:10330000FEF717F9364848214830FEF712F93448DD
:10331000344D80304CB194E80E00103080E80E003F
:103320002F489030016821B105E005F12C010EC94C
:10333000F3E72D490160002006F03EFA30B1852800
:1033400004D017A240F20631FDF764FF274E002497
:103350000DE0002703E000783146FFF769FD3946AC
:10336000781CC7B24046FFF7C5FA0028F3D12146C2
:10337000641CE4B23046FFF7E5FA5FEA0008E8D1E2
:10338000686800906946304601F03AF8040004D0BD
:1033900007F0BCF92046BDE8F8830020FBE70000F9
:1033A0002E2E5C2E2E5C2E2E5C2E2E5C2E2E5C2E57
:1033B0002E5C636F6D706F6E656E74735C6C6962AA
:1033C0007261726965735C757362645C6170705F71
:1033D000757362642E6300003D3100008C01002093
:1033E000AC140020D0EB0000C92E00008CEC0000D3
:1033F00040B1012808D0022809D007A140F20E20D0
:1034000000F038B9124804E01148001D01E01048EE
:103410000830FFF753BD00002E2E5C2E2E5C2E2EA2
:103420005C2E2E5C2E2E5C2E2E5C636F6D706F6E8C
:10343000656E74735C6C69627261726965735C75E8
:103440007362645C6170705F757362642E63000008
:10345000EAEB000010B506F099FF10B106F08CFF02
:1034600008B1082010BD054806F0B6F920B104A245
:103470004FF45871FDF7CEFE002010BDF8EB0000B0
:103480002E2E5C2E2E5C2E2E5C2E2E5C2E2E5C2E76
:103490002E5C636F6D706F6E656E74735C6C6962C9
:1034A0007261726965735C757362645C6170705F90
:1034B000757362642E63000010B506F05DFF20B9DD
:1034C00009A140F2763000F0D5F815480168C1F343
:1034D000400121B1BDE810401248FFF7EFBC016880
:1034E00011F0010FF2D110BD2E2E5C2E2E5C2E2E6F
:1034F0005C2E2E5C2E2E5C2E2E5C636F6D706F6EBC
:10350000656E74735C6C69627261726965735C7517
:103510007362645C6170705F757362642E63000037
:1035200038040040D5EB0000034808B580680090DF
:103530006846FFF7C3FC08BDD0EB0000074918B18F
:10354000052803D30020704708687047044A105CC0
:103550000028FAD051F8200070470000C401002074
:1035600018ED0000092808D2DFE800F0070705077A
:103570000705050505000120704700207047092850
:1035800008D2DFE800F0070705070707070705006F
:10359000012070470020704710B509F0E9FD0128AF
:1035A00003D004A11D2000F065F8BDE8104000F034
:1035B0004FB800002E2E5C2E2E5C2E2E5C2E2E5C24
:1035C0002E2E5C2E2E5C636F6D706F6E656E747345
:1035D0005C6C69627261726965735C7574696C5C5C
:1035E0006170705F7574696C5F706C6174666F7226
:1035F0006D2E630010B509F0BBFD012803D004A1B6
:103600002B2000F037F8BDE8104000F029B800008A
:103610002E2E5C2E2E5C2E2E5C2E2E5C2E2E5C2EE4
:103620002E5C636F6D706F6E656E74735C6C696237
:103630007261726965735C7574696C5C6170705FEE
:103640007574696C5F706C6174666F726D2E630067
:1036500072B602480168491C01607047D801002019
:1036600003490868401E086000D162B67047000038
:10367000D80100201CB56A46ADF800000191002178
:1036800044F20200FEF716FE1CBD102802D31038CB
:10369000C0B2704740F08000704700002DE9F0474D
:1036A0000546C61C90460F464FF001090020FFF763
:1036B00073FF1B4C20683860D4E90001401AA168F0
:1036C00004F21C47081A0EE00121384604F046FEB9
:1036D00004F062FA0146384604F040FED4E90001E5
:1036E000401AA168081A401C8642EDD8B8F1000FB4
:1036F00003D0052065F3891002E0062065F39F5092
:10370000A2682168114004EB8101C8602068304440
:1037100020600020FFF76EFF4846BDE8F0870000FC
:103720006419002030B482680468531C8360A1547B
:10373000D0E901128A4202D330BC07F05DB830BC38
:1037400070470000034803C8814201D1012070473F
:1037500000207047641900204360CA699A420DD363
:103760008A690260886918448861086F184408678C
:10377000C869C01AC86100D00120704701F1280251
:10378000026000208B67704710B5040003D1064922
:103790003920FFF76FFF206818B903493A20FFF777
:1037A00069FF2068083010BD14FC000070B50C469D
:1037B000060004D1224940F2B720FFF75BFF24B98D
:1037C0001F494FF42E70FFF755FF207800250F2872
:1037D00033D2DFE800F033083333320C11323208D1
:1037E000323333333300304600F0D3FB26E021463A
:1037F00030460AF067F80FE0304602F054FC01460C
:10380000A0780025814219D00106E1784FF003002D
:1038100004D531B901210CE005460FE021B10129A1
:103820000CD00329F8D109E0304600F0C3FB05466F
:10383000002130460AF0BAFF00E00625284670BD98
:1038400014FC00002DE9FF5F05460198DFF8F093B6
:103850001F46017A89F800101646019800F042FBD5
:10386000804625B9F74940F2E920FFF703FF2968B0
:103870004FF0000A40F21F325446A1F21F304FF0C1
:10388000020B914256D04CDC40F20132A1F20130E1
:10389000914272D029DC40F2F120A1F2F122814262
:1038A0006CD015DC40F2EE22A1F2EE2391426ED0F4
:1038B00009DC4FF43B73E1B3994270D0A1F500717C
:1038C000ED395ED17AE0012B74D0022B59D19BE007
:1038D000092A70D004DC012A6ED0022A51D1B7E047
:1038E0000A2A6AD00F2A4CD1DDE00E2871D00EDCF6
:1038F00007286ED006DC01286CD005286BD006287E
:103900003FD116E10C2867D00D283AD138E115389F
:10391000092836D2DFE800F0F535353535F4F3F215
:10392000F10013286FD010DCA0F10300102828D27A
:1039300001E02EE079E1DFE800F0F0EFEEEDEC24BD
:1039400024EBEAE9E82424E7E6E537280CD00CDC90
:10395000292878D004DC142876D0282811D125E233
:103960002D2872D032280CD150E244286ED006DCCB
:103970003E286CD03F2804D16FE29FE04CE04928FC
:10398000F4D00020C5F800A004B0BDE8F09F24E00A
:1039900005E008212971002F01D82B607FE20EB1CC
:1039A000297931700B2101242971012F06D840F2A9
:1039B000ED2073E21CE059E03AE062E00EB12979B3
:1039C000315598F81410641C2971BC4205D32A6043
:1039D00065E2BAE07FE0A1E0C7E00EB12979315598
:1039E000641C85F804B0BC4202D340F2EF2055E2DB
:1039F0000EB129793155641C85F804B0BC4203D35B
:103A00004FF43C704AE2A6E10EB129793155641CAD
:103A100085F804B0BC42CCD20EB12879305598F864
:103A20001900641C2871BC4202D340F2F22035E236
:103A30000EB128793055641C85F804A0BC4207D328
:103A400040F2F3202AE2BCE191E1CDE117E2F9E195
:103A50000EB12879305589F801A0641C35E209209F
:103A60002871BC4202D340F2FA2017E20EB1287945
:103A700030550420641C2871BC4202D340F2FB2064
:103A80000CE20EB12879305599F80110641C0198A8
:103A9000FEF76CFFC9F8040000782871BC4202D31D
:103AA0004FF44070FAE10EB128793055641C85F866
:103AB00004A0BC4202D340F20130EFE10EB12879FC
:103AC0003055D9F80400641CBC424078287102D3F8
:103AD00040F20230E2E10EB128793055D9F8040005
:103AE00098F81410641C0078814233D185F804B032
:103AF000BC4213D340F20630D0E18BE07FE073E0AC
:103B000067E054E01BE10FE103E1F7E0EBE0DFE009
:103B1000D3E0C7E0B9E0ADE0A1E095E00EB12879CF
:103B20003055641C85F804B0BC4202D340F2073023
:103B3000B4E10EB12879305598F81900641C287149
:103B4000BC4202D34FF44270A8E10EB1287930553F
:103B5000641C25E098F8161081421CD10A202871B7
:103B6000BC4202D340F20D3098E10EB128793055B5
:103B7000641C85F804A0BC4202D340F20E308DE1F3
:103B80000EB128793055641C85F804A0BC42DCD302
:103B900040F20F3082E12B4940F21330FFF76AFD0B
:103BA00085F804A0BC4202D340F2163076E10EB193
:103BB00028793055D9F8040098F81410641C00785E
:103BC00081426ED105202871BC4202D340F21B30E5
:103BD00064E10EB1287930552420641C2871BC4260
:103BE00002D34FF4477059E10EB128793055641C67
:103BF00085F804A0BC4202D340F21D304EE10EB164
:103C0000287930551020641C2871BC4202D340F240
:103C10001E3043E10EB1287930550120641C287113
:103C2000BC4202D340F21F3038E10EB12879305542
:103C30000520641C2871BC4206D340F222302DE1DD
:103C4000A001002014FC00000EB12879305524207A
:103C5000641C2871BC4202D340F223301EE10EB135
:103C6000287930550120641C2871BC4202D34FF4DE
:103C7000497013E10EB1287930550320641C287176
:103C8000BC4202D340F2253008E10EB1287930550C
:103C900098F81600641C2871BC4203D340F2263009
:103CA000FCE069E00EB1287930550420641C2871CD
:103CB000BC4202D340F22930F0E00EB128793055F1
:103CC0002420641C2871BC4202D340F22A30E5E073
:103CD0000EB128793055641C85F804B0BC4202D37B
:103CE00040F22B30DAE00EB128793055641C85F8AB
:103CF00004B0BC4202D34FF44B70CFE00EB1287930
:103D000030550520641C2871BC4202D340F22F308C
:103D1000C4E00EB1287930552420641C2871BC42BF
:103D200002D34FF44C70B9E00EB12879305506201B
:103D3000641C2871BC4202D340F23130AEE00EB1B7
:103D40002879305598F81400641C2871BC4202D3BD
:103D500040F23230A2E00EB12879305598F81600C2
:103D6000641C2871BC4202D340F2333096E00EB19D
:103D700028793055641C08E098F81610814204D068
:103D800057494FF44F70FFF775FCD9F804104846B7
:103D9000497889F80210514689F803A08CE0072081
:103DA0002871BC4202D340F2473077E00EB1287947
:103DB00030550520641C2871BC4202D34FF4527068
:103DC0006CE00EB12879305599F80310641CD9F8CD
:103DD0000400FEF7A3FDC9F8080000782871BC4272
:103DE00002D34FF4537059E00EB128793055D9F809
:103DF000040098F81410641C007881420BD1032051
:103E00002871BC4202D340F2513047E00EB128790C
:103E10003055641C0FE098F81610814206D185F8E1
:103E200004B0BC42F2D340F2563037E02C4940F2A5
:103E30005A30FFF71FFC40202871BC4202D340F2E9
:103E40005D302BE00EB128793055641C85F804A054
:103E5000BC4202D340F25E3020E00EB128793055EA
:103E6000D9F8040098F81410641C007881420BD132
:103E700010202871BC4202D340F263300EE00EB134
:103E800028793055641C11E098F81610814208D149
:103E900085F804A0BC42F2D34FF45A702860012088
:103EA00072E50F494FF45B70FFF7E4FB99F80310DC
:103EB0004846491C89F803108278C9B29142FFF440
:103EC0006EAF4178491C89F8011099F8011099F8F2
:103ED00000008142FFF4C3AD40F27330DEE7000022
:103EE00014FC000010B5040003D103492C20FFF797
:103EF000C1FB204610BD000014FC000070B5054653
:103F0000144808F0ABF830B9134800684068D0E9AD
:103F1000002100209047402210491148FEF78CFBF9
:103F200038B1922815D0BDE870400E4A4B21FDF7FC
:103F300071B92846FEF7C8FB044602460749054802
:103F400008F042F88442DBD006494220FFF792FB9A
:103F5000D6E770BD0014010054020020B416002002
:103F600098EF00006406010010B508B1032010BDF1
:103F70000846FFF709FC0178202901D0062010BD72
:103F8000D0F80210C160C1880182017A81740020DA
:103F900010BD10B5FFF7A6FFFFF7F6FB00218182E9
:103FA00081610162C16601674167816700F1280193
:103FB000816610BD2DE9FC478146FFF793FFFFF7AF
:103FC000E3FB0446484602F03EFB07462F48002626
:103FD0008068CDE90004E069B0B1D4F87880454646
:103FE000404500D205462A4604F12801A069FDF7A4
:103FF00079FA206F2844C4E91C60A8EB0500E0664C
:1040000060192830A06627E0206F60672667E666A3
:10401000216A304621B1626AA161C4E907202CE01F
:10402000A06130E004F11802616A82E84300E26EA8
:104030001AB38A4215D3A36E0A461946FDF752FAFF
:10404000E16EE069091AE166A16E0144A16660674C
:10405000002148460AF0AAFB206A0028E2D1A661A6
:1040600011E0A16EFDF73EFAE06E2067E169091AE2
:10407000E161A1690818A06105D069463846FEF7DC
:10408000BDFEBDE8FC870020FBE700001CEC000043
:104090004360CA699A4204D38A6902600B67CB61A4
:1040A00003E001F1280202608B67002070470000E6
:1040B00070B5044681B1012905D002291CD1BDE8A3
:1040C0007040FFF71BBF0D4800684068D0E9002131
:1040D000BDE8704001201047FEF7F6FA054602469B
:1040E0000749084807F070FF854203D006496C2055
:1040F000FFF7C0FA2046E2E770BD0000540200203E
:10410000B4160020001401006406010002490844AE
:1041100090F9300070470000C813002070B5816826
:1041200004464A8B002A4DD0888B00284AD0121AA8
:10413000084495B200F120016A1C1F30FDF7D2F946
:10414000A068818B491E8183A068418B491E4183F1
:104150008DB308221C49206906F00EFB204604F0AE
:104160008AF88188C088814211D1A06817A2818B0A
:10417000431808212046203304F082FE204600F038
:10418000BDF929462046BDE8704002F029B9204615
:1041900000F020FA204600F0B1F9A0680BA2818B54
:1041A000431808212046203304F06AFE2046BDE86B
:1041B000704000F0D9B92069BDE87040044A03A1FD
:1041C00006F0DABA70BD0000FC4300002573000061
:1041D00064EF000070B504468068428B818B521AF0
:1041E00015042D0C48D0084400F121012A46203046
:1041F000FDF778F9A068418B491E4183204604F001
:104200003AF88188C08881420CD1A0681BA2818BBA
:10421000431808212046203304F032FE4FF4707614
:10422000C4B913E0204600F0D5F9204600F066F945
:10423000A06812A2818B431808212046203304F085
:104240001FFE2046BDE8704000F08EB90CA130463C
:10425000FFF710FA206918B909A13046FFF70AFAEA
:10426000154A06A1206906F087FA6D1EA9B22046FC
:10427000BDE8704002F0B4B870BD000025730000C6
:104280002E2E5C2E2E5C2E2E5C2E2E5C2E2E5C2E68
:104290002E5C636F6D706F6E656E74735C6C6962BB
:1042A0007261726965735C636C695C6E72665F6390
:1042B0006C692E630000000068EF00002DE9F041FA
:1042C000044680680F46D0F84813828B11F001062F
:1042D000418BA1EB02039DB24FF4BF730BD0994207
:1042E00001D9002D7ED0A068818B0844002180F880
:1042F000207066B113E099427CD8002DF3D083186A
:1043000003F120012A46481CFDF7ECF8EBE7A06812
:10431000428B521C92B24283A068203281544DB32A
:10432000204603F0A8FF8188C08881420ED1A06892
:1043300031A2818B431808212046203304F0A0FDD0
:10434000A81B81B2204602F04BF821E0204600F085
:1043500041F9A06828A2818B431808212046203308
:1043600004F08EFD204600F0FFF80121204602F007
:1043700049F90DE03EB1A068428B521C92B24283D3
:10438000A068203281543A461CA1206906F0F4F955
:10439000A168888B401C8883204602F00EF8002814
:1043A000204603D0BDE8F04102F026B803F076F8CD
:1043B00000281FD0204603F05EFF0546C088A9886C
:1043C000401A401E81B2204601F098FF204602F0BC
:1043D00013F8E888A988401A81B2204602F01EF935
:1043E000288800E006E0401E81B22046BDE8F0418A
:1043F00002F008B9BDE8F0812573000025630000D4
:1044000070B50D46040003D10BA1E120FFF732F98E
:10441000606818B908A1E220FFF72CF9606800680D
:1044200018B905A1E320FFF725F96068294602685D
:104430002046BDE8704010472E2E5C2E2E5C2E2E9E
:104440005C2E2E5C2E2E5C2E2E5C636F6D706F6E5C
:10445000656E74735C6C69627261726965735C75B8
:104460007362645C6170705F757362642E630000D8
:1044700009B10620704700207047000041680A60BB
:1044800041684B60014908600020704754020020D9
:1044900070B51C0015460E4603D10649A020FFF753
:1044A000E9F82A463146044807F0A0FE20600020C3
:1044B00070BD000064060100001401000020704778
:1044C00070B51C0015460E4603D10A49AD20FFF712
:1044D000D1F82A4631460848FEF7FBF838B10828DB
:1044E00005D0112802D100202060002070BD256079
:1044F000FBE700006406010098EF000070B50400BF
:104500004FF4B27503D108A12846FFF7B3F820692C
:1045100018B905A12846FFF7ADF82069BDE870403D
:104520000F4A10A106F028B92E2E5C2E2E5C2E2EDE
:104530005C2E2E5C2E2E5C2E2E5C636F6D706F6E6B
:10454000656E74735C6C69627261726965735C63D9
:104550006C695C6E72665F636C692E6300000000BC
:104560005CEF00002573000070B504004FF4B875CF
:1045700003D108A12846FFF77DF8206918B905A1E5
:104580002846FFF777F82069BDE870400F4A10A170
:1045900006F0F2B82E2E5C2E2E5C2E2E5C2E2E5C9B
:1045A0002E2E5C2E2E5C636F6D706F6E656E747355
:1045B0005C6C69627261726965735C636C695C6E84
:1045C00072665F636C692E630000000053EF0000A9
:1045D0002573000070B504004FF4B57503D108A130
:1045E0002846FFF747F8206918B905A12846FFF7C4
:1045F00041F82069BDE870400F4A10A106F0BCB830
:104600002E2E5C2E2E5C2E2E5C2E2E5C2E2E5C2EE4
:104610002E5C636F6D706F6E656E74735C6C696237
:104620007261726965735C636C695C6E72665F630C
:104630006C692E630000000050EF0000257300003D
:104640002DE9F04F4FF000099FB005464E464C460D
:10465000CDF8509001F0DAFC284603F04FF8A86836
:10466000CA464FF4C07100F5D070FCF762FFA8682D
:1046700000F12001428B00F5D070FCF733FFA868F1
:1046800000F5D07009F050FAA86800F5D07000F07D
:1046900037FCA968401CC883284601F03BFE284629
:1046A00001F08BFE10B9284601F0A6FEAA680C2383
:1046B00004A912A8203203F035FC0346129840B139
:1046C0005BB170A20221284604F0DAFB1FB0BDE8FE
:1046D000F08F284601F090FEF8E7704970480027F7
:1046E000A1EB00080DF1100B13E008D36DA00090B2
:1046F00071A202212846049B04F0C2FBE6E700EB0E
:10470000C704606801685BF82900FCF740FF20B12E
:104710007F1C6348B7EBD80FE7D9207820B168A198
:1047200040F68200FEF7A6FF4FF00008CDF870803B
:104730006068C7680FB1A9684860606809F1010442
:104740004FF0000980680390129884425CD25BF8B5
:10475000240069A1FCF71BFFD0B15BF8240067A11E
:10476000FCF715FFA0B15BF824000AF07BF8B8B1A4
:104770000020139013A800905BF8243022462846AE
:10478000039901F0D1FC02283ED013998A4439E004
:10479000A868D0F8481341F00201C0F8481333E08C
:1047A00018A84A46009009F101091CAB214603985C
:1047B00001F09EF9B9F1000F26D01C9820B30168D2
:1047C0005BF82400FCF7E3FE0028BDD11C98C1680B
:1047D000A1B1BAF1000F0BD0284601F09BFD28468D
:1047E00001F0EBFD10B9284601F006FE45A23CE0C1
:1047F000A9F10101DDF80C802646149180684FF084
:1048000000090390641C9FE7BAF1000F10D0A8685C
:1048100000F5D071C28B2030FCF764FEA9680C2330
:10482000C88B4883AA6804A912A8203203F07AFB37
:10483000B8F1000F12D018A800901CAB31464046CA
:10484000149A01F055F9A9681C980BEB8602486090
:104850001299C368891B284698470AE027B104AA21
:1048600028461299B84704E032A20221284604F0F3
:1048700007FBA868D0F8481321F00201C0F84813DC
:1048800024E700006E6F74207465726D696E617448
:1048900065643A2025630D0A0000000064120100DF
:1048A000D41101003A20636F6D6D616E64206E6FEC
:1048B0007420666F756E6400257325730D0A000001
:1048C0002E2E5C2E2E5C2E2E5C2E2E5C2E2E5C2E22
:1048D0002E5C636F6D706F6E656E74735C6C696275
:1048E0007261726965735C636C695C6E72665F634A
:1048F0006C692E63000000002D6800002D2D686596
:104900006C7000004572726F723A20726571756545
:1049100073746564206D756C7469706C6520667560
:104920006E6374696F6E20657865637574696F6E08
:10493000730D0A00506C656173652073706563695F
:104940006679206120737562636F6D6D616E642E90
:104950000D0A00008068D0F84803C0F3C00070471B
:104960002DE9F0410446C0688EB00D460026C068AF
:10497000324601A907F0BAFA18B100200EB0BDE81E
:10498000F0816DB1019806F0C2FFA168D1F838033B
:10499000401CC1F8380300F00700012879D1012636
:1049A000204603F068FC05468088012804D9401E93
:1049B00081B2204601F032FE2888012804D9401E29
:1049C00081B2204601F00CFD2046FFF797FD2EB185
:1049D00031A20221204604F053FA5AE04FF00108B8
:1049E00000230C2202A9019806F0A0FF049805906C
:1049F000BDF80C00ADF81800BDF80E00ADF81A00B7
:104A00008DF81D8002980C2700F00300012802D0C9
:104A1000022818D032E002983B46860AC0F3C20052
:104A20008DF81C00029808A9C0F38315AA0001980C
:104A300006F07CFF2069009005AB2A4608A93046A5
:104A400006F0AAFE1AE00298850DC0F3C2008DF8A8
:104A50001C00082D01D22E4600E008263B463246B7
:104A600008A9019806F062FF3744AD1B05AA31463C
:104A700008A8236906F074FD002DEAD1019806F01C
:104A800046FFE068002201A9C06807F02FFA00285D
:104A9000A6D0012072E700004C6F7374206C6F6722
:104AA00073202D20696E637265617365206C6F677A
:104AB000206261636B656E64207175657565207336
:104AC000697A652E0D0A00002DE9F0411E46174651
:104AD0000D46040000D01DB909A1EA20FEF7CAFD69
:104AE000606818B906A1EB20FEF7C4FD6068334684
:104AF0003A4601680C692946A446BDE8F041604782
:104B00002E2E5C2E2E5C2E2E5C2E2E5C2E2E5C2EDF
:104B10002E5C636F6D706F6E656E74735C6C696232
:104B20007261726965735C636C695C6E72665F6307
:104B30006C692E630000000070B5044640680E46A4
:104B40000025007A38B1A0680068FDF7E3FC08B1E1
:104B500008281AD10025BEB96068007A50B90B4AFE
:104B60000021A068FDF76EFC616805004FF00100B0
:104B7000087209D1A068224640F6CD410068FDF7D1
:104B8000A5FC0546FCF7E4FF284670BD99DE000051
:104B900010B541680A6041684B60406800210172AD
:104BA000FCF7D6FF024901200870002010BD00006C
:104BB0005802002070B51C0015460E4603D106A110
:104BC0006620FEF757FD2A4631460020FCF7C2FF5B
:104BD0002060002070BD00002E2E5C2E2E5C2E2E3C
:104BE0005C2E2E5C2E2E5C2E2E5C636F6D706F6EB5
:104BF000656E74735C6C69627261726965735C6323
:104C00006C695C7274745C6E72665F636C695F720F
:104C100074742E630000000080680068FDF77ABCA1
:104C20002DE9F05F5FEA030815460E4603D11DA18A
:104C30007420FEF71FFD2B480068C0070FD0DFF877
:104C4000A8B000244FF0050AB14600BF09EB0401EB
:104C50002A460020FCF7CCFF060003D011E0C8F87C
:104C6000005018E09BF8000088B10A271F494FF454
:104C70007A4088477F1EF9D1AAF101005FEA000A55
:104C80000CD001218BF800103444AD1BDED1002C78
:104C9000E5D0C8F800400020BDE8F09F00218BF867
:104CA0000010F4E72E2E5C2E2E5C2E2E5C2E2E5C39
:104CB0002E2E5C2E2E5C636F6D706F6E656E74733E
:104CC0005C6C69627261726965735C636C695C7269
:104CD00074745C6E72665F636C695F7274742E6369
:104CE00000000000F0ED00E058020020E1EF0000BD
:104CF0007CB500260446019601AB01226946204698
:104D0000FFF7E2FE019800281CD09DF800007F28E4
:104D1000F2D807F0D9F8A068417821B1012964D010
:104D2000022966D16AE0217E9DF80050A9420DD18A
:104D3000408B0028204606D0FFF782FC0221204647
:104D400000F0CAF87CBD01F057FBF7E7092D1CD035
:104D500004DC002DD0D0082D04D11FE01B2D12D073
:104D60007F2D24D0FCF766FB0068405D10F03E0FFD
:104D7000C2D02046FFF7EEFD9DF8001000B320469C
:104D8000FFF79CFAB8E7012136E02046FFF7E2FD85
:104D90000028B1D0204600F0B9F8ADE72046FFF773
:104DA000D9FD0028A8D02046FFF7B8F9A4E720468F
:104DB000FFF7D0FD00289FD02046FFF70BFA9BE7B6
:104DC000A268508BB0F5BF7F96D8908B1318401C0B
:104DD000908383F82010A068818B084480F82060BD
:104DE000A068418B491C418386E79DF800105B2930
:104DF00001D0002100E0022141707DE700214170D7
:104E00002046FFF7A7FD00289CD09DF80000413800
:104E10000C28B7D2DFE800F007090E2D064C06502B
:104E20000606065468E7012100E00021204602F052
:104E300049FB61E7204603F01EFA054600886988B1
:104E4000884203D1A988EA8891429BD06989884227
:104E50004FF00101204606D101F050FA6989204641
:104E600001F0BEFA01E001F0CDFBA068818B491C86
:104E700015E0204603F0FFF905460088297B491C10
:104E8000884202D1A988012987D001284FF0010169
:104E9000204606D001F0A4FAA068818B491E8183C8
:104EA0002AE701F0BBFB6989204601F0ABFBF3E781
:104EB000204601F02FFA1FE7204601F054FA1BE7C5
:104EC000A068D0F8482301219143D0F8482361F32A
:104ED0000002C0F848230FE78268022911700CD144
:104EE0008268002182F82010826891838268518351
:104EF00002A20321036803F0C3BF704725730000BB
:104F0000002801D0FCF73CBB704700002DE9F04FB2
:104F1000A5B04FF000080546CDF83480CDF83080BC
:104F200080684746418BA1F27F11494289B25FEA0E
:104F3000010B71D0828B00F1200100F5D070FCF7DD
:104F4000D1FAA8680024818B084480F8A041FCF7BE
:104F500071FA20900168A8680C23828B0244D27FEA
:104F6000895CC0F84443AA6801F001090EA91FA892
:104F700002F5D07202F0D6FF0E98FFF7C1FF86B29D
:104F8000A2460A9407941F9921B101EB0900401E23
:104F9000B8426BD8B9F1000F01D0002605E00EA889
:104FA00050F82700FFF7ACFF86B200241BA822466A
:104FB0000090641C0AAB3946504600F099FD0A98EF
:104FC00000287CD001680EA8324650F82700FCF774
:104FD000F5FA0028079802D00028E7D06FE0E0B18A
:104FE0000A980068FFF78CFF0C9980B2884200D9BC
:104FF0000C90BBF1000F2BD021A8009007AB4246CC
:105000003946504600F074FD0A98006883190798E5
:1050100000688119002015E042E0601E0D900A989A
:105020000068FFF76DFF80B20C90801B58450FDAC7
:1050300080B20CE011F800C0624506D1401C0004AB
:10504000000C10D01A5C002AF4D1834500D98346A5
:105050000A98B4F101080790A8D267A20421284653
:1050600003F00EFF2BE04FF6FF70EEE700241BA8C5
:1050700022460090641C0AAB3946504600F038FDC9
:105080004CB10A9800280BD00EA850F8270009F060
:10509000E9FBA0B907E058A20421284603F0F0FE7E
:1050A00025B0BDE8F08F0A9801680EA850F82700D7
:1050B000FCF76DFA0028DAD10A98D0F808A0BAF106
:1050C000000F09D00A9838B11F997F1CBFB201EBBD
:1050D00009008742FFF457AF07980028E0D00D98E9
:1050E0004146404556D19AF8000038B11BA80A46FF
:1050F000009007AB3946504600F0FAFC079800686C
:10510000FFF7FEFEB04206D007985A4600688119A4
:10511000284601F06FF820980368A868818B421830
:1051200092F820209A5CD20715D0408B8142B7D2EA
:10513000284603F0A0F8A9688488888B401C8883DF
:10514000284603F098F88088A0421FD10121284604
:1051500001F058FAA4E7D0F84813C90711D0D0F8E5
:10516000481321F00101C0F8481320212846FFF719
:10517000A5F8A868D0F8481341F00101C0F8481319
:105180008EE720212846FFF799F889E7284601F0A5
:1051900033F985E7002128460C9A07F033FF0DF11B
:1051A0006C090D9C0EE00AAB224639465046CDF8FC
:1051B000009000F09DFC0A980C9A0168284607F0C0
:1051C00021FF641C4445EED917A2032128462B6811
:1051D00003F056FEAB6816A208212846203303F0E0
:1051E0004FFE284601F0D8F907985A460068811901
:1051F000284600F0FFFF53E75461622066756E6336
:1052000074696F6E3A20636F6D6D616E64732063B5
:105210006F756E746572206F766572666C6F7765F8
:10522000642E0D0A000000000D0A25730000000026
:105230002573000070B505460C0004D107A14FF49A
:105240001260FEF717FA002D06D0A068D0F84813B8
:1052500041F02001C0F8481370BD00002E2E5C2ED6
:105260002E5C2E2E5C2E2E5C2E2E5C2E2E5C636F02
:105270006D706F6E656E74735C6C69627261726979
:1052800065735C636C695C6E72665F636C692E63E8
:105290000000000000238B540A460068194603F002
:1052A000EFBD00002DE9F8431F461446884605006F
:1052B00002D0B8F1000F03D11EA1BB20FEF7DAF92E
:1052C0006868006818B91BA1BC20FEF7D3F9002656
:1052D00028E000BF686808EB06016B460268D2F858
:1052E0000CC02246E04718B112A1C620FEF7C2F951
:1052F0000098844203D20FA1C720FEF7BBF90098A3
:105300000644241A70B9A868017803290AD000BF9E
:10531000D0F848138906FBD5D0F8481321F02001B6
:10532000C0F84813002CD5D1002F01D00098386068
:10533000BDE8F8832E2E5C2E2E5C2E2E5C2E2E5C6D
:105340002E2E5C2E2E5C636F6D706F6E656E7473A7
:105350005C6C69627261726965735C636C695C6ED6
:1053600072665F636C692E630000000070B5084CC4
:10537000050009D010342168002907D00868206092
:10538000496828468847F6E70834F4E770BD00000E
:105390007C110020054A012120B1012805D191701E
:1053A000FFF7E4BF51700020FAE770477C1100203E
:1053B0003EB5044603F038FF38B103B02046BDE8DF
:1053C00030400022114603F0B9BD06490648CDE938
:1053D00000010346029105A20821204603F050FD7A
:1053E0003EBD000078050100001000004170706CA7
:1053F00069636174696F6E20616464726573733A86
:1054000025642028307825303858292C2073697A73
:10541000653A2025642028307825303858290D0A2F
:1054200000000000F8B514460E46050004D121A185
:105430004FF48770FEF71EF9A86818B1686808B1C4
:10544000286820B91BA140F20F10FEF713F9012EB6
:1054500003D0284603F0E2FE30B12846BDE8F8400C
:1054600001221B4903F06ABD022E08D0236801B057
:105470002846BDE8F04017A2022103F001BD1CA19F
:105480006068FCF784F868B11AA16068FCF77FF8DF
:1054900040B16068009019A202212846236803F0F9
:1054A000EFFCF8BD2846BDE8F8401BA2082103F038
:1054B000E7BC00002E2E5C2E2E5C2E2E5C64656DEB
:1054C0006F5F636C695F636D64732E63000000003F
:1054D00000EA000025733A20626164207061726105
:1054E0006D6574657220636F756E740D0A0000003F
:1054F0002D7400002D2D74657374000025733A20FF
:10550000756E6B6E6F776E20706172616D6574651C
:10551000723A2025730D0A0044756D6D792074650B
:105520007374206F7074696F6E2E0D0A0000000096
:10553000012904D0136804A2022103F0A1BC094987
:10554000002048607047000025733A2062616420A3
:10555000706172616D6574657220636F756E740D34
:105560000A00000008000020012904D0136804A2EA
:10557000022103F085BC0949012008707047000032
:1055800025733A2062616420706172616D65746593
:105590007220636F756E740D0A0000000800002011
:1055A000012904D0136804A2022103F069BC09494F
:1055B000002008707047000025733A206261642063
:1055C000706172616D6574657220636F756E740DC4
:1055D0000A0000000800002070B514460D4606467B
:1055E000012902D003F01AFE30B13046BDE8704008
:1055F0000022114603F0A2BC2368022D01D904A2A7
:1056000000E00AA23046BDE87040022103F038BC39
:1056100025733A2062616420706172616D65746502
:105620007220636F756E740D0A00000025733A20B6
:10563000706C65617365207370656369667920734A
:105640007562636F6D6D616E640D0A002DE9F04740
:1056500014460D46814603F0E1FD30B14846BDE8F1
:10566000F0470022114603F069BC022D07D04846DE
:105670002368BDE8F04728A2022103F001BCDFF84F
:10568000B48098F80100142801D32BA206E06068CA
:10569000FBF776FF86B2212E02D32DA2022132E043
:1056A000002567680AE000BFFBF7C4FE0068795D6B
:1056B000405C10F0380F2BD06D1CEDB2B542F3D327
:1056C000284E002505EB451030446168FBF75FFF6D
:1056D00000281FD06D1CEDB2142DF3D398F80110E3
:1056E000454601EB4110491C88F8011030441EA1C9
:1056F0006268FCF735FD1D4B212269781948FBF7DC
:10570000A3FE1BA208214846BDE8F04703F0B8BB42
:105710001FA2C3E72EA2C1E725733A20626164206D
:10572000706172616D6574657220636F756E740D62
:105730000A00000008000020636F6D6D616E642038
:105740006C696D697420726561636865640D0A0037
:10575000746F6F206C6F6E6720636F6D6D616E6428
:105760000D0A000004050020257300004DDC000038
:10577000636F6D6D616E6420616464656420737530
:10578000636365737366756C6C790D0A00000000C5
:1057900062616420636F6D6D616E64206E616D6522
:1057A000202D20706C6561736520757365206F6EA8
:1057B0006C7920616C7068616E756D65726963618A
:1057C0006C20636861726163746572730D0A000016
:1057D0006475706C69636174656420636F6D6D617D
:1057E0006E640D0A000000002DE9F84314460D46D2
:1057F000804603F013FD30B14046BDE8F843002277
:10580000114603F09BBB022D03D014A20221236892
:105810001DE00025184F194E09E000BF05EB4510AB
:1058200038446168FBF7B3FE70B16D1CEDB270785F
:105830008542F3D36068009011A20221404623689C
:1058400003F01EFBBDE8F883636814A2082101B0D1
:105850004046BDE8F04303F013BB000025733A2037
:1058600062616420706172616D6574657220636F3E
:10587000756E740D0A000000040500200800002069
:1058800025733A20756B6E6F776E20706172616D53
:10589000657465723A2025730D0A000064796E61A3
:1058A0006D696320636F6D6D616E643A2025730DC1
:1058B0000A0000002DE9F04117460C4680460129F8
:1058C00002D003F0ABFC30B14046BDE8F04100220D
:1058D000114603F033BB022C02D01BA23B6811E03F
:1058E0000024204E204D08E004EB44103044796839
:1058F000FBF74DFE60B1641CE4B268788442F3D3D8
:105900007B681AA24046BDE8F041022103F0B8BA14
:10591000132C14D06878001B00EB401204EB4410E9
:10592000304400F12101FBF7DDFD687816A2401E2E
:1059300068704046BDE8F041082103F0A1BA00209C
:1059400086F87302F1E7000025733A206261642053
:10595000706172616D6574657220636F756E740D30
:105960000A0000000405002008000020646964208B
:105970006E6F742066696E6420636F6D6D616E6416
:105980003A2025730D0A0000636F6D6D616E64200F
:1059900072656D6F76656420737563636573736696
:1059A000756C6C790D0A0000F8B514460D46074673
:1059B00003F034FC30B13846BDE8F840002211460F
:1059C00003F0BCBA012D08D0236801B03846BDE809
:1059D000F04013A2022103F053BA184D687838B191
:1059E00017A20821384603F04BFA00241A4E13E0A0
:1059F0003846BDE8F84019A2042103F041BA00BFBF
:105A000004EB44103044009023461DA20821384680
:105A100003F036FA641CE4B268788442F0D3F8BD2F
:105A200025733A2062616420706172616D657465EE
:105A30007220636F756E740D0A000000080000206C
:105A400044796E616D696320636F6D6D616E642072
:105A50006C6973743A0D0A0004050020506C65618E
:105A600073652061646420736F6D6520636F6D6D75
:105A7000616E64732066697273742E0D0A000000F3
:105A80005B2533645D2025730D0A000010B50446C4
:105A900003F0CAFB30B120460022BDE81040114699
:105AA00003F04CBA1F21BDE8104002A20320FBF70F
:105AB000B1BB00002E2E5C2E2E5C2E2E5C2E2E5C9A
:105AC0002E2E5C2E2E5C636F6D706F6E656E747320
:105AD0005C6C69627261726965735C636C695C635A
:105AE0006C695F7574696C735F636D64732E6300BA
:105AF0002DE9F05F1C000A9F15468846064603D133
:105B000021A1FF20FDF7B6FD27B91FA14FF480703A
:105B1000FDF7B0FD4FF00009B8F1000F0BD026B330
:105B2000307840B372683946284690473868E0B10B
:105B30002760BDE8F09F22492248A1EB0008B5EBA1
:105B4000D80F15D2DFF880A0002683460AE000BFF8
:105B50000BEBC607786801685AF82500FBF717FDBC
:105B600020B1761CB6EBD80FF2D301E0786808E0DC
:105B7000C4F80090DDE7706800EB051001680029AB
:105B8000F6D02060D5E700002E2E5C2E2E5C2E2E47
:105B90005C2E2E5C2E2E5C2E2E5C636F6D706F6EF5
:105BA000656E74735C6C69627261726965735C6363
:105BB0006C695C6E72665F636C692E630000000046
:105BC00064120100D4110100100300202DE9F041FE
:105BD00015460F46044603F027FB30B12046BDE8CA
:105BE000F0410022114603F0A9B90126214C7F1E85
:105BF0000ED0012F14D06068022F22D0002837D099
:105C000020881DA106EB0040BDE8F04105F074BC02
:105C1000606800282CD0208823A106EB0040F3E721
:105C20006068002824D00A2200216868FBF7D5FCB0
:105C30000246208821A106EB0040BDE8F04105F0B6
:105C40005FBC002814D00A220021A868FBF7C5FC1D
:105C500007460A2200216868FBF7BFFC024620883D
:105C60003B4606EB0040BDE8F0411AA105F04FBCF1
:105C7000BDE8F081F80400207465737420657272C9
:105C80006F72206D65737361676520776974682032
:105C90006D6F7265207468616E2033206172677564
:105CA0006D656E74730000007465737420657272A4
:105CB0006F72206D6573736167650000746573743E
:105CC000206572726F72206D6573736167653A202B
:105CD0002564000074657374206572726F72206DA4
:105CE0006573736167653A202564202564000000B0
:105CF0002DE9F04115460F46044603F095FA30B100
:105D00002046BDE8F0410022114603F017B90226F3
:105D1000214C7F1E0ED0012F14D06068022F22D09C
:105D2000022837D320881DA106EB0040BDE8F041D2
:105D300005F0E2BB606802282CD3208823A106EB83
:105D40000040F3E76068022824D30A220021686833
:105D5000FBF743FC0246208822A106EB0040BDE889
:105D6000F04105F0CDBB022814D30A220021A86817
:105D7000FBF733FC07460A2200216868FBF72DFC7D
:105D8000024620883B4606EB0040BDE8F0411CA1DE
:105D900005F0BDBBBDE8F081F804002074657374A4
:105DA000207761726E696E67206D657373616765D8
:105DB0002077697468206D6F7265207468616E2049
:105DC0003320617267756D656E74730074657374EA
:105DD000207761726E696E67206D657373616765A8
:105DE0000000000074657374207761726E696E67DD
:105DF000206D6573736167653A20256400000000BB
:105E000074657374207761726E696E67206D657357
:105E1000736167653A2025642025640010B5044647
:105E200003F0FCF930B120460022BDE810401146D5
:105E300003F084B8054A0721204603F021F82046E4
:105E4000BDE8104002A2082103F01AB844F6000091
:105E50002020202020202020202020202020202042
:105E60004E6F726469632053656D69636F6E64750C
:105E700063746F72202020202020202020202020EA
:105E800020200D0A0D0A0000F8B515460E46040044
:105E900003D117A12520FDF7EDFBA06818B16068BC
:105EA00008B1206818B912A12620FDF7E3FB012EE6
:105EB00003D0204603F0B2F930B12046BDE8F840E7
:105EC0000022114603F03AB8022E08D02B6801B028
:105ED0002046BDE8F0400DA2022102F0D1BF686863
:105EE000009011A2022120462B6802F0C9FFF8BDE4
:105EF0002E2E5C2E2E5C2E2E5C64656D6F5F636CA7
:105F0000695F636D64732E630000000025733A209F
:105F100062616420706172616D6574657220636F87
:105F2000756E740D0A00000025733A20756E6B6E55
:105F30006F776E20706172616D657465723A2025AD
:105F4000730D0A002DE9F04116460D46074601245F
:105F500008E000BF56F8243007A20821384602F0B6
:105F60008FFF641CAC42F5D33846BDE8F04103A274
:105F7000082102F085BF0000257320000D0A0000F3
:105F8000F8B516460D460746012409E056F82400E8
:105F90000090234604A20821384602F071FF641CD9
:105FA000AC42F3D3F8BD0000617267765B25645D97
:105FB000203D2025730D0A0001A2022102F060BFDE
:105FC0004E696365206A6F6B65203B290D0A0000EE
:105FD00010B5044603F028F930B120460022BDE890
:105FE0001040114602F0AABFBFF34F8F0548016869
:105FF000054A01F4E06111430160BFF34F8F00BF18
:10600000FDE700000CED00E00400FA052DE9F04189
:1060100085680646002495F82000002811D0A04687
:10602000FBF708FA0746006804F1200104F10104B7
:10603000695CA4B2415CC90705D0002CF4D185F895
:106040002080BDE8F081641E2404240C0FD0688BEE
:10605000021B04F12000291805F12000521CFBF757
:1060600041FAB168488B001B4883B1688883B268E5
:106070003D68538BD0181F300446002102E0491CB4
:1060800089B2401E0778EF5DFF07F8D18442D8D06F
:106090005B1A203302F80380B268508B401A508399
:1060A000B1688883CDE710B50021FCF75FFC0021C3
:1060B000FCF734FC007810BD2DE9F0410746154689
:1060C00088460846FEF71CFF84B2B868661CC18B80
:1060D0003144B1F5C07F07D9124A0421384602F095
:1060E000CFFE0020BDE8F081294600F5D070FBF717
:1060F0002BFA051EF6D0FEF703FF82B228192946B7
:10610000401C521CFBF7EEF9224641462846FBF79D
:10611000E9F920202855B868C18B3144C18301209A
:10612000E0E70000100601002DE9FF4F002787B0CF
:106130009A46DDF850B006463C46B84602250DF1B9
:1061400008090197DDE908013A467F1C01ABCDF84B
:106150000090FFF7CDFC019888B1016800225046FD
:1061600001F028F848B90198524601683046FFF717
:10617000A3FF5FEA000802D0641C002FE2D15CB3E9
:10618000CBF80040B0685546514600F5D070FBF79B
:10619000DBF904462846FEF7B3FE85B2C4B1B06809
:1061A00000F5D070A04206D214F8010C202802D1CC
:1061B0006D1CADB2641E2046FEF7A2FE421BB06805
:1061C000521CC18B491BC18361192046FBF78AF918
:1061D000B8F1000F01D0002500E001250BB02846E2
:1061E000BDE8F08F40684968884201D801207047B7
:1061F000002070472DE9F04115460F00044604D1F8
:1062000023A140F28650FDF735FAA068418B828BBE
:106210008B1A29449EB2B1F5C07F37D2002D35D0FC
:10622000104400F1200105F120021044721CFBF71C
:1062300059F9A0682A46818B084439462030FBF77B
:1062400051F9A0682030FEF75BFEA1681EA24883CA
:10625000A068818B431808212046203302F010FEED
:10626000A068818B29448183204600F0A6F818B9E4
:10627000204601F013F910B1204600F0BDF8002EC1
:1062800004D02046BDE8F04100F086B9BDE8F081B9
:106290002E2E5C2E2E5C2E2E5C2E2E5C2E2E5C2E38
:1062A0002E5C636F6D706F6E656E74735C6C69628B
:1062B0007261726965735C636C695C6E72665F6360
:1062C0006C692E630000000025730000EFF3058069
:1062D000C005C00D10D0103840B2002806DA00F01A
:1062E0000F0000F1E02090F8140D03E000F1E02031
:1062F00090F80004400970470F207047002904D02F
:106300000A46006901A104F037BA70471B5B256497
:106310004200000070B5054601F0ADFF044600885C
:106320006188884203D1A088E18888421AD0E18838
:10633000A088814204D9081A81B22846FFF7DEFFFF
:1063400020886188884205D9401A81B2284600F029
:1063500047F804E0081A81B2284600F053F9A8680B
:10636000418B818370BD70B5054601F084FF044602
:106370000188007B401C814202D1A08801281BD0EB
:10638000A088012804D9401E81B2284600F046F9B1
:106390002088217B884206D9401A401E81B22846B7
:1063A00000F01EF805E0081A401C81B2284600F0F3
:1063B00029F9A9680020888370BD10B504460068DB
:1063C000FEF79EFD0146A068828B408A1144B1FB16
:1063D000F0F200FB121008B1002010BD012010BD2A
:1063E000002904D00A46006901A104F0C5B970472C
:1063F0001B5B25644400000070B504004FF4BB75BE
:1064000003D108A12846FDF735F9206918B905A17F
:106410002846FDF72FF92069BDE870400F4A10A10A
:1064200004F0AAB92E2E5C2E2E5C2E2E5C2E2E5C35
:106430002E2E5C2E2E5C636F6D706F6E656E7473A6
:106440005C6C69627261726965735C636C695C6ED5
:1064500072665F636C692E630000000056EF0000F7
:10646000257300002DE9FC47002604468DF80460E2
:1064700080684FF4C07A3546B146B046514600F5C3
:10648000D070FBF756F84349206904F075F920698C
:1064900004F0B2F900276B46012201A92046FEF75D
:1064A00013FB0098D8B19DF804001B2806D0A16802
:1064B00091F8A0111B29EED152281FD0A26808F52F
:1064C000D071505408F101001FFA80F8B8F1090F9B
:1064D0000AD9A168042081F8A091BDE8FC872D4964
:1064E0004FF6C0100D31884700980028D3D17F1C8B
:1064F000BFB2B7F57A7FCED30D20EEE7A16808F5DD
:10650000D0704A4601F80090A16891F8A1015B287B
:1065100003D081F8A0210B20DFE7022057466FF05F
:106520002F0309E005EB850503EB4505401C654499
:1065300080B2ADB2B8420AD200F5D07C11F80CC0DE
:10654000BCF13B0FEED1401C80B2B84209D30C2005
:10655000C3E700BF06EB860603EB46066644B6B209
:10656000F1E700F5D07C11F80CC0BCF1000FF1D1BF
:10657000FA20FA2E01D9088100E00E81FA2D02D905
:10658000A168888101E0A0688581A06880F8A021C9
:106590000020A2E774EF000070B5054601F06BFE25
:1065A00004468088E188884201D1012600E0002667
:1065B0002846FFF702FF18B9284600F06FFF10B118
:1065C0002846FFF719FF1EB160882188401A12E0A3
:1065D000E088A188401A81B2284600F01FF8208880
:1065E0006188884206D9401A81B22846BDE87040C9
:1065F00000F008B8081A81B22846BDE87040FFF7DD
:10660000EFBE0000002904D00A46006901A104F091
:10661000B3B870471B5B256443000000002904D019
:106620000A46006901A104F0A7B870471B5B256406
:106630004100000010B50121FCF798F90021FCF79A
:106640006DF9007810BD10B50121FCF78FF901211B
:10665000FCF764F9007810BD10B50021024801F084
:1066600093FE80F3100010BD801D00204FF4A07237
:1066700002EB810189B200F099BC0068D0F80405F2
:10668000704700002DE9F04715460E46040003D17F
:1066900038492F20FCF7EEFF1EB936493020FCF7B1
:1066A000E9FF1DB933493120FCF7E4FF6079324935
:1066B000DFF8C480DFF8C49041F82050617908F118
:1066C000040808EBC100007958B1D9F80400082487
:1066D00002284CD3B9F80000022101EB004028A1A8
:1066E00043E035882768B5F5805F03D32DA1FD20F1
:1066F000FCF7C0FFC7F80855B67894F90450082E87
:1067000003D334A14520FCF7B5FF002D4FEA461016
:1067100006DA05F00F0101F1E02181F8140D03E024
:1067200005F1E02585F8000494F90410012201F038
:106730001F0302FA03F04909890001F1E021C1F8C1
:106740008002C1F80001617908EBC1010A71617929
:1067500048F83140D9F804000024032807D3B9F8D9
:106760000000032101EB004026A104F0C5FE2046F5
:10677000BDE8F0872CFD0000DC0100205004002063
:1067800052544320696E7374616E636520616C724C
:106790006561647920696E697469616C697A6564A0
:1067A0002E0000002E2E5C2E2E5C2E2E5C2E2E5CDB
:1067B0002E2E5C2E2E5C6D6F64756C65735C6E7234
:1067C00066785C68616C2F6E72665F7274632E68A7
:1067D000000000002E2E5C2E2E5C2E2E5C2E2E5CD9
:1067E0002E2E5C2E2E5C696E746567726174696F03
:1067F0006E5C6E7266785C6E7266785F676C7565EB
:106800002E6800005254433A20696E697469616CC5
:10681000697A65642E00000090F90400012100F0FF
:106820001F0291404009800000F1E020C0F80012F2
:1068300070470A46022100F0A5BB4FF4827100F0B8
:10684000B5BB000010B5040003D104496120FCF77A
:1068500011FF20680121016010BD00002CFD000027
:1068600010B5040003D104496720FCF703FF20683A
:106870000121416010BD00002CFD00002DE9F8430E
:10688000994616460F46050003D12E498620FCF78F
:10689000F1FE29684FF480344FF4A070BC4000EB47
:1068A000870080B226F07F46C1F808432968C1F806
:1068B0004843296800220A5008580090286800EBD5
:1068C0008701D1F84005C1F840652968D1F8041561
:1068D0001D4F401A20F07F404FF0040801280CD1D2
:1068E0007868042805D3398808EB014017A104F023
:1068F00003FE23494FF4046088472868C0F84443E6
:106900002968D1F80435F01A20F07F40020201D541
:1069100040F07F40C9F1000290420EDD02280CDCFD
:106920007868042806D33988324608EB014015A15F
:1069300004F0EDFD0D20BDE8F883C1F8044300200C
:10694000F9E700002CFD0000500400205254433AA7
:106950002044656C617920696E74726F647563653B
:10696000642064756520746F207269736B206F6694
:10697000207072652D666972696E672E00000000D6
:10698000A1ED00005254433A2057696E646F776559
:106990006420636F6D706172652073657420746923
:1069A0006D656F757420286162735F76616C7565C3
:1069B0003A25642C20636F756E7465723A256429DC
:1069C0002E00000070B50C00054604D10AA140F26B
:1069D0007510FCF74FFE0F48417800208D4209D218
:1069E0000D4AE06005EB4511A06011440BA0C4E91D
:1069F000001070BD206070BD2E2E5C2E2E5C2E2EE1
:106A00005C64656D6F5F636C695F636D64732E6357
:106A100000000000080000200405002053686F7784
:106A20002064796E616D696320636F6D6D616E6462
:106A3000206E616D652E00001FB514461A4AD061A4
:106A40000020019002900390886801908888ADF83A
:106A50000800086800F00302012A07D0022A15D0B6
:106A6000124940F27720FCF705FE1FBDC0F3C200BB
:106A70008DF80C000C4801AB2030009008682146CE
:106A8000C0F38312800A04F087FE1FBDC0F3C2006A
:106A90008DF80C000868044B810D203301AA2046B4
:106AA00004F05EFD1FBD0000600200202C0C010000
:106AB00010B50446010600F00F00092804D306A112
:106AC0004FF42B70FCF7D6FD6FEA0460C10F20462F
:106AD00061F31F1010BD00002E2E5C2E2E5C2E2E9A
:106AE0005C2E2E5C2E2E5C2E2E5C636F6D706F6E96
:106AF000656E74735C647269766572735F6E7266DC
:106B00005C757362645C6E72665F6472765F7573E7
:106B100062642E630000000070B50546000605F0B3
:106B20000F0402D5092C09D301E0092C08D307A1D1
:106B300040F29920FCF79EFD280601D5134801E09C
:106B40001248903800EB041070BD00002E2E5C2E11
:106B50002E5C2E2E5C2E2E5C2E2E5C2E2E5C636FF9
:106B60006D706F6E656E74735C6472697665727356
:106B70005F6E72665C757362645C6E72665F64728F
:106B8000765F757362642E6300000000201200209F
:106B900010B50446010600F00F00092804D303498C
:106BA0004FF41F70FCF766FD204610BDDCE30000CB
:106BB0002DE9FC4180461F4615460E4600240D482F
:106BC00001F0C9FB38B11120BDE8FC8106EB0430AF
:106BD00005F036F9641CAC42F8D1064801F0B2FB6E
:106BE000CDE90057334600220221404600F0AEF9BD
:106BF0000020E9E75C02002010B507F0C9FB802007
:106C0000FFF78AFF817B0124032902D00068002856
:106C100009D18020FFF74CFF8440E143BDE81040DC
:106C2000014801F0A1BB10BD38010020812005F012
:106C3000C5BD822005F0C2BD832005F0BFBD842004
:106C400005F0BCBD852005F0B9BD862005F0B6BDB8
:106C5000872005F0B3BD882005F002BE38B507F0E7
:106C600097FB0020FFF758FF817B0124032905D003
:106C7000006868B1BDE8384003F0A5BB0020FFF70D
:106C800017FF8440E143BDE838400A4801F06CBB7F
:106C90000020FFF70DFF8440E143064801F064FB4C
:106CA00005480449C0680C3900904968684688471F
:106CB00038BD000038010020D0EA0000012005F0B6
:106CC00011BE022005F00EBE032005F00BBE04200D
:106CD00005F008BE052005F005BE062005F002BE41
:106CE000072005F0FFBD000038B5082407F050FB71
:106CF0002046FFF711FF817B032915D0006800288B
:106D000012D12046FFF7D4FE01218140C943074834
:106D100001F02AFB06480549406900900C398DF8BE
:106D2000024049686846884738BD000038010020A5
:106D3000D0EA000070B5154804680460BFF36F8F97
:106D4000BFF34F8FBFF36F8FBFF34F8F03F088F9FF
:106D500038B10F48016921F0011201F0011114430B
:106D6000016101266CB194FAA4F0B0FA80F52846CE
:106D7000FCF78BFC06FA05F18C43294607F0A4FCCE
:106D8000F0E7BDE8704007F049BB00006C740240BA
:106D90002C01002010B5054CA078FFF789FE0146B4
:106DA000A078BDE8104007F08FBC00002C01002047
:106DB000F8B51A4800681A4DC6B2A878FFF778FEF1
:106DC000012404FA00F12889EA68C04380B2104324
:106DD000014202D0A87807F0EFFB06F08000A8700F
:106DE0000020FFF765FE04FA00F68020FFF760FE42
:106DF00004FA00F006430A48F1430C3001F0B4FAFB
:106E00008020FFF755FE8440A86804430548AC6025
:106E1000006A0090696868468847F8BD807402403F
:106E20002C010020D0EA000038B5002000900B486B
:106E30000068ADF802008820FFF73AFE012505FA48
:106E400000F40820FFF734FE054985402C4388688C
:106E500004438C6049686846884738BD2075024005
:106E60002C01002070470000F8B51C480568284632
:106E700005F0E0FDBFF36F8FBFF34F8F184E194C35
:106E8000E80506D501206070706A00906168684668
:106E90008847A8054FF0000705D56770B06A0090D5
:106EA000616868468847680516D56078002813D061
:106EB00005F0CAFD20B10CA140F2C540FCF7DAFB99
:106EC0006770194901200860582005F0C5FDF06A77
:106ED0000090616868468847F8BD00000074024071
:106EE000D0EA00002C0100202E2E5C2E2E5C2E2ECF
:106EF0005C2E2E5C2E2E5C2E2E5C636F6D706F6E82
:106F0000656E74735C647269766572735F6E7266C7
:106F10005C757362645C6E72665F6472765F7573D3
:106F200062642E630000000008750240054908B540
:106F3000002048708870044840680090496868469E
:106F4000884708BD2C010020D0EA00002DE9F0435D
:106F500087B00446DDE90E8980681D4616460F4657
:106F600000280BD018216846FAF7E3FA02A88DF83A
:106F7000007080E86003A1686846884707B0BDE8F4
:106F8000F083000070B516460C46050003D1064993
:106F9000B920FCF76FFB2868C0F84443002E02D0EC
:106FA0002868C0F8044370BD2CFD000038B50C46BD
:106FB000050003D10749CA20FCF75CFB286801598A
:106FC00029B10021015100590090012038BD002055
:106FD00038BD00002CFD000010B58168D1F84813C1
:106FE000C1F3400119B10022114601F0A7FFBDE82D
:106FF000104004F0ABB8000010B5134804F0BCF822
:1070000018B1124AFD21FAF705F90221104803F0E0
:10701000BBFF012414EBE07003D10C4A2102FAF704
:10702000F9F80B48032144720C3003F0ADFF14EB68
:10703000E07004D1054A40F20711FAF7EBF8044872
:107040000C30447210BD000060F00000A87E00000B
:10705000100000203EB505468068D0F84803C0F314
:10706000400020B100221146284601F067FF0020B1
:107070000290012400906A4601A902A804F0A2F837
:1070800038B1002C04D006A20221284601F0F8FEF7
:107090003EBDDDE900212846FFF7CEFC0024EAE7EB
:1070A000466C617368206C6F6720656D7074790D34
:1070B0000A0000007CB505468068D0F84803C0F39C
:1070C000400020B100221146284601F037FF14A2EB
:1070D0000821284601F0D4FE164C4FF48056230BAD
:1070E0001B0315A208212846009601F0C9FE200BBB
:1070F0001D4C40421DA2216901EB0031CDE9001673
:10710000642041430B0B0821284601F0B9FEA36916
:1071100002B02846BDE8704020A2082101F0B0BEB0
:10712000466C617368206C6F67207374617475734B
:107130003A0D0A007725010009092D204C6F636183
:1071400074696F6E2028616464726573733A2030CD
:1071500078253038582C206C656E6774683A202585
:1071600064290D0A000000006002002009092D209A
:1071700043757272656E742075736167653A256434
:10718000252520282564206F6620256420627974D7
:1071900065732075736564290D0A000009092D20A7
:1071A00044726F70706564206C6F67733A20256459
:1071B0000D0A00004023AFF300802DE9F04716468A
:1071C0000C4605005BD0ACB3B3F1010902D2032039
:1071D000BDE8F087884615F8010B314600F0A3F8AA
:1071E000C7B23F2F11D003DC3FB12A2F7DD122E05F
:1071F0005B2F69D05C2F78D182E0F00602D5207831
:107200002F283ED02078A8B9E2E7207890B12F2827
:1072100002D02E2803D06DE0B00730D46AE07007AA
:1072200068D544452BD0B00764D514F8010C2F283D
:1072300025D05FE023E0287801E015F8010F314602
:1072400000F071F8C0B22A28F7D021782E2909D190
:10725000710707D5444512D0B10703D514F8011CB6
:107260002F290CD010B12F280DD023E0B00708D55E
:10727000F00606D42F212046FAF778F908B101204C
:10728000A6E70020A4E7B00714D52F212046FAF77F
:107290006DF904009FD1F2E74B464246214628464D
:1072A000FFF78BFF012893D12F2F01D1B007E6D430
:1072B000641C01E026F004082078314600F033F821
:1072C00010F0FF07E8D1DAE720780028D7D02F2880
:1072D00001D1B107D3D4314600F025F8014632463A
:1072E000284605F0EBFF002800E014E0C7D0411C61
:1072F00002D00546641C6EE720785B28BFD1F9E711
:10730000F00708D115F8010B314600F00CF810F029
:10731000FF0700D16D1E14F8010B314600F003F891
:10732000B842E8D0ABE710B5044608070AD5FAF72B
:1073300081F80068005DC00604D52046BDE8104015
:10734000FAF77CB8204610BD2DE9F05F17460E0015
:10735000814670D013B1B9B2FFF754F90024FAF79F
:1073600069F88246006800E0641C315D415CC90731
:10737000FAD100253046FDF7C3FDD9F80810001BEF
:107380004A8AD11B814228D306EB040805E000BFDE
:1073900018F805100A290CD06D1C8542F8D3311954
:1073A000D9F8100003F0E8F94846BDE8F05FFFF7B0
:1073B00023B8D9F8100003F01FFA414600232A46EB
:1073C0004846FDF76FFF2C444846641CFFF714F84D
:1073D000B9B24846FFF716F9E1E78B46DAF8001034
:1073E00006EB040818F805000B5CDB0702D0AB467F
:1073F0000A2804D0E819904201D26D1CF2E7D9F8AE
:10740000100003F0F9F9414600235A464846FDF7BB
:1074100049FF5C44DAF8000000E0641C315D415C27
:10742000C907FAD14846FEF7E7FFB9B24846FFF769
:10743000E9F89EE7FFE7BDE8F09F000010B50446BD
:1074400014480021027862B1012A09D12278022A67
:1074500006D1114AA3686FF30B02934200D1017069
:1074600010BD2278012AFBD162684AB18169491CAA
:10747000816160690028F3D0BDE8104004F047BA8C
:10748000D0E904231A44C0E904210021406800F037
:1074900035FBEEE7600200207725010010B50446B9
:1074A0000068FDF72DFD0146A068428B408A11441B
:1074B000B1FBF0F200FB121008B1002010BD01205A
:1074C00010BD0000FEB50026044600960196029607
:1074D0008068E9B3D0E9D0128A4273D0D0F83C0377
:1074E00000286FD02046FEF73EFFA068D0F8445336
:1074F000002D6AD000230A226946284604F016FAB5
:10750000A168BDF808500098C1F84403A0680023A2
:107510000A22D0F84403694604F008FAA168BDF8CD
:1075200008200A23D1F844032031521C04F0FEF94C
:10753000A168BDF808008883A168BDF808004883E9
:10754000BDF80800A84202D22046FCF7D7FF00E0B1
:107550000BE0A3682CA208212046203301F090FC08
:107560002046FEF72AFF70BB45E0D0F84403002810
:1075700049D02046FEF7F7FEA06800230A22D0F883
:107580004403694604F0D2F9A0680199C0F8441395
:10759000A0680029458BB9D100F5D070FDF7B0FC8B
:1075A0000028A06805D000F5D0712030F9F7FDFF64
:1075B00001E080F82060A0682030FDF7A1FCADF864
:1075C0000800B5E71FE01BE0FFE72030FDF798FC5F
:1075D0000504A0682D0CD0F83C13C0F84413A06833
:1075E00006D000F1200100F5D070F9F7DEFF8DE73D
:1075F00080F8A0618AE72046FFF750FF002802D0FC
:107600002046FEF7F9FEFEBD25730000FEB50D0015
:10761000044604D11E4940F2DD40FCF72BF8A16876
:107620000026D1F83C0338B300230A22694604F04F
:107630007DF90195A06800230A22D0F83C03694631
:1076400004F07AF90196A068D0F83C130091408BC1
:10765000ADF80800A068C0F83C5300230A22694630
:10766000284604F069F9A1680A2328464A8B20318C
:10767000521C04F061F9FEBDC1F83C53A068C0F88B
:10768000405300960196A068408BADF80800E4E7EF
:10769000C8DD0000FEB504468068D0F84063002EC7
:1076A00028D000230A226946304604F03FF9A16839
:1076B00001980025C1F84003009501952B460A2248
:1076C00069463046029504F037F9304604F000F977
:1076D000A168D1F8400370B100230A22694604F082
:1076E00025F90095A06800230A22D0F840036946D6
:1076F00004F022F9FEBDC1F83C53FEBDFEB50446C0
:1077000080682030FDF7FCFB0504A0684FF0000600
:107710002D0CC0F8446333D0A068D0F83C03E0B12E
:1077200000230A22694604F001F9BDF80820AA42A4
:1077300013D1A0680A2300F5D071D0F83C03521C85
:1077400004F0F4F8A06800F5D0712030F9F71FFFBD
:107750000028A06880F8A06112D000260B352946C9
:10776000606904F085F80100204604D003B0BDE84C
:10777000F040FFF74BBFFFF78DFF761C082EEED3CE
:10778000FEBD0000014941600020704754F0000038
:107790002DE9FC5F0E008346DDE90C47C6F10000D1
:1077A00098469246814600D40846012503E000BF72
:1077B00090FBFAF06D1C5045FADAA84500D9454611
:1077C00024B1002E01DB780700D5641EB80702D56E
:1077D000B8F1000F0AD0F80708D13CB1A54205D294
:1077E00020215846641EFBF79DFFF6E7002E02DAC3
:1077F0004E462D2102E0780703D52B215846FBF792
:1078000091FF07F0030002280BD1B8F1000F08D157
:107810003CB1A54205D230215846641EFBF782FFD9
:10782000F6E7CDE90047434652463146584606F052
:1078300099FCBDE8FC9F000010B5024600201268CC
:10784000930702D0530702D410BD500719D502F098
:107850000300012807D002280BD00D494FF4917086
:10786000FBF708FF0BE0C2F383100B68C01C184441
:1078700004E00323086803EB9252104408600120DF
:1078800010BD086800EB9253C2F38910401CEEE76C
:10789000800C010002480068002800D001207047D9
:1078A0005C0200200268134602E08A4204D012689B
:1078B000002AFAD10B600160704700001CB5012955
:1078C00005D08168D1F84813C1F3400131B102B04D
:1078D0000022BDE81040114601F030BB536804A1FE
:1078E000CDE90013136808A2022101F0C9FA1CBDFA
:1078F00020756E6B6E6F776E20706172616D65744E
:1079000065723A200000000025733A257325730D37
:107910000A0000002DE9F74F82B0154602980F00CB
:107920004FF00006C068007A009058D0072248A1A6
:107930002868F9F743FE78B1082247A12868F9F7CB
:107940003DFE002830D02B6845A2029805B00221E8
:10795000BDE8F04F01F094BA012F02D0022F08D0F9
:1079600008E0029805B044A2BDE8F04F022101F002
:1079700087BA0126DFF81881002400BF58F82410C8
:107980000A226868F9F71AFE10B1641C052CF5D3B9
:10799000052C06D004F0FF090224002E54D0002448
:1079A00019E03CA26B68D0E7012F4FF00009F6D038
:1079B000012449E04A462146009800F0E6FB48B918
:1079C0000021204603F0C6FE03463AA20221029897
:1079D00001F056FA641C03F06BFEA042EAD805B031
:1079E000BDE8F08F4FF0000A55F824B003F060FEB8
:1079F0008046002609E00021304603F0ABFE20223D
:107A00005946F9F7DBFD90B1761C4645F3D3464560
:107A100006D155F8243030A20221029801F030FA44
:107A20004A465146009800F0B0FB10B10BE0B24658
:107A3000EDE70021504603F08DFE03461DA2022112
:107A4000029801F01DFA641CBC42CBD3C7E70000CA
:107A5000656E61626C65000064697361626C6500EB
:107A6000556E6B6E6F776E206F7074696F6E3A2013
:107A700025730D0A0000000042616420706172618C
:107A80006D6574657220636F756E742E0D0A00004B
:107A900098020020556E6B6E6F776E207365766569
:107AA00072697479206C6576656C3A2025730D0ACD
:107AB000000000004C6576656C20756E617661692A
:107AC0006C61626C6520666F72206D6F64756C65A9
:107AD0003A2025730D0A0000556E6B6E6F776E208D
:107AE0006D6F64756C653A25730D0A00C0680121DD
:107AF00041727047C0680021417270477CB50D46E5
:107B00000646214C26E040201F4A606114321F497E
:107B1000019800F075FBE8B101980090D4E90413D6
:107B20001A4A1B4803F0A8F808B155B10BE0002D24
:107B30001BD0D4E9040108442061019803F0E7FE5A
:107B400008E0042812D0102817D0124940F217106C
:107B5000FBF790FD002201A9304604F0C7F9002888
:107B6000D1D009480C3000F0EDFB7CBD019803F04A
:107B7000CEFEA069401CA061F3E7019803F0C7FEA8
:107B800001202070E6E7000060020020541700206A
:107B9000580300202C0C01002DE9FF410026264847
:107BA00000F0D6FB2448001F074600F0D1FB234C11
:107BB00060680090A56800E000986946284004EBE2
:107BC00080000C30FFF738FE0028F5D101AA00999B
:107BD00001EA050304EB8303491CDB6842F820300B
:107BE000401C00910328F2D3019800F00300012803
:107BF0001AD002280ED012494FF4AF70FBF73AFDAD
:107C0000384600F0A2FB08B10098606004B030462E
:107C1000BDE8F0810198032101EB90500099BDF877
:107C20000A6001EB900005E00198BDF80A60C0F31E
:107C3000831008440090E3E77C1D002064190020B5
:107C4000800C01002DE9FE4F814603F031FD07460F
:107C5000D9F80C0090F80880407A20B91FA20221C0
:107C6000484601F00DF922A324A20821484601F05C
:107C700007F92AA20821484601F002F9002429E068
:107C800001231A462146404603F01CFD824600238C
:107C900001222146404603F015FD0546042801D285
:107CA000064600E004260121204603F053FD03466A
:107CB000AE4201D229A200E027A2294850F826109E
:107CC00050F82A008DE8070026A20821484601F056
:107CD000D7F8641CBC42D3D3BDE8FE8F4C6F6773EA
:107CE000206172652068616C746564210D0A000072
:107CF0006D6F64756C655F6E616D6500252D343048
:107D000073207C2063757272656E74207C206275AE
:107D1000696C742D696E200D0A0000002D2D2D2D2B
:107D20002D2D2D2D2D2D2D2D2D2D2D2D2D2D2D2D83
:107D30002D2D2D2D2D2D2D2D2D2D2D2D2D2D2D2D73
:107D40002D2D2D2D2D2D2D2D2D2D2D2D2D2D2D2D63
:107D50002D2D2D2D2D2D0D0A000000002A000000D4
:107D600098020020252D343073207C20252D377378
:107D7000207C20257325730D0A00000008B54FF400
:107D800000442146414803F041FC20B140A240F2AA
:107D90002111F9F73FFA01F09FFC20B13CA24FF40A
:107DA0009371F9F737FA002001F0B6FCFAF768FB97
:107DB00020B137A24FF49571F9F72CFA384A012116
:107DC0003848FAF73FFB20B131A240F22D11F9F704
:107DD00021FA3448002221460068FAF777FB20B1E7
:107DE0002BA24FF49871F9F715FA2E4803240123BA
:107DF0001A4600211830009401F01CFA18B12AA28A
:107E0000B521F9F707FA274801231A460021343033
:107E1000009401F00FFA18B123A2C221F9F7FAF980
:107E200006F072FC1F48183001F062FB18B11EA268
:107E3000A321F9F7EFF91B48343001F059FB18B1D1
:107E400019A2AC21F9F7E6F9FFF7D6F81A4C6068E9
:107E500003280FD32088052505EB004017A103F068
:107E60004BFB6068032805D320881FA105EB004069
:107E700003F042FB03F016FA0A48183001F0D2FA78
:107E80000848343001F0CEFAF4E70000392400004D
:107E90002E2E5C2E2E5C2E2E5C6D61696E2E630084
:107EA00055DE000010EA00002E2E5C2E2E5C2E2ED9
:107EB0005C6D61696E2E6300F8040020436F6D6D88
:107EC000616E64204C696E6520496E7465726661EE
:107ED0006365206578616D706C6520737461727480
:107EE00065642E0D0A000000506C6561736520709A
:107EF000726573732074686520546162206B6579C4
:107F000020746F2073656520616C6C2061766169F7
:107F10006C61626C6520636F6D6D616E64732E0DB4
:107F20000A0000002DE9FF4F4FF0000881B0144611
:107F30008B468146C246C0F800802578002D71D05E
:107F4000F9F778FA00900068405DC00702D004F8A5
:107F500001AB84E0D9F800008300401CC9F80000A0
:107F60004BF8034015E02678002E78D0B8F1000FCA
:107F700005D1222E10D0272E0ED05C2E1ED0B0455B
:107F800014D12046FCF7BCFF0246611C2046F9F7DD
:107F9000A9FA4FF00008E6E72046FCF7B1FF0246D9
:107FA000611C2046F9F79EFAB046DCE7B8F1000FF5
:107FB00050D05C2E6AD16078404508D12046FCF74D
:107FC0009FFF0246611C2046F9F78CFA5EE03028DC
:107FD0001CD100270225605DA0F13001072906D8D9
:107FE0006D1C41EAC701EDB2CFB2052DF3D3022DCE
:107FF0000CD92046FCF784FF421B61192046491E1C
:10800000921CF9F76FFA04F8017BACE778281ED1CF
:1080100000270225605DA0F13001092903D841EA5B
:1080200007100DE021E0A0F16101052901D85738C2
:1080300004E0A0F14101052907D8373840EA0710CC
:108040006D1CEDB2C7B2042DE4D3022DD1D8B8F126
:10805000000F1BD100980068805DC00716D0D9F8CA
:10806000001004988142FFF468AFD9F800000C2892
:1080700004D907A140F25B40FBF7FCFAD9F80020D5
:1080800040464BF822A005B0BDE8F08F641C6AE7BB
:108090002E2E5C2E2E5C2E2E5C2E2E5C2E2E5C2E1A
:1080A0002E5C636F6D706F6E656E74735C6C69626D
:1080B0007261726965735C636C695C6E72665F6342
:1080C0006C692E63000000002DE9F05FC7888A46C6
:1080D000191D1646B1FBF7F2B1FBF7F507FB1219B4
:1080E00099193944C91CB1FBF7F104464079C9B26A
:1080F000DDF828B0884206D217499420FBF7BAFA77
:1081000001E024686D1E002DFBD1A846A7EB0905F0
:10811000B5421AD81CE000BFBBF1000F06D004EB3B
:1081200009010AEB08002A46091D05E004EB0900D5
:108130000AEB08012A46001DF9F7D4F92468761BDA
:108140004FF00009A844B74201D9354600E03D464A
:10815000002EE1D1BDE8F09FFC06010033B581B0EF
:108160000546002409E000226946284603F0BEFEC9
:1081700018B9009803F0CBFB641C02A9284604F050
:1081800079F80028EFD120463EBD70B51446002393
:108190000D4606461A4603F095FA844201D900209E
:1081A00070BD22462946304603F0B2FA012070BD68
:1081B00030B5024669B103F07BFA0021084C0BE0B0
:1081C00001EB410304EB830315685B88AB4202D1EA
:1081D0001160002030BD491C8142F1D3052030BD23
:1081E0006C03002010B50C460021E160616003497A
:1081F000A160012103F0AEFA206010BD84F20000FE
:108200002DE9FE43002416460D460C2780460094B7
:10821000019423463A466946029403F087FB00988E
:1082200045F8040B019845F8040B029845F8040B37
:10823000009800F00300012803D0022806D0346023
:1082400017E00098C0F38310840004E00098800DCC
:1082500005F048F904463B4622462946404603F0CD
:1082600065FB30680C34A04203D301203460BDE8C4
:10827000FE830020FBE770B58468006804F1080500
:10828000FCF73EFEC1B22973A08B6A890844B0FB9B
:10829000F2F302FB13035B1C2B80A08B0844B0FBA2
:1082A000F2F35B1CAB80608B0844B0FBF2F35B1C09
:1082B000EB80608B0844B0FBF2F102FB1101491C1A
:1082C0006980284670BD10B531B1B2FBF3F403FBF1
:1082D00014241CB1092010BD0E2010BD0160002126
:1082E000416081608281C381084610BD70B50C4633
:1082F0000546F8F7B7FF002802D02188286808440F
:1083000070BD10B50A8849888A4203D1F8F7ECFF9E
:10831000012010BD002010BD70B50C460546F8F7D1
:10832000C6FF002802D061882868084470BD10B5D7
:108330000A8849888A4203D1F8F7B0FF012010BDAE
:10834000002010BD002100F00FB8002100F012B88D
:10835000012100F01EB8012100F011B808B56A46ED
:10836000F9F717F8009808BD08B56A46F8F7F7FF5F
:10837000009808BD08B56A46F8F7F1FF08BD08B5D2
:108380006A46F8F7DFFF08BD08B56A46F8F7CEFF82
:1083900008BD08B56A46F8F7D5FF009808BD08B5CE
:1083A0006A46F9F703F8009808BD000070B50400AC
:1083B00003D113A1FE20FBF75DF900252846FBF74A
:1083C000EBF8206862680168914214D9491E016087
:1083D0000D781CB919A1C220FBF74CF9208BE1687C
:1083E00005FB00152068217A0278891A0279C9B242
:1083F0008A4200D201710020FBF7FCF8284670BDCC
:108400002E2E5C2E2E5C2E2E5C2E2E5C2E2E5C2EA6
:108410002E5C636F6D706F6E656E74735C6C6962F9
:108420007261726965735C62616C6C6F635C6E72C1
:10843000665F62616C6C6F632E6300002E2E5C2E93
:108440002E5C2E2E5C2E2E5C2E2E5C2E2E5C636FF0
:108450006D706F6E656E74735C6C69627261726967
:1084600065735C62616C6C6F635C6E72665F6261A7
:108470006C6C6F632E63000070B50C46050004D170
:1084800010A140F22110FBF7F5F824B90DA14FF42B
:108490009170FBF7EFF80020FBF77EF81DB9184943
:1084A000CF20FBF7E7F8E8682A68211A288BB1FB90
:1084B000F0F11068431C13600170BDE870400020AB
:1084C000FBF798B82E2E5C2E2E5C2E2E5C2E2E5C8A
:1084D0002E2E5C2E2E5C636F6D706F6E656E7473E6
:1084E0005C6C69627261726965735C62616C6C6F0D
:1084F000635C6E72665F62616C6C6F632E6300001A
:108500003C84000010B5040002D0206830B901E0BE
:108510000E2010BD17A1D920FBF7ACF8606818B980
:1085200014A1DA20FBF7A6F8A06818B911A1DB2086
:10853000FBF7A0F8E06818B90EA1DC20FBF79AF869
:10854000208B18B90BA1DD20FBF794F8207A616825
:108550002268401AC0B2116004E0226811684B1C06
:1085600013600870401EC0B2F7D221680020087165
:1085700010BD00002E2E5C2E2E5C2E2E5C2E2E5C4E
:108580002E2E5C2E2E5C636F6D706F6E656E747335
:108590005C6C69627261726965735C62616C6C6F5C
:1085A000635C6E72665F62616C6C6F632E63000069
:1085B0002DE9F04F8146806889B0D0F84803C0F3B8
:1085C000400038B109B04846BDE8F04F00221146DE
:1085D00000F0B4BC012907D909B04846BDE8F04F06
:1085E00024A2022100F04CBC27492848081A1C216B
:1085F000B0FBF1F8002538E02448C5EBC50110EBCD
:1086000081044FF0000AB4F818B0D4E90101A1EBDD
:10861000000604D11EA140F21F10FBF72BF82068C2
:10862000077924B91AA140F22F10FBF723F820682C
:10863000217A0078081AC0B2642117FB01F1B1FB5E
:10864000F6F2642110FB01F1B1FBF6F16369CDE9AB
:108650000210CDE90462CDE90676CDE900BA1B4AE5
:108660000821484600F00CFC6D1C4545C4D309B0F8
:10867000BDE8F08F42616420617267756D656E744C
:1086800020636F756E740000C8130100741301003D
:108690002E2E5C2E2E5C2E2E5C2E2E5C2E2E5C2E14
:1086A0002E5C636F6D706F6E656E74735C6C696267
:1086B0007261726965735C62616C6C6F635C6E722F
:1086C000665F62616C6C6F632E680000DC02010003
:1086D000C20800F007030120895C984008407047F9
:1086E00010B5C20800F00703885C01249C402043B9
:1086F000885410BD70B515468268D2F84843C4F35B
:10870000400424B11A46294600F018FC06E039B1AD
:10871000516804A20B68022100F0B2FB012070BD79
:10872000002070BD25733A2077726F6E67207061EC
:1087300072616D6574657220636F756E740D0A00E9
:1087400070B50D46040004D122A140F65640FAF758
:1087500091FFA06818B1606808B1206820B91DA118
:1087600040F65740FAF786FF022D0CD1A068D0F8EA
:108770004803C0F3400030B12046BDE870400022FD
:10878000114600F0DBBB40F65F451CB911A128463D
:10879000FAF770FF206918B90EA12846FAF76AFFA8
:1087A0001A4A1BA1206901F0E7FF4FF446651CB986
:1087B00008A12846FAF75EFF206918B905A12846E6
:1087C000FAF758FF2069BDE87040104A10A109323D
:1087D00001F0D2BF2E2E5C2E2E5C2E2E5C2E2E5C37
:1087E0002E2E5C2E2E5C636F6D706F6E656E7473D3
:1087F0005C6C69627261726965735C636C695C6E02
:1088000072665F636C692E630000000070EF000009
:108810002573000070B50D46040004D113A140F685
:108820006540FAF727FFA06818B1606808B12068B2
:1088300020B90EA140F66640FAF71CFF012D07D0C3
:10884000022D0CD1A068D0F84803C0F3400030B12D
:108850002046BDE870400022114600F06FBB204664
:10886000BDE870400FA2022100F00ABB2E2E5C2E44
:108870002E5C2E2E5C2E2E5C2E2E5C2E2E5C636FBC
:108880006D706F6E656E74735C6C69627261726933
:1088900065735C636C695C6E72665F636C692E63A2
:1088A00000000000506C656173652073706563693A
:1088B0006679206120737562636F6D6D616E642EE1
:1088C0000D0A00001CB5012905D002290BD014D9CE
:1088D0004FF0010112E002B04FF00002BDE810407D
:1088E000114600F02BBB536808A1CDE900131368B3
:1088F0000CA2022100F0C4FA1CBD002102B000232A
:10890000BDE810401A46FFF7F5BE000020756E6BFB
:108910006E6F776E20706172616D657465723A205A
:108920000000000025733A257325730D0A0000002E
:1089300010B50446012901D0012100E000210023E7
:108940001A46FFF7D7FE002808D1A168C1F83803FE
:10895000E068C068BDE8104003F00CBC10BD00002A
:108960003EB50446012901D0012100E00021002389
:108970001A46FFF7BFFE002818D1E068C06803F070
:10898000CFFBC0B2642110FB01F2E168C9688968BD
:10899000B2FBF1F2D2B20092CDE90101A06804A2CB
:1089A0000821D0F83833204600F06AFA3EBD0000B6
:1089B0004C6F7374206C6F67733A2025750D0A4DE8
:1089C0006178206C6F6720717565756520757469B5
:1089D0006C697A6174696F6E3A2025752525205B74
:1089E00025752F25755D0D0A000000007CB5154624
:1089F0000E46040004D118A140F68640FAF73AFE6C
:108A0000A06818B1606808B1206820B912A140F6CA
:108A10008740FAF72FFE012E03D0022E09D0012144
:108A200008E002B02046BDE870400022114600F088
:108A300085BA002100231A462046FFF75BFE002876
:108A400009D1696812A0CDE9000117A202212046D0
:108A50002B6800F015FA7CBD2E2E5C2E2E5C2E2E7F
:108A60005C2E2E5C2E2E5C2E2E5C636F6D706F6EF6
:108A7000656E74735C6C69627261726965735C6364
:108A80006C695C6E72665F636C692E630000000047
:108A900020756E6B6E6F776E20706172616D65749C
:108AA00065723A200000000025733A257325730D86
:108AB0000A00000010B50446012901D0012100E0A0
:108AC000002100231A46FFF715FE002806D1A068F2
:108AD000D0F8481321F00401C0F8481310BD10B5B8
:108AE0000446012901D0012100E0002100231A469B
:108AF000FFF700FE002806D1A068D0F8481341F027
:108B00000401C0F8481310BD7CB514460D46064656
:108B1000022901D9012100E0002100231A46FFF7B4
:108B2000E9FD002811D1022D05D03046FBF712FFD8
:108B300060B10BA30BE061680AA0CDE900010FA2B0
:108B400002213046236800F09BF97CBD0EA302B0E1
:108B50003046BDE870400DA2082100F091B9000038
:108B60006F6E000020756E6B6E6F776E2070617295
:108B7000616D657465723A200000000025733A2526
:108B80007325730D0A0000006F6666004563686F09
:108B9000207374617475733A2025730D0A00000008
:108BA00010B50446012901D0012100E00021002375
:108BB0001A46FFF79FFD002806D1A068D0F8481399
:108BC00021F00801C0F8481310BD10B50446012972
:108BD00001D0012100E0002100231A46FFF78AFDA1
:108BE000002806D1A068D0F8481341F00801C0F869
:108BF000481310BD7FB50D46040004D123A140F6F3
:108C0000CC40FAF737FDA06818B1606808B1206859
:108C100020B91EA140F6CD40FAF72CFD012D01D060
:108C2000012100E0002100231A462046FFF762FDE3
:108C3000002829D1A0680026D0F8405305B301E0F0
:108C4000082E1DD200230A2201A9284602F06EFE3A
:108C5000BDF80C20A1680A23284601F5D071521CEA
:108C600002F064FEA068334600F5D0700090029DCB
:108C7000761C14A20821204600F002F9002DDFD155
:108C8000A168002081F8A0017FBD00002E2E5C2E7F
:108C90002E5C2E2E5C2E2E5C2E2E5C2E2E5C636F98
:108CA0006D706F6E656E74735C6C6962726172690F
:108CB00065735C636C695C6E72665F636C692E637E
:108CC000000000005B2533645D2025730D0A000061
:108CD0007CB515460E46040004D120A140F6325062
:108CE000FAF7C8FCA06818B1606808B1206820B91C
:108CF0001AA140F63350FAF7BDFC012E03D0022E24
:108D000018D9012117E0A168204601F110021231A3
:108D100005F01CF800281FD0A16850201DA2488231
:108D2000A1681820088202B02046BDE870400421E6
:108D300000F0A6B8002100231A462046FFF7DAFC0F
:108D4000002809D1696822A0CDE9000126A20221EC
:108D500020462B6800F094F87CBD00002E2E5C2E7F
:108D60002E5C2E2E5C2E2E5C2E2E5C2E2E5C636FC7
:108D70006D706F6E656E74735C6C6962726172693E
:108D800065735C636C695C6E72665F636C692E63AD
:108D9000000000004E6F20726573706F6E73652067
:108DA00066726F6D20746865207465726D696E619E
:108DB0006C2C20617373756D6564203830783234A3
:108DC0002073637265656E2073697A650D0A000011
:108DD00020756E6B6E6F776E20706172616D657459
:108DE00065723A200000000025733A257325730D43
:108DF0000A00000070B50446012901D0012100E0FD
:108E0000002100231A46FFF775FC002817D140F611
:108E10002B551CB90AA12846FAF72CFC206918B971
:108E200007A12846FAF726FC134A14A1206901F08D
:108E3000A3FCA16850204882A1681820088270BD58
:108E40002E2E5C2E2E5C2E2E5C2E2E5C2E2E5C2E5C
:108E50002E5C636F6D706F6E656E74735C6C6962AF
:108E60007261726965735C636C695C6E72665F6384
:108E70006C692E630000000086EF0000257300007F
:108E80000FB4F8B5044608980E4620B91DA140F667
:108E90005120FAF7EFFB24B91AA140F65220FAF755
:108EA000E9FBA06818B1606808B1206820B915A175
:108EB00040F65320FAF7DEFB09A80090A068D0F82E
:108EC0004813490717D5817DB14214D0C58A314670
:108ED000204605F09FFC6A462069089901F0B8FC1D
:108EE000E9B2204605F096FC290A204605F074FCFC
:108EF000F8BC5DF814FB6A462069089901F0A8FCEB
:108F0000F6E700002E2E5C2E2E5C2E2E5C2E2E5CA4
:108F10002E2E5C2E2E5C636F6D706F6E656E74739B
:108F20005C6C69627261726965735C636C695C6ECA
:108F300072665F636C692E63000000002DE9F04FDC
:108F400089B090460D46040004D191A140F6D2208C
:108F5000FAF790FBA06818B1606808B1206820B9E2
:108F60008BA140F6D320FAF785FB9748FBF7C8FFA3
:108F7000064695483338FBF7C3FF301A1FFA80F9CD
:108F8000914892A220380090A068082140680368A8
:108F90002046FFF775FFA06840680068FBF7B0FF48
:108FA000064689482038FBF7ABFF304482B2A06800
:108FB0000023406841682046FEF7C6F985A20821D3
:108FC0002046FFF75DFFB8F1000F22D00DB3002659
:108FD0001DE000BF06EB460A05EB8A0BDBF8040038
:108FE000FBF78EFF074655F82A00FBF789FF391873
:108FF00049450BD9DBF80400FBF782FF074655F81B
:109000002A00FBF77DFF38441FFA80F9761C46459D
:10901000E0D36D483338FBF773FF4844801C1FFAD8
:1090200080F9694800904B466DA208212046FFF761
:1090300027FF09F1030087B2079000233A466AA18F
:109040002046FEF781F9002D51D000264DE000BFEB
:1090500006EB460A05EB8A0B55F82A00DBF80430CC
:1090600063B348B3584965A23339CDE900100821EC
:109070002046FFF705FF09F102000090DBF804002D
:10908000FBF73EFF074655F82A00FBF739FF074478
:109090004D483338FBF734FF39180098401A801ECA
:1090A00081B22046FDF7AEFA3A225749206901F015
:1090B00063FB0098401C0AE0009301E040B100907F
:1090C0004B4647A208212046FFF7DAFE079887B2F1
:1090D000DBF8081029B100233A462046FEF734F9A0
:1090E00002E02046FDF788F9761C4645B0D3A0681B
:1090F00040688068002847D0814600200646054623
:1091000003AF02902A466D1C02AB0121484600972E
:10911000FCF7EEFC029850B10068FBF7F1FEB0429C
:10912000F0D902980068FBF7EBFE86B2EAE7012D62
:109130002AD036A208212046FFF7A2FE0025B84615
:109140002A466D1C02AB01214846CDF80080FCF791
:10915000CFFC0298002817D0B11C8FB20068009095
:109160003B461FA208212046FFF78AFE0298FF1CFB
:10917000BAB2416821B100232046FEF7E5F8DFE7E7
:109180002046FDF739F9DBE709B0BDE8F08F0000B4
:109190002E2E5C2E2E5C2E2E5C2E2E5C2E2E5C2E09
:1091A0002E5C636F6D706F6E656E74735C6C69625C
:1091B0007261726965735C636C695C6E72665F6331
:1091C0006C692E63000000008CEF0000257325738E
:1091D000000000004F7074696F6E733A0D0A000052
:1091E0002020252D2A733A0053686F7720636F6D16
:1091F0006D616E642068656C702E00002020257300
:109200002573257300000000FC4300005375626362
:109210006F6D6D616E64733A0D0A00008068D0F85E
:109220004803C0F3400070478068D0F84803C0F39B
:10923000400070472DE9F0411E46DDF818801546C4
:109240000F46040004D10DA140F69410FAF712FA6B
:109250002A463946204600F02DF805000CD15EB1B3
:109260004146E06801F090FE002802DA0420BDE8E3
:10927000F081E068012141722846F8E72E2E5C2E2D
:109280002E5C2E2E5C2E2E5C2E2E5C2E2E5C636FA2
:109290006D706F6E656E74735C6C69627261726919
:1092A00065735C636C695C6E72665F636C692E6388
:1092B000000000002DE9F04715460E46040004D1D9
:1092C00043A140F63610FAF7D5F9A06818B16068E6
:1092D00008B1206820B93EA140F63710FAF7CAF964
:1092E000207E0A2806D00D2804D039A140F6381077
:1092F000FAF7C0F9E0682346434A446160680168B0
:109300000F683146B84700285FD1606920B930A1A5
:1093100040F64710FAF7AEF9606902F0F6FA002855
:1093200053D1A168C1F83C03A168C1F840034FF4D0
:109330005371A068F8F7FDF8A068D0F8481341F021
:109340002001C0F84813A068D0F8481365F38201E3
:10935000C0F84813A068D0F8481341F00801C0F8DD
:109360004813A1680120294F0870A168502040F6D9
:1093700063194882A16818200024088224482549DE
:1093800040F6641A0D1A804613E000BF18EBC406BD
:1093900003D10FA14846FAF76DF97068006818B953
:1093A0000BA15046FAF766F97068006847F8240088
:1093B000641CB4EBD50FE9D3072D05D9E908164B8A
:1093C00004223846F8F740F80020BDE8F087000096
:1093D0002E2E5C2E2E5C2E2E5C2E2E5C2E2E5C2EC7
:1093E0002E5C636F6D706F6E656E74735C6C69621A
:1093F0007261726965735C636C695C6E72665F63EF
:109400006C692E630000000035520000100300203C
:10941000D41101006412010091DC00000023FBF76D
:1094200041BF000010B5040004D122A140F61B206A
:10943000FAF720F9A06818B1606808B1206820B96F
:109440001CA140F61C20FAF715F9A068102100F5C0
:109450005270FEF79EFFA0680078F8B101281DD079
:1094600002281BD12046FBF743FC00212046FBF7D6
:1094700077FA98B11DA2032120462368FFF700FD6B
:109480002046FBF767FA48B1A36818A208212046D6
:109490002033FFF7F5FC2046FDF77EF8206901F048
:1094A000ABF9A068BDE810406FF0100100F55270F4
:1094B000FEF75ABF2E2E5C2E2E5C2E2E5C2E2E5CBE
:1094C0002E2E5C2E2E5C636F6D706F6E656E7473E6
:1094D0005C6C69627261726965735C636C695C6E15
:1094E00072665F636C692E630000000025730000E4
:1094F00070B5040004D117A140F6EA10FAF7BAF8E3
:10950000A06818B1606808B1206820B911A140F6C0
:10951000EB10FAF7AFF8A0680078012801D0082016
:1095200070BD606801688A680021904705000FD10E
:109530000821204605F06EF90121204605F04CF97E
:1095400012A1206901F018F902212046FBF7C4FCA2
:10955000284670BD2E2E5C2E2E5C2E2E5C2E2E5C90
:109560002E2E5C2E2E5C636F6D706F6E656E747345
:109570005C6C69627261726965735C636C695C6E74
:1095800072665F636C692E63000000000D0A0A00BA
:1095900000F180400068002800D00120704708B525
:1095A00000F18040002101600068009008BD0000CB
:1095B00010B5104C207820B90FA140F21F10FAF717
:1095C00059F8606820B90CA14FF49070FAF752F87E
:1095D0000020F9F7E1FF6068401E6060606818B91C
:1095E00003F0A8FA00206070BDE810400020FAF7F0
:1095F00001B800007C1100202E2E5C2E2E5C2E2E39
:109600005C2E2E5C2E2E5C2E2E5C696E746567724D
:109610006174696F6E5C6E7266785C6C65676163BD
:10962000795C6E72665F6472765F636C6F636B2EDB
:109630006300000070B5184C0546207818B917A1D2
:10964000FE20FAF717F8607838B115B16968002084
:1096500088470020F9F7A0FF0CE00020F9F79CFFF5
:1096600025B10D4829460830FEF71CF9606808B995
:1096700003F030FA6068401C60600020F9F7BAFF20
:109680006068002806D1BDE8704004A14FF48D70D9
:10969000F9F7F0BF70BD00007C1100202E2E5C2E6B
:1096A0002E5C2E2E5C2E2E5C2E2E5C2E2E5C696E79
:1096B000746567726174696F6E5C6E7266785C6CFB
:1096C00065676163795C6E72665F6472765F636C16
:1096D0006F636B2E6300000070B50A4C207808B1F0
:1096E00085250CE00020A06060602061E0600648F5
:1096F00003F058FA054603F0BBF901202070284614
:1097000070BD00007C1100209553000001480078D6
:10971000704700007C11002070B5174C054620787A
:1097200018B916A1C120F9F7A5FFA07838B115B175
:109730006968012088470020F9F72EFF0CE000201F
:10974000F9F72AFF25B10C4829461030FEF7AAF890
:10975000E06808B903F084FAE068401CE06000208B
:10976000F9F748FFE068002805D1BDE8704003A183
:10977000DD20F9F77FBF70BD7C1100202E2E5C2EFE
:109780002E5C2E2E5C2E2E5C2E2E5C2E2E5C696E98
:10979000746567726174696F6E5C6E7266785C6C1A
:1097A00065676163795C6E72665F6472765F636C35
:1097B0006F636B2E6300000010B500B9044803F01E
:1097C000B7FA002802D1034A0121117010BD000030
:1097D000CCEA00002801002010B5044600F007F88C
:1097E000204603F079FB03F070FB002010BD10B59C
:1097F00003F064FBBDE8104003F078BB0349024866
:10980000C1F8040370470000041480010070024096
:109810002DE9F0411D46174606460C46AA4204D2E1
:1098200013A140F2C310F9F725FF206838B103F007
:1098300053FA20B90EA14FF4E270F9F71BFF6068EC
:10984000A84204D2002171602168316007E0756090
:109850002168401B31606060216829442160AF426B
:1098600003D110B10120BDE8F0810020FBE700002A
:109870002E2E5C2E2E5C2E2E5C2E2E5C2E2E5C2E22
:109880002E5C636F6D706F6E656E74735C6472696D
:10989000766572735F6E72665C757362645C6E721D
:1098A000665F6472765F757362642E630000000009
:1098B00010B50D4C207820B90CA140F2EF60F9F7FB
:1098C000D9FE00F017FE1949D1F80403C1F80803C6
:1098D000174900200860BFF36F8FBFF34F8F04F06C
:1098E00057FD0120207010BD2C0100202E2E5C2E73
:1098F0002E5C2E2E5C2E2E5C2E2E5C2E2E5C636F2C
:109900006D706F6E656E74735C6472697665727388
:109910005F6E72665C757362645C6E72665F6472C1
:10992000765F757362642E63000000000070024071
:10993000007502402DE9F047DFF8049199F8000026
:10994000012804D03FA140F28C60F9F793FE4FF458
:109950000068404603F06EF800F05CFB494E4A4D4B
:1099600049F2753450B10020F9F716FE296803203A
:10997000002952D030600020F9F73CFE0020F9F7B2
:109980000BFE2968404FC020143700294AD03860A8
:109990000020F9F72FFE3D4901200860BFF36F8FCB
:1099A000BFF34F8F3A4801680905FCD5404603F0E4
:1099B00041F80020F9F7F0FD2868A846002580B39B
:1099C0003D600020F9F716FE00F024FB50B10020A6
:1099D000F9F7E2FDD8F80010404669B33560002081
:1099E000F9F708FE2B4940F2E37008604020091D9A
:1099F0000860BFF36F8FBFF34F8F244980201C3165
:109A000008604C4640F2FF10C4E9020504F0C0FCB7
:109A1000A57002202070BDE8F0872C6030602C60BB
:109A2000A9E703E02C6038602C60B1E7C8F800407B
:109A30003D60C8F80040C4E7046035600460CEE7CC
:109A40002C0100202E2E5C2E2E5C2E2E5C2E2E5CE9
:109A50002E2E5C2E2E5C636F6D706F6E656E747350
:109A60005C647269766572735F6E72665C75736250
:109A7000645C6E72665F6472765F757362642E6397
:109A80000000000014ED064000EC064000750240A6
:109A9000007402400078024004F08EBD70B50546A7
:109AA00004F08AFD2846FDF773F8044600F00F0025
:109AB000092804D30E4940F2B640F9F7DBFD04F063
:109AC0000F0122064FF0010001D50A4A01E0094AC0
:109AD000121D1368884083431360BFF36F8FBFF379
:109AE0004F8F284600F0BAF90349C1F8080370BD4A
:109AF000D8A60000107502400070024070B5010643
:109B000000F00F050446092D04D30C4940F28240B1
:109B1000F9F7B0FD082D04D3084940F28340F9F766
:109B2000A9FD07480460BFF34F8F44F480710160C2
:109B3000BFF36F8FBFF34F8F70BD0000D8A600003A
:109B40000C75024070B5054600F088F92149C1F84E
:109B50000403284602F0FAFD00283AD12846FDF712
:109B600017F8044600F00F00092804D31A4940F200
:109B7000A540F9F77FFD04F00F0021064FF0010426
:109B800001D5164901E01549091D0A6804FA00F0DB
:109B900002430A60BFF36F8FBFF34F8F280718D0BF
:109BA000280616D405F00F00082812D20020F9F775
:109BB000F3FC284600F024FD2846FCF779FF84409A
:109BC0000748C168A143C160BDE870400020F9F7B3
:109BD00011BD70BD00700240D8A600001075024093
:109BE0002C01002010B5FCF7D3FFBDE8104002F0B7
:109BF000ADBD00002DE9F0410E460746FCF758FFC9
:109C0000054626B918A140F65600F9F733FD0020A5
:109C1000F9F7C2FC244C380704D1A078874201D060
:109C200010241BE02089E168C04380B20843012171
:109C300001FA05F5284201D011240FE03846FCF75F
:109C40006BFF00218160326802607268426081733C
:109C5000E0680543E5600C4604F082FD0020F9F75A
:109C6000C9FC2046BDE8F0812E2E5C2E2E5C2E2EE7
:109C70005C2E2E5C2E2E5C2E2E5C636F6D706F6ED4
:109C8000656E74735C647269766572735F6E72661A
:109C90005C757362645C6E72665F6472765F757326
:109CA00062642E63000000002C01002010B5FCF758
:109CB00033FF808910BD000070B50C00054602D04E
:109CC000601E044204D011A140F29B70F9F7D2FC4F
:109CD00005F00F0008280CD31C480068C1B2802989
:109CE00004D04FF48060A0420AD204E04FF4007028
:109CF000F9E7402C04D905A140F29D70F9F7BAFCB0
:109D00002846FCF709FF848170BD00002E2E5C2ED2
:109D10002E5C2E2E5C2E2E5C2E2E5C2E2E5C636F07
:109D20006D706F6E656E74735C6472697665727364
:109D30005F6E72665C757362645C6E72665F64729D
:109D4000765F757362642E63000000001C7502402C
:109D500010B5FCF71DFF044600F00F00082804D3DF
:109D6000064940F2CF40F9F785FC054944F480707C
:109D70000860BFF36F8FBFF34F8F10BDD8A60000F0
:109D80001875024010B5FCF703FF00F00F01082919
:109D900001D3002010BD0206054800EB810002D56A
:109DA000D0F8200401E0D0F844040128F1D110BD1E
:109DB0000070024010B5FCF7EBFE044600F00F0007
:109DC000082804D3054940F2D740F9F753FC04486A
:109DD0000460BFF36F8FBFF34F8F10BDD8A6000094
:109DE0001875024070B50446000604F00F0502D550
:109DF000092D09D301E0092D08D307A140F2631012
:109E0000F9F738FC200601D5134801E0124812305A
:109E100030F8150070BD00002E2E5C2E2E5C2E2E0C
:109E20005C2E2E5C2E2E5C2E2E5C636F6D706F6E22
:109E3000656E74735C647269766572735F6E726668
:109E40005C757362645C6E72665F6472765F757374
:109E500062642E63000000007CEB000070B50546D4
:109E6000000605F00F0402D5092C09D301E0092CE6
:109E700008D307A14FF4C670F9F7FCFB280601D5FB
:109E8000134801E012480930015D0120884070BD8F
:109E90002E2E5C2E2E5C2E2E5C2E2E5C2E2E5C2EFC
:109EA0002E5C636F6D706F6E656E74735C64726947
:109EB000766572735F6E72665C757362645C6E72F7
:109EC000665F6472765F757362642E6300000000E3
:109ED000A0EB00002DE9F0410D460646FCF7E8FD39
:109EE000044625B930A140F2E770F9F7C3FB002022
:109EF000F9F752FB3C48310704D181788E4201D0FA
:109F0000102438E001898046C943C06889B201271E
:109F10000143A740394201D011242CE03046FCF720
:109F2000FBFD044606F00F00310600EB40002AD589
:109F30002E4901EB8006286802F0CEFE0028287A20
:109F40004FEAC07004D008B1294803E0294801E075
:109F5000B8B12948206095E8070086E8070000208E
:109F6000C4E90160A073D8F80C1004460F43C8F888
:109F70000C7004F0F5FB0020F9F73CFB2046BDE82F
:109F8000F0811E48E6E719496C3101EB800628682C
:109F900038B102F0A1FE20B903A14FF40460F9F733
:109FA00069FB1748D6E700002E2E5C2E2E5C2E2E65
:109FB0005C2E2E5C2E2E5C2E2E5C636F6D706F6E91
:109FC000656E74735C647269766572735F6E7266D7
:109FD0005C757362645C6E72665F6472765F7573E3
:109FE00062642E63000000002C010020B0120020EB
:109FF00061A20000DDA1000035A1000095A00000D5
:10A000001198000010B5FCF7C3FDBDE8104002F048
:10A01000D1BC000010B500F013F858B10748007823
:10A02000C0F30310012805D10448001D007810F08A
:10A03000F00F01D0002010BD012010BDE80F00F08E
:10A0400006480078082804D10448001D007800075D
:10A0500001D000207047012070470000E00F00F0A1
:10A0600010B5FFF7EDFF50B10748007810F0F00F82
:10A0700005D10548001D007810F0F00F01D0002038
:10A0800010BD012010BD0000E80F00F0004870472F
:10A09000881300202DE9F041804616460C460868DA
:10A0A00002F01AFE20B112A14FF40B70F9F7E2FA98
:10A0B00065681F4FB54200D93546402D04D90CA123
:10A0C00040F23620F9F7D6FA2A4638462168F7F7E3
:10A0D00009FAC8E900756068401B60602068284480
:10A0E00020606068002800D00120BDE8F0810000F9
:10A0F0002E2E5C2E2E5C2E2E5C2E2E5C2E2E5C2E9A
:10A100002E5C636F6D706F6E656E74735C647269E4
:10A11000766572735F6E72665C757362645C6E7294
:10A12000665F6472765F757362642E630000000080
:10A13000881300202DE9F041064690460D46086838
:10A1400002F0CAFD20B114A140F25220F9F792FAB0
:10A150006C68214F4046444500D90446402C04D940
:10A160000DA14FF41770F9F785FA34B1224638463D
:10A170002968F7F7B7F9376001E0002030607460B4
:10A180006868001B686028682044286014B10120BA
:10A19000BDE8F0810020FBE72E2E5C2E2E5C2E2EDB
:10A1A0005C2E2E5C2E2E5C2E2E5C636F6D706F6E9F
:10A1B000656E74735C647269766572735F6E7266E5
:10A1C0005C757362645C6E72665F6472765F7573F1
:10A1D00062642E6300000000881300202DE9F04126
:10A1E000074616460C46086802F076FD20B90CA119
:10A1F0004FF4F570F9F73EFA6568B54200D9354677
:10A200002068C7E900056068401B6060206828443A
:10A2100020606068002800D00120BDE8F0810000C7
:10A220002E2E5C2E2E5C2E2E5C2E2E5C2E2E5C2E68
:10A230002E5C636F6D706F6E656E74735C647269B3
:10A24000766572735F6E72665C757362645C6E7263
:10A25000665F6472765F757362642E63000000004F
:10A260002DE9F041074616460C46086802F034FD19
:10A2700020B910A140F20B20F9F7FCF96568B5424E
:10A2800000D93546002D0FD0D4F80000C7E90005ED
:10A290006068A0EB0500606020682844206006D05C
:10A2A0004FF00100BDE8F0814FF00000EEE74FF005
:10A2B0000000F7E72E2E5C2E2E5C2E2E5C2E2E5CE0
:10A2C0002E2E5C2E2E5C636F6D706F6E656E7473D8
:10A2D0005C647269766572735F6E72665C757362D8
:10A2E000645C6E72665F6472765F757362642E631F
:10A2F000000000002DE9F04128B11E490A7822B182
:10A300000820BDE8F0810720FBE748600120002419
:10A31000087046024FEA040544F0800707F00F007A
:10A32000082801D3314600E040213846FFF7C4FC3D
:10A330003846FCF7F1FB8573641C0560E4B2856068
:10A34000092CE9D35FF0000404F00F00082801D3C2
:10A35000314600E040212046FFF7AEFC2046FCF7E6
:10A36000DBFB8573641C0560E4B28560092CEBD3CC
:10A370000020C6E72C01002003480078022801D302
:10A3800001207047002070472C010020024800780F
:10A39000002800D0012070472C01002010B5FFF7E5
:10A3A000EBFF28B12720F7F779FE08B1012010BD97
:10A3B000002010BD01488078704700002C0100206B
:10A3C000502002F049BB10B5FFF74AFE58B1EFF339
:10A3D000108472B64C2002F03FFB4C2002F03CFB94
:10A3E00084F3108810BDBDE810404C2002F034BB4F
:10A3F0000021016041601149096801700F49091D80
:10A40000096841700D49083109680C4A0C3212681C
:10A4100041EA02214180094910310968074A143292
:10A42000126841EA02218180044918310968034A0F
:10A430001C32126841EA0221C180704780740240D8
:10A44000542002F009BB000070B5144C054620787A
:10A45000022804D012A140F2FD60F9F70BF90020A8
:10A4600060701F4C15B9FFF7FBFD00B11D4C1E4875
:10A47000C0F804431D49E02081F800041B49012273
:10A4800080202339C1F88002C1F800011848026019
:10A49000BFF36F8FBFF34F8F70BD00002C01002002
:10A4A0002E2E5C2E2E5C2E2E5C2E2E5C2E2E5C2EE6
:10A4B0002E5C636F6D706F6E656E74735C64726931
:10A4C000766572735F6E72665C757362645C6E72E1
:10A4D000665F6472765F757362642E6300000000CD
:10A4E0000714C0010714E0010070024027E000E0FB
:10A4F00004750240104810B50078022804D00FA15E
:10A5000040F21C70F9F7B6F82720F7F7C7FD0028CE
:10A5100010D004F0B3F8194900200860BFF36F8F22
:10A52000BFF34F8F16498020C1F8800148171549A5
:10A53000C1F8080310BD00002C0100202E2E5C2E57
:10A540002E5C2E2E5C2E2E5C2E2E5C2E2E5C636FCF
:10A550006D706F6E656E74735C647269766572732C
:10A560005F6E72665C757362645C6E72665F647265
:10A57000765F757362642E6300000000047502400C
:10A5800004E000E00070024010B500242046F9F716
:10A5900003F812484078B0B104F070F81048016830
:10A5A000890510D40F4901220A60006882054FF026
:10A5B000000001D5086006E00B4901240B680A4A37
:10A5C00014322BB110600020F9F714F8204610BDAA
:10A5D00049F275330B6010600B60F4E72C0100202A
:10A5E000007402402C75024000EC0640034902480A
:10A5F000C1F8080370470000041480010070024095
:10A600002DE9F0410446000604D521A14FF40E6067
:10A61000F9F730F8FFF724FD01274FF000082C4D23
:10A62000002804F00F06404612D0F8F7B5FF204688
:10A63000FCF73EFA8740A8682649B843A86040F274
:10A64000C57000EB46000860091DC1F800801AE0E3
:10A65000F8F7A2FF2046FCF72BFA8740A868B8431A
:10A66000A860082E0FD2200604D51BA140F262403C
:10A67000F9F700F8244A02EB8601C1F8A084BFF381
:10A680006F8FBFF34F8FBDE8F0410020F8F7B2BFE6
:10A690002E2E5C2E2E5C2E2E5C2E2E5C2E2E5C2EF4
:10A6A0002E5C636F6D706F6E656E74735C6472693F
:10A6B000766572735F6E72665C757362645C6E72EF
:10A6C000665F6472765F757362642E6300000000DB
:10A6D0002C010020007802402E2E5C2E2E5C2E2EA7
:10A6E0005C2E2E5C2E2E5C2E2E5C6D6F64756C6560
:10A6F000735C6E7266785C68616C5C6E72665F75C6
:10A700007362642E68000000007002400548017802
:10A71000012901D0082070470021416001700846DE
:10A72000704700002C01002010B500242046F8F7E7
:10A7300033FF0E48407868B102F086F950B10C49F9
:10A74000002008600B4901240B680A4AC02014321B
:10A750002BB110600020F8F74DFF204610BD49F2E4
:10A7600075330B6010600B60F4E700002C010020D3
:10A770002C75024000EC06400FB438B5040003D13C
:10A7800010A11C20F8F776FF606918B90DA11D20F3
:10A79000F8F770FF206818B90AA11E20F8F76AFFC1
:10A7A000606818B907A11F20F8F764FF0599002910
:10A7B00005D006A800906A46204600F049F838BC4B
:10A7C0005DF814FB2E2E5C2E2E5C2E2E5C2E2E5C45
:10A7D0002E2E5C2E2E5C65787465726E616C5C66E4
:10A7E0007072696E74665C6E72665F667072696EB6
:10A7F00074662E630000000010B5040003D107A1A9
:10A800000B20F8F737FFA268002A05D0D4E904032B
:10A81000216898470020A06010BD00002E2E5C2EFD
:10A820002E5C2E2E5C2E2E5C2E2E5C2E2E5C6578E1
:10A830007465726E616C5C667072696E74665C6E73
:10A8400072665F667072696E74662E630000000047
:10A850002DE9FC4791460C465FEA000804D183A12C
:10A860004FF49F70F8F706FFD8F8140020B97FA1C5
:10A870004FF4A070F8F7FEFED8F8000020B97BA1D5
:10A8800040F24110F8F7F6FED8F8040020B977A19D
:10A890004FF4A170F8F7EEFE002C76D014F8011BEF
:10A8A00039B125290ED04046F8F73CFF2078002822
:10A8B000F4D198F80C00002867D04046BDE8FC476A
:10A8C000FFF79ABF0020012221782B291BD02D29C8
:10A8D00002D0302908D102E040F0010001E040F050
:10A8E0000200641C002AEFD100252A290ED021780D
:10A8F000A1F130020A2A11D205EB850201EB4205D3
:10A90000641C303DF1E740F00400EAE7D9F800109C
:10A910000B1DC9F800300968641C0D442178002320
:10A920002E290BD114F8011FA1F130020A2A05D2F9
:10A9300003EB830201EB4203303BF3E76C290DD0BC
:10A9400068290BD0692921D00BDC252918D058297A
:10A9500031D063290ED0642915D117E014F8011FF6
:10A96000ECE7702969D0732932D075291BD078297A
:10A9700009D120E0D9F80000011DC9F800100178C4
:10A980004046F8F7CFFE641C90E76CE0D9F8001061
:10A990000A1DC9F800200968CDE900500A22404686
:10A9A000FCF7F6FEEFE7D9F800100A1DC9F8002001
:10A9B00009680A2206E0D9F800100A1DC9F800202B
:10A9C00009681022CDE90050404603F0CBFBDAE7DE
:10A9D000D9F8001000270A1DC9F800200E68C0072A
:10A9E00005D112E04046761C7F1CF8F79BFE3178BB
:10A9F0000029F7D104E0202140466D1EF8F792FEB1
:10AA0000BD42C0D9002DF6D1BDE74EB13046F6F7B4
:10AA1000B7FD074604E0202140466D1EF8F782FE90
:10AA2000BD4206D9002DF6D103E04046761CF8F76A
:10AA300079FE31780029F8D1A5E7D9F80000011D89
:10AA4000C9F80010056830214046F8F76BFE782100
:10AA50004046F8F767FE08200021CDE900010346D3
:10AA600010222946B0E7BDE8FC8700002E2E5C2EA0
:10AA70002E5C2E2E5C2E2E5C2E2E5C2E2E5C65788F
:10AA80007465726E616C5C667072696E74665C6E21
:10AA900072665F667072696E74665F666F726D6112
:10AAA000742E63002DE9F84F2E4D04008946288846
:10AAB0004FF0010C69689A4616460CEB004025D011
:10AAC0002268002A2DD0002E35D062684FF0100782
:10AAD0001268531E13EA090F12D1E0467243494629
:10AAE0002046F7F7DAFB00282FD02068534632467D
:10AAF000056901B049462046AC46BDE8F04F6047C5
:10AB000000292DD0184B19A2009726E031B10E2153
:10AB10000091154B1FA221A100F001FD0E20BDE800
:10AB2000F88F31B1082100910F4B27A21BA100F033
:10AB3000F6FC0820F3E731B1092100910A4B25A268
:10AB400016A100F0ECFC0920E9E7686840B1009725
:10AB50002988054B204A08EB014010A100F0DFFCDA
:10AB60001020DCE7B004002041F000006164647252
:10AB70005F69735F706167655F616C69676E65646B
:10AB800028705F66732C20706167655F6164647212
:10AB900029000000705F66730000000025732063C9
:10ABA0006865636B206661696C656420696E202549
:10ABB00073282920776974682076616C7565203068
:10ABC0007825782E00000000705F66732D3E705F60
:10ABD000617069006C656E00AC060100F8B5030099
:10ABE00010484FF001064FF00E054468008806EB50
:10ABF000004009D069B119600C6801B0A446BDE8F5
:10AC0000F04011461846604754B1074B07A2009523
:10AC100003E02CB1044B07A2009508A100F07FFCD3
:10AC20000E20F8BDB0040020F6EF0000705F6673E0
:10AC300000000000705F61706900000025732063F0
:10AC40006865636B206661696C656420696E2025A8
:10AC500073282920776974682076616C75652030C7
:10AC60007825782E0000000018B102680AB15269F8
:10AC700010470020704700002DE9F84F414C0500B7
:10AC80008B46208891464FF00106DDF828A06168C8
:10AC900098464FF00E0206EB00401BD0B9F1000FB2
:10ACA0001DD02A68002A23D00922B8F1000F29D02C
:10ACB0006B685F68B8FBF7FC07FB1C83002B27D091
:10ACC00029B1314B009231A23BA100F028FC0920B0
:10ACD000BDE8F88F51B100922B4B42A203E029B19D
:10ACE000294B009241A234A100F019FC0E20EFE79D
:10ACF00031B108210091244B3EA22FA100F00FFC9E
:10AD00000820E5E70029E2D000921F4B3CA2DBE7D8
:10AD10005846F7F7BCFA102798B14846F7F7B7FA44
:10AD2000C8B1424659462846F7F7B7FAF8B1CDF808
:10AD300000A0286843464A46C46859462846A047AA
:10AD4000C6E7606800281BD0009720880E4B06EBF2
:10AD500000402CA207E0606890B1009720880A4B61
:10AD600006EB00402DA214A100F0D9FB08E06068BA
:10AD700030B100972088044B06EB004030A2F2E788
:10AD80001020A5E7B00400202EF0000021286C65FB
:10AD90006E202520705F66732D3E705F666C617358
:10ADA000685F696E666F2D3E70726F6772616D5F6E
:10ADB000756E697429000000257320636865636BF4
:10ADC000206661696C656420696E202573282920DE
:10ADD000776974682076616C756520307825782EE7
:10ADE00000000000705F667300000000705F737207
:10ADF00063000000705F66732D3E705F61706900D4
:10AE00006C656E00616464725F69735F616C696731
:10AE10006E656433322864657374290061646472FA
:10AE20005F69735F616C69676E656433322828758A
:10AE3000696E7433325F7429705F73726329000026
:10AE4000616464725F69735F77697468696E5F6279
:10AE50006F756E647328705F66732C2064657374FD
:10AE60002C206C656E29000013B50C46684600F076
:10AE700013F8009900EB8101D1F8002722F4403249
:10AE8000C1F80027009900EB8100D0F8001741EAD3
:10AE90000441C0F800171CBD10B5044600683028F6
:10AEA00004D308A140F2A110F8F7E4FB20682028A1
:10AEB00002D24FF0A04010BD00F01F0020600D48EE
:10AEC00010BD00002E2E5C2E2E5C2E2E5C2E2E5CD5
:10AED0002E2E5C2E2E5C6D6F64756C65735C6E72CD
:10AEE00066785C68616C2F6E72665F6770696F2E42
:10AEF00068000000000300507CB5154604460C4A6B
:10AF00006618022ED2E90002CDE9000204D909A197
:10AF100040F2B920F8F7AEFB694605E051F824008D
:10AF2000D0F81005641C01C5A642F7D87CBD00000E
:10AF3000B4EB00002E2E5C2E2E5C2E2E5C2E2E5C92
:10AF40002E2E5C2E2E5C6D6F64756C65735C6E725C
:10AF500066785C68616C2F6E72665F6770696F2ED1
:10AF600068000000034908B508440021016000683A
:10AF7000009008BD0060004002494058012800D000
:10AF800000207047006000402DE9F0410E461C494A
:10AF900004460025D1F81024104609E0037AAB429C
:10AFA00005D16D1C0A2DF7DB4FF0FF3525E0406819
:10AFB0000028F3D1681C20D02572D1F8100440B1CC
:10AFC00040686060D1F8100444600027DFF83480E6
:10AFD0000FE00020C1F810446060F6E708EBC700FE
:10AFE000C279B24200D33246207A394600F090FB53
:10AFF0007F1C00F05DFBB842F0D82846BDE8F08128
:10B00000641900206412010038B54469C068002248
:10B01000694600F06BFF002803D100212046F9F7B4
:10B020009FFC38BD10B54469606801688A680121D9
:10B03000904718B10420A168087010BD0320FAE7FA
:10B040002DE9F34146690446B068007804281ED013
:10B05000032807D0002501A9E06801F00BF985F06D
:10B06000010709E00125F6E739463046F9F778FC93
:10B0700001A9E06801F0FEF80028F5D1019800F080
:10B0800040FC002D03D000213046F9F769FCBDE8F3
:10B09000FC8100000148806802F078B8600200205E
:10B0A00038B5002216491748FFF798FD164C0121C4
:10B0B00008B1217038BD0220207014480025C0F866
:10B0C000801101216068FCF719FD1149486A0A8D59
:10B0D000CB6A61F39F200F49086090B2C1E9010378
:10B0E0000A4600950C2307482169FFF7C5FD206932
:10B0F0000C302061A068BDE838400121FCF7FEBC9F
:10B1000060F00000580300206002002004E000E02E
:10B11000E4F100005417002070B50B4C0D46207868
:10B1200001280FD0084600F0ECFB2946A068FDF787
:10B1300015F82078022805D1A068BDE870400121EB
:10B14000FCF7DCBC70BD00006002002070B5074D4C
:10B1500001200023287006480122010B09030C4638
:10B160000448FFF79FFC2C6170BD000060020020C6
:10B1700077250100580300203EB50F490B0B0F49FE
:10B180001B0303F6FF72C1E90332014600220B489C
:10B19000FFF724FD04000DD10025009502AA01A9A6
:10B1A000684600F00FF80028F8D0054800990161C2
:10B1B000057020463EBD00007725010058030020A1
:10B1C0006002002070B50D4601681646044611B9AC
:10B1D0001248010B090312482160FFF745FD68B1D1
:10B1E000206828600C3030602868006800F0030197
:10B1F000012905D0022907D0052070BD062070BDA9
:10B20000C0F38310800002E0800D02F06BF921682A
:10B210000C3008442060002070BD0000772501003C
:10B22000580300200148406801F0B0BF60020020D0
:10B230007047000070B50E4C0D462078002815D1DF
:10B24000084600F05EFB29466068FCF787FFA169AD
:10B250000844A06104F10C00FDF77DF8002805D139
:10B260006068BDE870400021FCF748BC70BD00007C
:10B27000600200200A4A012902EBC00007D002291F
:10B2800007D0032907D0042907D0002070470220E7
:10B29000704704207047007970474079704700007C
:10B2A000641201002DE9FF5FF8F74CFA18B1002095
:10B2B00004B0BDE8F09F874C0020C4F81804BFF329
:10B2C0004F8F60680090A6684FF00009304004EB93
:10B2D000800008E021680098814201D86160E6E7BB
:10B2E000304004EB80000C306946FCF7A5FA0028DA
:10B2F000F0D101AAA046009901EA060408EB8403F4
:10B30000491CDB6842F82030401C00910328F2D32E
:10B31000019800F00300022802D0012850D0BEE0BE
:10B320000198A022810D8A46B2EB905F00D8A0213F
:10B330000C4664F39F50C0F3C20701900C3166487D
:10B3400000F096FA0500EAD000F0DBFA4B460C223A
:10B3500001A9284600F0F0FA009909F10C0B3140E0
:10B36000701A8000001D844223D95A4E0C3630B129
:10B37000C2B208EB8101201A91460C3104E031463B
:10B38000E2B2002691463046C4B25B46284600F041
:10B39000D3FA0BEB09032EB1224631464FEA0500E2
:10B3A00000F0CAFA00990AF1030001EB9000009046
:10B3B0003DE008EB81015B46224628460C31EFE771
:10B3C0000198C0F38310062800D30620019960F38A
:10B3D0008911C1F38310C1F3C207C01C0191810020
:10B3E0003D4800F045FA050059D000F08AFA4B4676
:10B3F0000C2201A9284600F09FFA09F10C0900244B
:10B400000FE000984B460246304008EB8001501C8C
:10B410000090042228460C3100F08EFA09F104094C
:10B42000641C0198C0F38310A042EAD8B5B3D8F8E1
:10B430001044D8F818044646F8B1284600F067FAD8
:10B4400042E0607A012817D1BDF80800234A00EBDA
:10B45000400002EB8000217A806801EB4101C84086
:10B4600000F00700052F00D10327B84204D322685B
:10B4700020462946126890476468002CE1D128468E
:10B4800000F045FA0020F8F787F8D6F8180408B954
:10B49000009870600020F8F7ADF815E0FFE7D8F8E5
:10B4A000104404E021682046896888476468002CBD
:10B4B000F8D10B484168022906D30088022101EB2C
:10B4C000004008A100F018F8F8F73CF980F00100FE
:10B4D000EEE6000064190020AC1301006C030020AC
:10B4E000F80400204261636B656E647320666C75BE
:10B4F000736865640000000000231A4602F046BB32
:10B5000008B5012300926A4602F040FB08BD1CB555
:10B51000CDE9002302236A4602F038FB1CBD3EB58C
:10B52000069C8DE81C0003236A4602F02FFB3EBDFB
:10B530007FB5DDE908458DE83C0004236A4602F04A
:10B5400025FB7FBD70B586B00DF1280C9CE870001E
:10B550008DE87C0005236A4602F018FB06B070BD3A
:10B560002DE9F0470E4680461C46924608293ED8F3
:10B5700094F80C90002020731946104601F0A8FDA5
:10B580000025B54206D218F805201AA12046FFF77B
:10B59000F3F803E019A12046FFF7EEF86D1C082D23
:10B5A000EFD317A12046FFF7E7F80025B54210D2E8
:10B5B00018F80570F5F73EFF0068C05D10F03E0F0B
:10B5C00001D03A4600E02E220EA12046FFF7D4F823
:10B5D00003E00DA12046FFF7CFF86D1C082DE5D341
:10B5E00001222146504601F055FD84F80C90BDE83B
:10B5F000F087000020253032780000002020200055
:10B600007C00000025630000200000002DE9F047C9
:10B6100005001FD0214C4FF00009FF20C4F8009016
:10B62000C4E90190C4F81894C4F8149484F82094E0
:10B63000084600F00DF91A48C4F80C5400F065F9FA
:10B64000002808D11749DFF86080A1EB0800C7087F
:10B6500000241EE00720BDE8F087002635460CE0F8
:10B66000AC4209D058F8340058F835101422F5F7D8
:10B67000A5FF002800DD761C6D1CBD42F0D30B49F0
:10B6800004EB440001EB8000C0F804900480468085
:10B69000641CBC42E1D30020DDE7000064190020F7
:10B6A000AC13010074130100641201006C0300204C
:10B6B00002480349401AC008704700007413010093
:10B6C000641201007FB505461146002401A87BB134
:10B6D000FCF76EFDA0B901980B4900EB400001EBAF
:10B6E000800005EB45018068C84000F0070407E0D2
:10B6F000FCF75EFD20B90548019900EBC100847993
:10B7000004B0204670BD00006C03002064120100EC
:10B7100030B50F4B01EB410103EB810400EB40001E
:10B720000723A56803FA00F18D4302F00701814069
:10B73000294300252A46A16003FA02F00840D040C0
:10B74000A84200D90546D21C0A2AF5D3656030BD4F
:10B750006C03002013B56846FCF72AFD08B10020F1
:10B760001CBD0248009950F831001CBD6412010054
:10B7700070B508480125D0F8104480F8205405E041
:10B78000657221682046496888476468002CF7D1B3
:10B7900070BD0000641900202DE9FF4781460C9D13
:10B7A00000200C462F7B28739846164629461846DB
:10B7B00001F08EFC072E42D2DFE806F004090F16D6
:10B7C0001F2A360049462846FEF7D6FF37E049468D
:10B7D00028462268FEF7D0FF31E0D4E9002349462D
:10B7E0002846FEF7C9FF2AE0A0680090D4E90023AC
:10B7F00049462846FEF7C0FF21E0D4E90201CDE921
:10B800000001D4E9002349462846FEF7B5FF16E0BB
:10B8100004F1080007C88DE80700D4E90023494671
:10B820002846FEF7A9FF0AE004F108000FC88DE8DA
:10B830000F00D4E9002349462846FEF79DFF002269
:10B840002946404601F026FC2F73BDE8FF87000023
:10B85000054A0121054B516001E04008490098422A
:10B86000FBD8C2E900017047C802002040420F0027
:10B870002DE9F041058B80462D1F4819C01CB0FBF7
:10B88000F5F0C6B24046FCF791FD041E19D0002029
:10B89000207101206071E58000272546761EC4F8DE
:10B8A00000800BE04046FCF781FD60B16179491CE6
:10B8B0006171286005467F1CC0F80080B742F1D353
:10B8C0002046BDE8F081204600F002F80020F8E7AD
:10B8D0002DE9F041457901466B1E002201E009681F
:10B8E000521C9A42FBD30F680146002605E03846F9
:10B8F0000C68FCF7C1FD2146761CAE42F7D3BDE8CB
:10B90000F0810121001DFCF729BDFCF7FBBD10B53E
:10B9100004460121001DFCF742FD10F0FF0F04D189
:10B920002046BDE81040FFF7D3BF10BD38B5012455
:10B930000094FCF7C9FB38BD38B500240094FCF72F
:10B94000C3FB38BD2DE9F84F834600F091F9054659
:10B95000DBF80800D0F84803C0F3400030B1584687
:10B96000BDE8F84F00221146FDF7E8BA1C4803680D
:10B970001CA208215846FDF783FA1948001D0368E8
:10B980001DA208215846FDF77BFADFF85480DFF846
:10B99000509008F10808002409F1100908F1040A80
:10B9A0001AE00020F7F7F8FDC8F80040D9F8007059
:10B9B000DAF800600020F7F71DFE234613A20821E5
:10B9C00058460096FDF75CFA234617A20821584610
:10B9D0000097FDF755FA641CAC42E2D3BDE8F88F3E
:10B9E00090ED00E04D50555F545950453A0930787C
:10B9F000253038580D0A00004D50555F4354524CC5
:10BA00003A093078253038580D0A00000D0A4D509B
:10BA1000555F524241525B25755D3A0930782530B9
:10BA200038580D0A000000004D50555F52415352E6
:10BA30005B25755D3A093078253038580D0A0000CD
:10BA40002DE9FC4107468068D0F84803C0F3400068
:10BA500038B102B03846BDE8F04100221146FDF78A
:10BA60006DBA00F005F90646009030480068C0073E
:10BA700001D02FA300E030A332A208213846FDF701
:10BA8000FFF900244EE00020F7F786FD2748001D4F
:10BA9000046026480C300568001FD0F800800020A4
:10BAA000F7F7A8FDE807234633D032A2082138462D
:10BAB000FDF7E6F9C5F344010120491C884008EB75
:10BAC0000001491ECDE90010434630A20821384646
:10BAD000FDF7D6F9284600F0D3F8034637A208212F
:10BAE0003846FDF7CDF9284600F048F9034637A25D
:10BAF00008213846FDF7C4F9284600F0FBF8034654
:10BB000036A208213846FDF7BBF9E80003D538A373
:10BB100002E038A201E03DA33DA208213846FDF72E
:10BB2000AFF9641CB442AED3BDE8FC8194ED00E0F3
:10BB3000456E61626C65640044697361626C656442
:10BB4000000000004D50552053746174653A202563
:10BB5000732C20257520756E696669656420726591
:10BB600067696F6E732061766961626C652E0D0A7C
:10BB70000D0A0000526567696F6E2025753A2045F1
:10BB80006E61626C65640D0A00000000092D204C96
:10BB90006F636174696F6E3A093078253038582DBB
:10BBA000307825303858202873697A653A20257511
:10BBB000206279746573290D0A000000092D204167
:10BBC00063636573733A0925730D0A00092D2054C8
:10BBD0007970653A090925730D0A0000092D204383
:10BBE000616368696E673A0925730D0A00000000F9
:10BBF000584E0000526567696F6E2025753A2044E3
:10BC0000697361626C65640D0A0000002D2D0000EF
:10BC1000092D20466C6167733A0925730D0A0D0AD8
:10BC20000000000008B5012905D08168D1F848134B
:10BC3000C1F3400129B10022BDE808401146FDF7DB
:10BC40007DB951680091136802A20221FDF718F92D
:10BC500008BD000025733A20756E6B6E6F776E20FD
:10BC6000706172616D657465723A2025730D0A000A
:10BC700002480068C0F307207047000090ED00E024
:10BC8000C0F30260082813D2DFE800F00406080AB7
:10BC90000C0E101007A0704708A0704709A070474D
:10BCA0000AA070470BA070470CA070470DA070470A
:10BCB0000EA070472D2D2F2D2D00000052572F2D37
:10BCC0002D00000052572F524F00000052572F52A4
:10BCD000570000003F3F2F3F3F000000524F2F2DE5
:10BCE0002D000000524F2F524F000000556E6B6E1A
:10BCF0006F776E0010B5C0F3C241C0F34043C0F38C
:10BD0000004200F47C100404240C17D10014152800
:10BD100014D2DFE800F00B0B0D0F0B0B0B0B0B130A
:10BD200013110B13130B0B1313130B000A4810BD45
:10BD30000AA010BD0BA010BD0CA010BD042908D393
:10BD40008807000F40EA43000B49104351F82000D8
:10BD500010BD0148383010BDB4BC000057542F57F7
:10BD60005400000057422F574200000057425741ED
:10BD70002F57425741000000E800002000F47C10DB
:10BD80000104090C15D10114152912D2DFE801F0C4
:10BD90000B0D18180B0D1616181111181611111677
:10BDA0000F1111110F0008A070470EA0704712A0CC
:10BDB0007047C10C042905D3400301D510A070477A
:10BDC00014A0704715A070475374726F6E676C793A
:10BDD0002D6F7264657265642C20536861726561B1
:10BDE000626C65004465766963652C2053686172F6
:10BDF0006561626C650000004465766963650000FA
:10BE00004E6F726D616C2C20536861726561626C5B
:10BE1000650000004E6F726D616C000052657365C5
:10BE200072766564206F7220496D706C656D656E09
:10BE3000746174696F6E20446566696E65640000A4
:10BE4000094902220A60BFF36F8FBFF34F8F0A1DAB
:10BE5000106006480268002AFCD000200860BFF38A
:10BE60006F8FBFF34F8F704704E5014000E401403E
:10BE700070B50E4C01232360BFF36F8FBFF34F8F5C
:10BE800000230B4D08E000BF51F8236040F8236009
:10BE90002E68002EFCD05B1C9342F5D3002020605E
:10BEA000BFF36F8FBFF34F8F70BD000004E50140FB
:10BEB00000E4014000F180410868002210B1012037
:10BEC0000A607047104670477047000010B50400C4
:10BED00004D105494FF4F670F7F7CCFB204600F08B
:10BEE000BBFAA168081A10BD38C100002DE9F04165
:10BEF00090460D4604004FF0000703D123A1B32064
:10BF0000F7F7B8FB1DB921A1B420F7F7B3FB002068
:10BF1000F7F742FB204600F0A1F830B105270020DA
:10BF2000F7F768FB3846BDE8F08120680668B8F18D
:10BF3000000F05D10168204600F046F9216808602D
:10BF4000E268012A0CD0022A0ED0042A11D06068BF
:10BF5000082A13D006FB02012846F5F7C3FADEE7EC
:10BF60006068805D2870DAE7606830F81600288025
:10BF7000D5E7606850F826002860D0E700EBC601DE
:10BF8000D1E90001C5E90001C9E700002E2E5C2EB1
:10BF90002E5C2E2E5C2E2E5C2E2E5C2E2E5C636F65
:10BFA0006D706F6E656E74735C6C696272617269DC
:10BFB00065735C71756575655C6E72665F717565DC
:10BFC00075652E630000000070B514460E4605002E
:10BFD00004D113A14FF4A170F7F74CFB26B910A1BF
:10BFE00040F24310F7F746FB4FF00000002C12D050
:10BFF000F7F7D2FA287C78B12846FFF767FF84422A
:10C0000000D3044622463146284601F010F90020AC
:10C01000F7F7F0FA204670BDA868A042F2D8F0E722
:10C020002E2E5C2E2E5C2E2E5C2E2E5C2E2E5C2E4A
:10C030002E5C636F6D706F6E656E74735C6C69629D
:10C040007261726965735C71756575655C6E726647
:10C050005F71756575652E630000000010B5040002
:10C0600004D107A14FF4F270F7F704FB21680868C8
:10C070004968884201D1012010BD002010BD000098
:10C080002E2E5C2E2E5C2E2E5C2E2E5C2E2E5C2EEA
:10C090002E5C636F6D706F6E656E74735C6C69623D
:10C0A0007261726965735C71756575655C6E7266E7
:10C0B0005F71756575652E630000000070B5040042
:10C0C00003D108A16420F7F7D5FA20680568416814
:10C0D000204600F079F8A84201D1012070BD00206F
:10C0E00070BD00002E2E5C2E2E5C2E2E5C2E2E5C43
:10C0F0002E2E5C2E2E5C636F6D706F6E656E74738A
:10C100005C6C69627261726965735C717565756595
:10C110005C6E72665F71756575652E630000000068
:10C1200010B5040004D104A14FF4F970F7F7A2FA96
:10C130002068806810BD00002E2E5C2E2E5C2E2EF6
:10C140005C2E2E5C2E2E5C2E2E5C636F6D706F6EDF
:10C15000656E74735C6C69627261726965735C713F
:10C16000756575655C6E72665F71756575652E6364
:10C170000000000010B5040004D104A14FF4FC70CD
:10C18000F7F778FA21680020886010BD2E2E5C2E0B
:10C190002E5C2E2E5C2E2E5C2E2E5C2E2E5C636F63
:10C1A0006D706F6E656E74735C6C696272617269DA
:10C1B00065735C71756575655C6E72665F717565DA
:10C1C00075652E630000000070B50C46050003D1B4
:10C1D00005495120F7F74EFAA868A04201D9601C22
:10C1E00070BD002070BD000038C1000070B514465D
:10C1F0000D46060004D110A140F2AF10F7F73AFA4D
:10C2000025B90DA14FF4D870F7F734FA4FF00000BC
:10C21000002C10D0F7F7C0F9304600F0FCFF844244
:10C2200000D3044622462946304600F0C1FF0020D4
:10C23000F7F7E0F9204670BD2E2E5C2E2E5C2E2ED8
:10C240005C2E2E5C2E2E5C2E2E5C636F6D706F6EDE
:10C25000656E74735C6C69627261726965735C713E
:10C26000756575655C6E72665F71756575652E6363
:10C27000000000002DE9F0410E4604004FF00008D8
:10C2800003D12CA16F20F7F7F5F91EB929A1702071
:10C29000F7F7F0F90020F7F77FF92046FFF70EFFD8
:10C2A000070009D0207C38B14FF004080020F7F7D0
:10C2B000A1F94046BDE8F081206845684168204604
:10C2C000FFF782FF2168486037B120680168204687
:10C2D000FFF77AFF21680860E268012A14D0022A79
:10C2E00016D0042A19D0082A1CD06068314605FBF4
:10C2F0000200F5F7F7F8204600F08DFF21688A6804
:10C300008242D3D28860D1E7616830784855F2E73D
:10C310006168308821F81500EDE76168306841F800
:10C320002500E8E7D6E90001626802EBC502C2E930
:10C330000001E0E72E2E5C2E2E5C2E2E5C2E2E5C55
:10C340002E2E5C2E2E5C636F6D706F6E656E747337
:10C350005C6C69627261726965735C717565756543
:10C360005C6E72665F71756575652E630000000016
:10C370002DE9F04F8046806889B0D0F84803C0F3BB
:10C38000400038B109B04046BDE8F04F00221146E8
:10C39000FCF7D4BD012907D909B04046BDE8F04FEC
:10C3A0001FA20221FCF76CBD2249DFF88CB0A1EB83
:10C3B0000B001C21B0FBF1F7002529E0C5EBC501FE
:10C3C0000BEB81042046D4E9026AFFF7A9FE8146FF
:10C3D000204600F041F8642209FB02F14243B1FB20
:10C3E000F6F1B2FBF6F26369247CB4B10FF24C0CA7
:10C3F000CDF81CC0CDF800A0CDE90596CDE901200F
:10C40000CDE90361104A08214046FCF739FD6D1C57
:10C41000BD42D3D309B0BDE8F08F0FF2300CE7E78F
:10C4200042616420617267756D656E7420636F751B
:10C430006E74000054140100C81301004E6F206F89
:10C44000766572666C6F7700700701004F766572D3
:10C45000666C6F770000000010B5040004D108A1DD
:10C4600040F2D710F7F706F90020F7F795F82046C5
:10C4700000F0D1FE04460020F7F7BCF8204610BDBE
:10C480002E2E5C2E2E5C2E2E5C2E2E5C2E2E5C2EE6
:10C490002E5C636F6D706F6E656E74735C6C696239
:10C4A0007261726965735C71756575655C6E7266E3
:10C4B0005F71756575652E630000000070B50D46EF
:10C4C000060003D10BA11420F7F7D4F81DB909A178
:10C4D0001520F7F7CFF8746804E0B2682946904752
:10C4E00018B1246820680028F7D1206828602560EA
:10C4F00070BD00002E2E5C2E2E5C2E2E5C2E2E5C2F
:10C500002E2E5C2E2E5C636F6D706F6E656E747375
:10C510005C6C69627261726965735C736F72746C72
:10C520006973745C6E72665F736F72746C69737436
:10C530002E63000010B5040003D103A13D20F7F7DE
:10C5400099F8206810BD00002E2E5C2E2E5C2E2E39
:10C550005C2E2E5C2E2E5C2E2E5C636F6D706F6ECB
:10C56000656E74735C6C69627261726965735C7329
:10C570006F72746C6973745C6E72665F736F7274E1
:10C580006C6973742E63000010B5040003D103A11D
:10C590003720F7F76FF86068006810BD2E2E5C2E0C
:10C5A0002E5C2E2E5C2E2E5C2E2E5C2E2E5C636F4F
:10C5B0006D706F6E656E74735C6C696272617269C6
:10C5C00065735C736F72746C6973745C6E72665FB2
:10C5D000736F72746C6973742E63000010B504007D
:10C5E00003D105A12B20F7F745F8616808680028FA
:10C5F00001D002680A6010BD2E2E5C2E2E5C2E2EFD
:10C600005C2E2E5C2E2E5C2E2E5C636F6D706F6E1A
:10C61000656E74735C6C69627261726965735C7378
:10C620006F72746C6973745C6E72665F736F727430
:10C630006C6973742E63000070B50C46050003D15D
:10C640000BA14320F7F716F81CB909A14420F7F70E
:10C6500011F80021686806E0A24203D12168016058
:10C66000012103E010460268002AF5D1084670BD9A
:10C670002E2E5C2E2E5C2E2E5C2E2E5C2E2E5C2EF4
:10C680002E5C636F6D706F6E656E74735C6C696247
:10C690007261726965735C736F72746C6973745CD8
:10C6A0006E72665F736F72746C6973742E630000D0
:10C6B0000C4A10B502F58C730EE0991AC91001EB03
:10C6C000D171491002EBC1010C68844201D90B46BB
:10C6D00002E005D201F108029A42EED3002010BD1B
:10C6E000486810BDCCF0000000B5FFF7E1FF00285E
:10C6F00000D1014800BD0000B8F0000030B50506CB
:10C7000000F00F030E4C03EB830004EB80000AD50E
:10C71000082B03D30B480160001D09E0C0F8001688
:10C72000C0F8042630BD082B04D307480160001D63
:10C73000026030BDC0F80017C0F8042730BD00000B
:10C7400000700240A0760240A077024010B5044677
:10C7500000F00F00092804D30BA140F29640F6F731
:10C7600089FF21064FF0010004F00F0200FA02F0E9
:10C7700001D5114901E01049091D0968014201D0A4
:10C78000012010BD002010BD2E2E5C2E2E5C2E2E02
:10C790005C2E2E5C2E2E5C2E2E5C6D6F64756C658F
:10C7A000735C6E7266785C68616C5C6E72665F75F5
:10C7B0007362642E680000001075024070B5044674
:10C7C000000604D415A140F29B30F6F753FF04F0A5
:10C7D0000F00082804D311A14FF46770F6F74AFF41
:10C7E000200704D10DA140F29D30F6F743FF01F080
:10C7F000CFFD2046FAF790F9817B0125032902D06D
:10C800000068002809D12046FAF752F98540E9432B
:10C81000BDE870401148FBF7A7BD70BD2E2E5C2E01
:10C820002E5C2E2E5C2E2E5C2E2E5C2E2E5C636FCC
:10C830006D706F6E656E74735C6472697665727329
:10C840005F6E72665C757362645C6E72665F647262
:10C85000765F757362642E6300000000380100206B
:10C8600038B50446000604D41B4940F2BB30F6F745
:10C8700001FF04F00F00082804D217494FF46F702D
:10C88000F6F7F8FE01F084FD2046FAF745F9817BC2
:10C890000125032915D00068002811D12046FAF798
:10C8A00007F98540E9430D48FBF75EFD0C480B494D
:10C8B000806800900C398DF80240496868468847C6
:10C8C00038BD2046FAF7F4F88540E943BDE8384022
:10C8D0000248FBF749BD0000DCE3000038010020FE
:10C8E000D0EA000038B50446000604D51FA14FF475
:10C8F0007F70F6F7BFFE04F00F00082804D31BA1D9
:10C9000040F2FD30F6F7B6FE200704D117A140F241
:10C91000FE30F6F7AFFE01F03BFD2046FAF7FCF8DB
:10C92000817B0125032902D0006848B11AE0204626
:10C93000FAF7BEF88540E9431C48FBF715FD11E006
:10C940002046FAF7B5F88540E9431848FBF70CFD97
:10C9500017481649006900900C398DF80240496863
:10C9600068468847BDE8384001F058BD2E2E5C2E41
:10C970002E5C2E2E5C2E2E5C2E2E5C2E2E5C636F7B
:10C980006D706F6E656E74735C64726976657273D8
:10C990005F6E72665C757362645C6E72665F647211
:10C9A000765F757362642E6300000000380100201A
:10C9B000D0EA000070B50546000605F00F0402D568
:10C9C000092C09D301E0092C0BD30D4940F23E405C
:10C9D000F6F750FE280604D5094940F23F40F6F725
:10C9E00049FE082C05D307480068C10300D5002084
:10C9F00070BD054901EB8400D0F8A00470BD0000B3
:10CA0000D8A60000C074024000700240024940589D
:10CA1000002800D0012070470070024004490844FB
:10CA200000210160BFF36F8FBFF34F8F704700008D
:10CA30000070024003490860BFF36F8FBFF34F8F50
:10CA4000704700000074024002480068002800D0CF
:10CA5000012070472C7502400449084401210160FF
:10CA6000BFF36F8FBFF34F8F70470000007002401D
:10CA7000084810B5007918B907A19520F6F7FAFD16
:10CA800000F032F91249012008600249091F0870BC
:10CA900010BD0000440100202E2E5C2E2E5C2E2E98
:10CAA0005C2E2E5C2E2E5C2E2E5C6D6F64756C657C
:10CAB000735C6E7266785C647269766572735C73BF
:10CAC00072635C6E7266785F636C6F636B2E63007B
:10CAD00018050040084810B5007918B907A1D420FE
:10CAE000F6F7C8FD4FF48070FCF759FD012081076F
:10CAF000C1F80403086010BD440100202E2E5C2EF6
:10CB00002E5C2E2E5C2E2E5C2E2E5C2E2E5C6D6FDF
:10CB100064756C65735C6E7266785C647269766568
:10CB200072735C7372635C6E7266785F636C6F6362
:10CB30006B2E630010B50A4C207918B909A1DC20CE
:10CB4000F6F798FD15490120086015494FF00110CE
:10CB50000A6802F001128242FAD00020607110BD12
:10CB6000440100202E2E5C2E2E5C2E2E5C2E2E5C80
:10CB70002E2E5C2E2E5C6D6F64756C65735C6E7210
:10CB800066785C647269766572735C7372635C6EFE
:10CB90007266785F636C6F636B2E63000400004005
:10CBA0000C04004010B5040003D108A17C20F6F766
:10CBB00061FD144900200A790AB1852010BD0122C7
:10CBC0000C600A7100224A7110BD00002E2E5C2EEE
:10CBD0002E5C2E2E5C2E2E5C2E2E5C2E2E5C6D6F0F
:10CBE00064756C65735C6E7266785C647269766598
:10CBF00072735C7372635C6E7266785F636C6F6392
:10CC00006B2E63004401002070B54FF480763046EF
:10CC1000FCF7BEFC114CB50560B13046FCF7BFFC1B
:10CC20000120C5F80803607920B9012060712168EE
:10CC3000002088474FF482763046FCF7A9FC002894
:10CC40000AD03046FCF7ABFC0220C5F80803216887
:10CC5000BDE870400120084770BD0000440100207D
:10CC6000094810B5007918B908A1BF20F6F702FDF0
:10CC70004FF48270FCF793FC02204107C1F80403D3
:10CC800010490120086010BD440100202E2E5C2EAA
:10CC90002E5C2E2E5C2E2E5C2E2E5C2E2E5C6D6F4E
:10CCA00064756C65735C6E7266785C6472697665D7
:10CCB00072735C7372635C6E7266785F636C6F63D1
:10CCC0006B2E630008000040002802D0014980015B
:10CCD0000847704711EB00000121B1EB507F01D1F3
:10CCE000012070470020704707480068012110F0BC
:10CCF000010F08D14FF0E020E02280F80024C0F8B6
:10CD00008012C0F80011704700E100E00748006899
:10CD1000012110F0010F08D14FF0E020E02280F84F
:10CD20000024C0F88012C0F80011704700E100E054
:10CD300070B5040003D10DA14620F6F79BFC194DF8
:10CD4000287808B1852070BD20781749C0F34000CD
:10CD5000086015492078083900F001000860FFF7E5
:10CD6000D5FF01202870002070BD00002E2E5C2E03
:10CD70002E5C2E2E5C2E2E5C2E2E5C2E2E5C6D6F6D
:10CD800064756C65735C6E7266785C6472697665F6
:10CD900072735C7372635C6E7266785F706F7765D6
:10CDA000722E63004C0100208005004070B54FF0EA
:10CDB0008040D0F80453324C68070CD54FF484708F
:10CDC000FFF778F838B1606818B92EA1E020F6F7BF
:10CDD00051FC60688047A8060DD54FF48A70FFF7B4
:10CDE00069F840B1A06818B926A1E820F6F742FC1E
:10CDF000A1680020884768060DD54FF48C70FFF7B6
:10CE000059F840B1A06818B91EA1EF20F6F732FC1E
:10CE1000A1680120884728060DD54FF48E70FFF7D2
:10CE200049F840B1E06818B916A1F820F6F722FCDD
:10CE3000E16800208847E8050DD54FF49070FFF7B2
:10CE400039F840B1E06818B90EA1FF20F6F712FCDE
:10CE5000E16801208847A80511D54FF49270FFF7CB
:10CE600029F800280BD0E06820B906A14FF48370A0
:10CE7000F6F700FCE168BDE870400220084770BD8D
:10CE80004C0100202E2E5C2E2E5C2E2E5C2E2E5C55
:10CE90002E2E5C2E2E5C6D6F64756C65735C6E72ED
:10CEA00066785C647269766572735C7372635C6EDB
:10CEB0007266785F706F7765722E63004FF0804105
:10CEC0004FF46070C1F8080370474FF080414FF491
:10CED0006070C1F80403704703490022CA6000680B
:10CEE000002800D0C86070474C0100200149002094
:10CEF000C86070474C01002010B5124C606898B1B2
:10CF0000606840694068042808D36068042140696B
:10CF1000008801EB00400CA1FEF7EEFA606800F01B
:10CF20006FFF0020606010BD0A4841680229FAD3F3
:10CF30000088022101EB0040BDE8104006A1FEF789
:10CF4000DBBA000064010020436F6D7061726520E0
:10CF50004556540050040020436F6D706172652087
:10CF60006576656E7420627574206E6F20616374DF
:10CF70006976652074696D65722028616C726561DF
:10CF800064792073746F707065643F29000000003D
:10CF900070B516484168042906D30088042101EBC6
:10CFA000004013A1FEF7A8FA1548416829B141686D
:10CFB0004968406821F07F41416000F0A9FD04000C
:10CFC00013D04FF080756068A84203D2204600F06D
:10CFD00017FF03E0606820F07F4060602046FFF7A5
:10CFE000A9FA002801D00446EDE770BD50040020E6
:10CFF0004F766572666C6F772045565400000000CE
:10D00000640100202DE9F84317460C0005462BD09B
:10D01000DFF870804646D8F80000F7F771FF384413
:10D0200087B23068F7F76CFFA968498A081AB0FB25
:10D03000F7F086B22046F7F763FFA968381A87B27F
:10D04000088BB0FBF6F206FB1202401C088382B18B
:10D0500023460DA207212846FBF712FF3946284632
:10D06000BDE8F843F9F7CEBAA96800200883BDE807
:10D07000F883009405A207212846D8F80030FBF772
:10D08000FFFEEBE750020020257300000D0A257318
:10D090002573000010B50C46017A052908D0407AA6
:10D0A00038B1084808A102682046FDF765FB00E09A
:10D0B0001AB106A12046FDF75FFB2046BDE81040EF
:10D0C000FDF79ABBE4020020257300000D0A000062
:10D0D00038B5C3880D46044633B116A0009017A298
:10D0E00018A12846FDF748FB217A052920D0607A4F
:10D0F00048B1A088FEF7BEF8184951F8202018A1C1
:10D100002846FDF739FB2846216800F0DDFFA0889E
:10D110000021FEF71FFB03461049207A143951F80D
:10D12000202001B02846BDE830400EA1FDF724BB09
:10D1300038BD00001B5B306D000000001B5B313B05
:10D1400033316D0025734C6F67732064726F70709C
:10D150006564202825642925730D0A00E402002057
:10D16000257300003C25733E2025733A2000000003
:10D17000EFF30580C005C00D01D001207047EFF32B
:10D18000148040F30000401C7047000008B50022E6
:10D190006946FEF7ABFE002806D104488169491CA8
:10D1A00081610098FEF7B3FB08BD0000600200201B
:10D1B0002DE9F04104460068174688460568406836
:10D1C000854201D8461B02E0A068461B761CE26837
:10D1D0006068B74205FB02010CD87A434046F4F779
:10D1E00081F9A168E819884200D900202168086007
:10D1F000BDE8F08102FB06F52A464046F4F772F9D5
:10D20000E268BE1B724308EB05006168F4F76AF937
:10D2100020680660ECE701680A684968914201D31A
:10D22000881A70478068801A0844401C70472DE9AE
:10D23000F047164689460446FEF748FE80462068B9
:10D24000A168426840688F1A6168E2687F1C00FB31
:10D250000210BE420FD872434946F4F743F92068E2
:10D260004168A2683144914202D84168314400E0EB
:10D270000021416018E002FB07F52A464946F4F711
:10D2800031F9E268F71B7A4309EB05016068F4F7AE
:10D2900029F920684760B04506D2206841682046D9
:10D2A000FEF792FF216808602046FFF7B4FF21686F
:10D2B0008A68824200D28860BDE8F0872DE9F04795
:10D2C0009246894604004BD02078212805D05E285C
:10D2D00003D000270126002035E00127641CF9E770
:10D2E00000262F2D02D05C2D04D00CE04FF0FF3033
:10D2F000BDE8F0875FEACA7006D114F8010B514609
:10D30000FAF711F8C5B25DB320782D282AD16078DC
:10D310005146FAF708F810F0FF0023D05D2821D01D
:10D32000A41C5C280AD15FEACA7107D114F8010B6A
:10D330005146F9F7F8FF10F0FF00D9D04D4503DC56
:10D34000814501DC0120804614F8010B5146F9F7B4
:10D35000EAFFC5B25D2DC3D1002EC1D1B84504D1BD
:10D360000020C5E74D45EFD1ECE72046C0E710B5FA
:10D3700010461A46F4F7B6F8002010BD084670476C
:10D3800010B50446F9F759FA08B1FFF701FE00217C
:10D390002046F9F76BF908B1FFF7AEFD204600F023
:10D3A000BBFD2046BDE81040AFF300802DE9F047FB
:10D3B000334C814600264FF0040800BF00F0A8FB64
:10D3C000002854D04768606840686168C1B16168EE
:10D3D00000294AD0B84248D96068007E80B16068B0
:10D3E00040694068042807D360684069018808EBF9
:10D3F000014024A1FEF780F861682748FFF75EF836
:10D4000000F08CFB054640694168042906D3018879
:10D410003A4608EB014021A1FEF772F86A68184805
:10D420004FF47A7300210830F9F728FA80B10D28FB
:10D4300011D021499C20F6F71DF96869416804293B
:10D44000BCD3018808EB01401CA1FEF755F8B5E7F5
:10D45000606820B106E0284600F0D2FCEDE74846BF
:10D46000F9F7F0F96560002EA8D1BDE8F087606893
:10D470000028FAD14846BDE8F047F9F7F1B90000B5
:10D480006401002054696D657220707265656D706D
:10D490007465642E00000000C4EB000041637469F1
:10D4A000766174696E672074696D657220284343E4
:10D4B0003A2564292E00000088FB000054696D6540
:10D4C000722065787069726564206265666F726546
:10D4D000207363686564756C656420746F205254B2
:10D4E000432E0000342800D93420C01C20F0030053
:10D4F00070470020704700002DE9FE4308790C4674
:10D50000012804D0022805D0032872D172E012222B
:10D51000404977E0B4F80700092800D9092081467E
:10D5200009264FF00008F5F7DFF925E0686820B913
:10D5300039A140F29720F6F79DF86868406820B955
:10D5400035A14FF42670F6F795F80027009700E014
:10D550007F1C686801230022D0F804C02946684671
:10D56000E0470028F4D1297A3E4401EB080000F09E
:10D57000FF082846F5F71CFA0500D7D102A8F5F7F1
:10D58000ADFB02990546894504D923A140F2AD209F
:10D59000F6F770F81F494A4612312846F3F7A2FF02
:10D5A00085F804806E80F5F72BFA18B1E87940F021
:10D5B0002000E871F5F798F90146264880E8220234
:10D5C000B4F80710C1600020F5F7E6FF114980208C
:10D5D0000839F5F713FC040005D10E4980201039F5
:10D5E000F5F7D8FA04460020F6F704F82046BDE81F
:10D5F000FE830DE0E078B4F80510F5F79FFF010019
:10D6000006D00A7803B0601CBDE8F043F5F736BBDE
:10D610000620ECE75CEC00002E2E5C2E2E5C2E2EFD
:10D620005C2E2E5C2E2E5C2E2E5C636F6D706F6EEA
:10D63000656E74735C6C69627261726965735C7546
:10D640007362645C6170705F757362645F636F7254
:10D65000652E63008815002038B50D466846F5F73D
:10D660003DFB04460098022804D20CA140F26F2032
:10D67000F6F700F8002020802078174940F00100DC
:10D68000207049784908C90702D040F00200207094
:10D6900002222146681CF5F7F1FA38BD2E2E5C2EC9
:10D6A0002E5C2E2E5C2E2E5C2E2E5C2E2E5C636F3E
:10D6B0006D706F6E656E74735C6C696272617269B5
:10D6C00065735C757362645C6170705F75736264CE
:10D6D0005F636F72652E6300AC010020F8B50C46E5
:10D6E000070004D142A140F22930F5F7C3FF24B965
:10D6F0003FA140F22A30F5F7BDFF607810F0600FCF
:10D700002AD10006494DA0784FF0000626D520B159
:10D71000062808D008281FD10BE021463846BDE86E
:10D72000F840FFF799BF21463846BDE8F840FFF7BB
:10D73000E3BE6846F5F7D2FA01462878052802D0FC
:10D74000042803D008E00120087000E00E700122D8
:10D75000601CF5F793FAF8BD0620F8BD0A28FBD245
:10D76000DFE800F0051E051305060505052DF3E7A6
:10D770002878032803D0042801D0052824D1F4F701
:10D78000EDFE042000F050FD15E0B4F80300012880
:10D79000E2D1F5F735F980B1687840F0020009E090
:10D7A000B4F803000128D7D1F5F72AF928B1687831
:10D7B00020F0020068700020F8BD0F20F8BD287826
:10D7C000052803D0042801D00820F8BDE07818B15E
:10D7D000012805D00720F8BDF4F7C0FE042002E0C0
:10D7E000F4F7D4FE052000F01FFD3046F8BD000020
:10D7F0002E2E5C2E2E5C2E2E5C2E2E5C2E2E5C2E63
:10D800002E5C636F6D706F6E656E74735C6C6962B5
:10D810007261726965735C757362645C6170705F7C
:10D82000757362645F636F72652E6300AC010020E4
:10D83000F8B50546407810F0600F31D120486C797A
:10D84000A978007821B1012923D0032928D111E03A
:10D85000052801D0200729D16846F5F73FFA06468A
:10D860002046FCF78FFA308002223146681CF5F71B
:10D8700005FAF8BD04F00F01082911D2B5F803101C
:10D8800071B9052801D0200710D12046FCF760FAB5
:10D8900014E004F00F01082902D2B5F8031009B111
:10D8A0000620F8BD052803D0200701D00820F8BDC8
:10D8B0002046FCF723F92046FCF77CFA0020F8BD4F
:10D8C000AC010020FEB50C46050004D12F494FF4F1
:10D8D000D170F5F7CFFE24B92C4940F2A310F5F72B
:10D8E000C9FE60784FF00606010642D5C0F341112B
:10D8F00011B1012924D125E000F01F0001281FD11A
:10D90000A07806281CD10020019002A8F5F7E6F9BE
:10D91000064601A80090E278217933462846F4F7BC
:10D9200083FF05280CD00198402803D31749A32072
:10D93000F5F7A0FE3146601C019AF5F79FF9FEBD90
:10D940000620FEBD2846F6F7CDFAF5F71DFFA178B3
:10D95000212903D1B4F80710072901D03046FEBDB4
:10D96000072200F10C0103B0601CBDE8F040F5F7A0
:10D9700085B9C0F341100028F0D00128E0D103B0F0
:10D9800021462846BDE8F04000F046B814FC0000EF
:10D99000F8B50B4651780646144611F0600F25D1B4
:10D9A0001C480906A17800781ED511B10A291DD19D
:10D9B00009E005281ED16846F5F790F901460020D8
:10D9C000088002220CE0052814D16846F5F786F994
:10D9D000054619463046F5F773FC287001222946A2
:10D9E000601CF5F74BF9F8BD0B2901D00620F8BDF6
:10D9F000052801D00820F8BDB4F80300FF2801D99C
:10DA00000720F8BDD27819463046BDE8F840F5F752
:10DA100029BC0000AC010020F0B585B00D460746DA
:10DA2000F6F760FAF5F7B0FE0446A878002620283D
:10DA300002D022282FD12BE0B5F8070007282AD1E1
:10DA40003846F6F74FFA0446F5F79EFEA9780170BE
:10DA5000E9794170811C019602960091407801900D
:10DA60000020F5F799FD69460020F5F713FA050047
:10DA700008D11D4803A90068CDE903040020F5F78B
:10DA800089F805460020F5F7B5FD284605B0F0BD3C
:10DA9000B5F8070008B10620F8E7207DB5F80310B7
:10DAA00000F0010001F00105A182A8421AD00DB1D9
:10DAB000022100E00321384600F078FE95B938468F
:10DAC000F8F7B8FDFBF7E8FF3846F8F7BCFDFBF7C1
:10DAD000E3FFA6612662E6662667666704F1280012
:10DAE000A667A0660020D1E71CEC00000022CA60F7
:10DAF0004A60054A8A60052803D2044A52F8200089
:10DB000000E000200860704784F20000AC020020B2
:10DB10000148FEF739BD0000C4EB00000148FEF7E4
:10DB20005DBD0000C4EB00002DE9F0410746002573
:10DB3000F7F7E6F986B2002F25D0002420E000BFD9
:10DB4000F3F778FC0168385D085CC00716D0601CEC
:10DB500006E03A5C8A5CD20706D06D1CADB2401C70
:10DB600080B2B042F5D309E045B13918751B3819B8
:10DB70006A1C401CF3F7B6FCAEB20025641CA4B2CC
:10DB8000701E8442DCDBBDE8F08100002DE9F84F17
:10DB9000DFF8B0809246894606461F460122694654
:10DBA0001846D8F80850F5F779FDE8B30098002139
:10DBB0000446C01C0AE000BF00EA05025AF821C072
:10DBC00008EB8202401C491CC2F80CC0B942F3D3D6
:10DBD000BA46370CF8F740FD8346FDF769FDB842B9
:10DBE00004D8194940F28310F5F744FD601C284021
:10DBF00008EB800047EA0B41C160D8F80C044746A7
:10DC00008047A11C294007EB81012C40C86007EB2D
:10DC10008401C86866F3C5006AF3891069F39F2020
:10DC200020F00300401C00E002E020F00400C86087
:10DC300098F8200402E000BFFDF734FB0028FBD178
:10DC4000BDE8F88F64190020800C010070B50C4607
:10DC5000050003D107A15420F5F70CFD1CB905A15F
:10DC60005520F5F707FD21462846BDE87040F3F73B
:10DC70008EBC00002E2E5C2E2E5C2E2E5C64656DFC
:10DC80006F5F636C695F636D64732E6300000000F7
:10DC900070B50C46050004D108A140F61410F5F744
:10DCA000E9FC24B905A140F61510F5F7E3FC21685D
:10DCB0002868BDE87040F3F76ABC00002E2E5C2E89
:10DCC0002E5C2E2E5C2E2E5C2E2E5C2E2E5C636F18
:10DCD0006D706F6E656E74735C6C6962726172698F
:10DCE00065735C636C695C6E72665F636C692E63FE
:10DCF0000000000070B50546F5F734FC124C0646EE
:10DD00002078F5F72FFC86420AD02846F5F72AFC42
:10DD100020B104F10C00FBF78DFC01E0FBF748FC9F
:10DD20002846F5F72CFC06462078F5F728FC8642B5
:10DD300008D02846F5F723FC10B1FBF75FFD01E0A2
:10DD4000FCF754FC257070BD8C0100202DE9F041DA
:10DD500014460D00064604D11BA140F27A20F5F7C7
:10DD600089FC24B918A140F27B20F5F783FC3046EA
:10DD7000F8F778FB78B9B068FA210789B0F80C8019
:10DD80003046F8F73FFCFA213046F8F7B7FA30464C
:10DD9000F8F768FB10B10620BDE8F081B068008993
:10DDA0002880B068808920802888C01B81B23046D6
:10DDB000F8F716FB2188A1EB080081B23046F8F78E
:10DDC0002DFC0020E8E700002E2E5C2E2E5C2E2E6F
:10DDD0005C2E2E5C2E2E5C2E2E5C636F6D706F6E33
:10DDE000656E74735C6C69627261726965735C63A1
:10DDF0006C695C6E72665F636C692E630000000084
:10DE000070B50446C06818B90F496120F5F732FCB7
:10DE10000E4800250078A0B19CB1207E88B1D4E9DD
:10DE200003108847A06850B1217E41B16168084461
:10DE3000606021460648FEF741FB012501E0002015
:10DE40002076284670BD000088FB00006401002099
:10DE5000C4EB00000948007800280ED0084802688A
:10DE6000521C026007484168032906D30088052137
:10DE700001EB004004A1FDF743BB70470800002000
:10DE80000C000020F8040020636F756E746572202A
:10DE90003D2025640D0A000010B504460020F3F76C
:10DEA0004BFE20B16068D0E90021002090476068F7
:10DEB000D0E9002101209047A068224640F6CD41DC
:10DEC0000068F4F703FB002805D0BDE8104002A16C
:10DED0001B20F5F7CFBB10BD2E2E5C2E2E5C2E2EF8
:10DEE0005C2E2E5C2E2E5C2E2E5C636F6D706F6E22
:10DEF000656E74735C6C69627261726965735C6390
:10DF00006C695C7274745C6E72665F636C695F727C
:10DF100074742E63000000002DE9F84F374D8346DE
:10DF200069462868FAF7F8F904464FF00408002714
:10DF30004FF00109324EDFF8CCA05BE0207820B131
:10DF4000012828D002284CD138E06068017E0029E1
:10DF500047D180F818905846F8F78FFB0146606863
:10DF60004268511A284A914203D9416821F07F4101
:10DF70004160224861680830FEF7A0FA616848698C
:10DF80004268042A2DD34A68018808EB01401FA18A
:10DF9000FDF7B6FA25E061687068814200D17760CC
:10DFA00016480830FEF748FB60684069416804295C
:10DFB00017D3018808EB01401AA110E0FFF7AEFD6E
:10DFC00008B10776FAE786F80090DAF8041003291A
:10DFD00007D3BAF80000032101EB004015A1FDF7BB
:10DFE0008BFA69462868FAF78CF969462868FAF7C7
:10DFF00093F90446002CA1D1BDE8F88FBCEB0000DA
:10E00000640100205004002017FCFF00537461726B
:10E01000742072657175657374202843433A2564D2
:10E02000292E000053746F702072657175657374CA
:10E030002E00000053746F7020616C6C207265714B
:10E04000756573742E000000F8B5114C0D46064638
:10E0500069462068FAF74AF9B8B106704560694622
:10E060002068FAF764F918B10A48F8F7D5FB0AE016
:10E0700009484168022906D30088022101EB0040CB
:10E0800006A1FDF739FA0020F8BD0420F8BD000014
:10E09000BCEB00006C010020500400205363686555
:10E0A00064756C696E6720696E74657272757074E0
:10E0B000656420616E6F746865722073636865645F
:10E0C000756C696E672E0000FEB51A4A6FF0E005A8
:10E0D0005368B1FBF3F411684FF46162B4FBF1F3E0
:10E0E000B3FBF2F2554303EB05153C23B5FBF3F309
:10E0F000A3EB031605EB8606B4FBF1F501FB154413
:10E100004FF47A756543B5FBF1F504EB440C05FB60
:10E1100001F7CCEBC414C7EBC4044FF47A777C430B
:10E12000B4FBF1F10096CDE9015103A1FCF724FB0A
:10E13000FEBD0000C80200205B253032643A253065
:10E1400032643A253032642E253033642C25303346
:10E15000645D200010B50248FAF7F4F8002010BD05
:10E160005C0200202DE9F05F8346DDE90A4A99460A
:10E1700090460D460846012703E000BFB0FBF8F0CB
:10E180007F1C4045FAD2B94500D94F465FEACA70B4
:10E1900012D18CB15FEA8A7002D5B9F1000F01D0BB
:10E1A000202607E0302605E031465846641EF5F784
:10E1B000B9FA0CB1A742F7D35FF00106B9F1010F2C
:10E1C00002D9A9F1010903E0B5FBF6F0404502D3FD
:10E1D00006FB08F6F2E7DFF83C9000BFB5FBF6F06F
:10E1E00000FB165519F800105846F5F79BFAB6FBD8
:10E1F000F8F6002EF2D15FEACA7009D0002C07D0E1
:10E20000A74205D220215846641EF5F78BFAF5E7A0
:10E21000BDE8F09FE6EF000002480068002800D04B
:10E2200001207047B401002007490A78824209D0D2
:10E230000870052803D0487820F002004870034891
:10E24000F4F742BE70470000AC01002048EC00002B
:10E250002DE9FE4F8046486891464FF0010A0C4672
:10E2600028B92068F4F7A4FB08B9A06890B1B9F107
:10E27000400F04D937A140F27110F5F7FBF90026E1
:10E280000096FBF703FFE768834648464F4559D998
:10E29000074657E04FF0000AC8F800A0C8F804A0ED
:10E2A00054E0A068B84201D93D4600E005466168E7
:10E2B00039B10BEB06002A46F3F714F90020606031
:10E2C0000CE058B121680BEB06022B464868D0F8E9
:10E2D00004C004F11000E04701200090A068A7EB03
:10E2E0000507411BA160E0682E44A0EB0500E0603B
:10E2F00005D1009818B12068F4F75AFB2060E06857
:10E3000010B1A068F0B902E04FF0000A1AE02068EE
:10E3100000284FF0000001D0019009E060609EB13C
:10E320004E4511D24FF0000A0EE0A068401CA060DC
:10E330002168012300224868456801A8A8470028F1
:10E34000F3D12061002FACD1C8E900B65046BDE83A
:10E35000FE8F00002E2E5C2E2E5C2E2E5C2E2E5C50
:10E360002E2E5C2E2E5C636F6D706F6E656E7473F7
:10E370005C6C69627261726965735C757362645C1E
:10E380006170705F757362645F636F72652E6300A6
:10E390000249002008600249C87070471C7C024096
:10E3A0002C01002070B50446010600F00F0502D5CF
:10E3B000092D09D301E0092D08D308A140F28920D5
:10E3C000F5F758F9200601D5042000E0282000EBDD
:10E3D0008500BDE87040FEF73FBB00002E2E5C2E8E
:10E3E0002E5C2E2E5C2E2E5C2E2E5C2E2E5C636FF1
:10E3F0006D706F6E656E74735C647269766572734E
:10E400005F6E72665C757362645C6E72665F647286
:10E41000765F757362642E63000000002DE9F04F93
:10E42000514D89B0E878002846D180464FF0010967
:10E430003EE000BF90FAA0F0B0FA80F63046F5F763
:10E4400024F98346F8F768FB0446006820B947A121
:10E4500040F23150F5F70EF95FEA0B6007D5D4E9C9
:10E460000031A28902A89847002836D037E05846E4
:10E47000FBF7C8FDD4E9007182460346A28902A8D1
:10E48000B84707460298D0B1039951451DD20220E2
:10E49000A07309FA06F0C14333480C30F9F764FF62
:10E4A0004248006B00908DF802B069686846884762
:10E4B000D5E902100840BDD109B0BDE8F08F03983E
:10E4C00050B12AA140F24D5004E0514504D027A19B
:10E4D00040F25C50F5F7CEF80FB9C4F8008034492B
:10E4E0008220086085F80390A96809FA06F0814344
:10E4F000A960A06803990844A060DDE902125846AB
:10E50000FEF7FCF8FBF7ACFD18B32A4C4FF482750C
:10E510002846FEF783FA5846FFF744FF0220FEF72D
:10E52000D3FB2846FEF772FA0028F1D01E2000E047
:10E530000220FEF7C9FB20688006F9D50120FEF70E
:10E54000C3FB5846FBF74EFCFEF760FA0028DFD00D
:10E55000B2E75846FFF726FF5846FBF743FCFEF7A5
:10E5600055FA0028F8D0A7E72C0100202E2E5C2EAB
:10E570002E5C2E2E5C2E2E5C2E2E5C2E2E5C636F5F
:10E580006D706F6E656E74735C64726976657273BC
:10E590005F6E72665C757362645C6E72665F6472F5
:10E5A000765F757362642E6300000000D0EA00009D
:10E5B0001C7C0240747402402DE9F8430746002099
:10E5C000F4F7EAFF3846F8F7A7FA06463806294D69
:10E5D0004FF000084FF003094FF0010438461ED4F5
:10E5E000F8F766FAE96804FA00F0884303D0384681
:10E5F000FCF706F810E03846C6F80080F8F758FA3D
:10E60000E96804FA00F081433846E960F8F750FA07
:10E610008440A868A043A86086F80E9024E0F8F72C
:10E6200047FAD5E9022104FA00F061EA0201084242
:10E630001AD03846F8F73CFAE96804FA00F081434A
:10E640003846E960F8F734FA8440A8680443AC60BF
:10E650000948C6F8008086F80E90006800908DF892
:10E660000270696868468847BDE8F8430020F4F7FF
:10E67000C1BF00002C010020D0EA00002DE9F041CC
:10E68000104EB068040CF06824040443012712E023
:10E6900094FAA4F0B0FA80F52846F4F7F6FF00F0FB
:10E6A0000F00082804D22846F4F7EFFFFFF784FF95
:10E6B00007FA05F08443002CEAD140F2FF10B06065
:10E6C000BDE8F0812C010020012238B58A400C49B8
:10E6D0000C468B6813438B606168E468094B050640
:10E6E00002EA040203D5002A09D19A6902E0002A4D
:10E6F00005D1DA6900928DF802006846884738BD76
:10E700002C010020D0EA00002DE9F0411148F4F777
:10E71000E1FD18B1104ACF21F2F77CFD0F48F3F765
:10E72000EFFF18B10C4AD421F2F774FDF4F792FE12
:10E7300018B1094AD921F2F76DFD064E4FF47A74EB
:10E74000403EA701751C3846A847641EFAD1BDE8B3
:10E75000F081000060EA0000A87E000098EF000051
:10E7600002498020C1F800027047000004E000E088
:10E7700010B5082809D009280FD00A2811D00E2872
:10E7800013D1BDE81040F4F7B1BAFBF7F5FD00284E
:10E790000BD1BDE81040F4F7D3BABDE81040F4F750
:10E7A000C3BEBDE81040F4F787BE10BD70B50C467F
:10E7B0000546F5F797FBC269002A04D02146284692
:10E7C000BDE87040104770BD02494968002900D07B
:10E7D000084770473C1500201CB5002913D08268FB
:10E7E000D27D8A420FD008A3D3E90023CDE90023CC
:10E7F00001F12F028DF803208268D17500696A4605
:10E8000003A1FBF7B9FF1CBD1B5B34006D000000CA
:10E81000257300001CB5826899B1927D8A420FD0A1
:10E820000CA2D2E90032CDE9003201F12F028DF8BD
:10E8300005208268917500696A4608A1FBF79CFF74
:10E840001CBD9175006902B0054ABDE8104003A1E6
:10E85000FBF792BF1B5B313B33006D00257300005B
:10E8600060EF000010B50446F6F74AFB002105E012
:10E87000625C3F2A06D02A2A04D0491C8142F7D381
:10E88000002010BD012010BD002070472DE9FC4183
:10E8900080461C4617460E460C48089DF9F75BFD5E
:10E8A00010B11120BDE8FC81A20839463046FDF7C1
:10E8B000DFFA0648F9F746FD33463A46012140465D
:10E8C000CDE90045F8F742FB0020EBE75C020020B1
:10E8D000B8F3000094F30000000000001D5E00008B
:10E8E00000000000E8E8000004F40000E4F3000089
:10E8F00000000000455F000008F40000C0F30000C5
:10E9000000000000815F0000000000000000000027
:10E91000000000000000000010F4000010F40000EF
:10E92000E0E80000895E000018F4000018F4000020
:10E9300000000000B95F00000000000040E9000096
:10E9400070F4000038F400000000000031550000B1
:10E9500078F4000050F40000000000006955000049
:10E9600068F4000020F4000000000000A155000041
:10E970000000000000000000000000000000000097
:10E98000A4F4000080F4000038E9000025540000E1
:10E9900001000000C569000000000000A0E90000BF
:10E9A000FCF50000D4F40000000000004D5600000B
:10E9B00000F60000ACF4000090E90000E957000008
:10E9C00008F60000C0F4000090E90000B55800000F
:10E9D00010F60000D8F5000000000000A959000062
:10E9E0000000000000000000000000000000000027
:10E9F0003CF6000018F6000098E90000D955000028
:10EA00007CFA000078FA00005CFA000000000000C8
:10EA100028000020000000000000000000000000AE
:10EA20000338FDD87047000084FA00006CEA00004B
:10EA3000980700205C0000204400002074130100AF
:10EA40000D00000090FA000078EA0000900C002011
:10EA5000A800002090000020901301000A00000090
:10EA6000C92E000071E7000000000000B8EF0000B0
:10EA7000C000002074000020CCEF0000840C0020B7
:10EA800074EA0000000000008CEA0000DCFA0000DC
:10EA9000C0FA00000000000045B90000D4FA0000F0
:10EAA0009CFA00000000000041BA000000000000D5
:10EAB00000000000000000000000000000FB00005B
:10EAC000E4FA000084EA000025BC00000000000019
:10EAD0000600000301000000060000000600000020
:10EAE000060000000600000006000000060000010D
:10EAF0000500000002000000030000000400000008
:10EB000006000002000000000000000000000000FD
:10EB10000338FDD8704700002D6F0000656E0000BF
:10EB2000F96B00002D6C0000336C0000396C0000A4
:10EB30003F6C0000456C00004B6C0000516C000005
:10EB4000956D0000576C00005D6C0000BD6C00000E
:10EB5000C36C0000C96C0000CF6C0000D56C0000D5
:10EB6000DB6C0000E16C0000E96C0000296E000025
:10EB7000696E0000B16D0000356D000008010C01E8
:10EB80001001140118011C01200124012C01300185
:10EB9000340138013C014001440148014C0150015D
:10EBA00002030405060708090B0C0D0E0F101112C5
:10EBB00013140000000000500003005074010020F6
:10EBC000000007000000000088010020E56100004F
:10EBD000800000000B810000820000008300000024
:10EBE000840D0E030B0000000C000800000009005B
:10EBF00000000A0000000000F1330000C92E0000F0
:10EC00000000000000000000AD37000045380000A3
:10EC1000000000000000000000000000693F00004C
:10EC200000000000593700000000000059370000C4
:10EC30000000000091400000000000000000000003
:10EC40000A000000000000000F000000F3D40000E4
:10EC50000000000051E200008815002012010002AF
:10EC60000000004015190F520001010203010902C2
:10EC70000000000100C0FA00112A0000000000009E
:10EC8000000000000000000000000000BC010020A7
:10EC900078EC00000100020300800000040309007A
:10ECA0002A034E006F0072006400690063002000B8
:10ECB000530065006D00690063006F006E00640022
:10ECC0007500630074006F00720026036E0052002E
:10ECD000460035003200200055005300420020005D
:10ECE0004300440043002000440065006D006F00B5
:10ECF0001A033000300030003000300030003000A7
:10ED0000300030003000300030000E03550073003A
:10ED100065007200200031000001020304000000C1
:10ED200070F4000064FC000000000000D15F0000EF
:10ED3000F800010074FC0000000000008D5A000083
:10ED40009CFC000084FC000000000000B1530000A7
:10ED50000000000058ED0000F8000100D4FC0000A5
:10ED600000000000CD5B0000A8FC0000B0FC00002B
:10ED700000000000F15C0000000000000000000046
:10ED80000000000000000000F8FC000000FD000092
:10ED900050ED000000000000000000000000000036
:10EDA0000338FDD87047000000000000B0ED0000FF
:10EDB000AC0201008802010000000000B1850000E3
:10EDC0000000000000000000000000000000000043
:10EDD000B4020100BC020100A8ED0000B1850000F2
:10EDE00041B0000025B0000009B0000000000000A4
:10EDF000F4ED00009C03010084030100000000000A
:10EE0000B58A0000A00301006C03010000000000AF
:10EE1000DF8A000000000000000000000000000089
:10EE200000000000000000002CEE00009C03010028
:10EE3000A403010000000000A18B0000A00301005A
:10EE40000004010000000000CB8B00000000000067
:10EE500000000000000000000000000000000000B2
:10EE600064EE000070F400004004010000000000A7
:10EE70003189000010F600001404010000000000B9
:10EE80006189000000000000000000000000000098
:10EE900000000000000000009CEE0000B004010033
:10EEA00090040100ECED0000ED890000A8040100D1
:10EEB0006C04010024EE0000098B0000B80401007E
:10EEC000800401005CEE0000C58800000000000026
:10EED0000000000000000000000000000000000032
:10EEE000E4EE000004050100C00401000000000081
:10EEF000F58D000000000000000000000000000090
:10EF0000000000001C0501000C05010000000000CD
:10EF100041870000480501002405010094EE00002F
:10EF200015880000600501004C050100000000008C
:10EF3000F58B00000806010068050100DCEE00000A
:10EF4000D18C000000000000000000000000000064
:10EF50001B37001B38001B45002C20001B5B4A00A0
:10EF60001B5B6D00082008001B5B4B00202D200060
:10EF70001B5B48001B5B366E001B5B324A000000C7
:10EF80000338FDD870471B5B3F336C002D682C2085
:10EF90002D2D68656C700000A015002008EC0000A5
:10EFA000020001060102048281010000000001014B
:10EFB00081010000B14000007D440000BD4400001C
:10EFC00071440000C144000091440000914B0000D6
:10EFD000194C0000394B0000214C0000B54B0000DB
:10EFE0000338FDD87047303132333435363738394D
:10EFF0004142434445466E72665F6673746F726148
:10F0000067655F696E6974006E72665F6673746FC0
:10F01000726167655F756E696E6974006E72665FB6
:10F020006673746F726167655F72656164006E72AA
:10F03000665F6673746F726167655F777269746526
:10F04000006E72665F6673746F726167655F65728A
:10F050006173650000100000040000000100000062
:10F060008577000055E100006FD300008DE80000B7
:10F07000B16B00007DD3000089E8000095780000A6
:10F080000000000088F00000AC020100440701000D
:10F090000000000071C3000000000000000000003C
:10F0A000000000000000000068070100BC02010031
:10F0B00080F0000071C30000556E6B6E6F776E209C
:10F0C0006572726F7220636F64650000000000005B
:10F0D000500B010001000000100A010002000000B6
:10F0E0000408010003000000840A0100040000007D
:10F0F000D80A010005000000B80901000600000060
:10F100005409010007000000C00A010008000000C7
:10F11000CC09010009000000300A01000A000000CB
:10F12000380B01000B000000EC0701000C00000090
:10F13000E40901000D000000880B01000E00000032
:10F14000B00A01000F000000EC0A010010000000EE
:10F15000200B0100110000009C0B0100800000004A
:10F160006C09010081000000A80801008200000075
:10F1700068080100830000004808010084000000C6
:10F18000840801008500000090090100860000004D
:10F19000980A01009000000034090100910000006D
:10F1A0002808010092000000F80901000082000018
:10F1B000000B0100018200004C0A010002820000E5
:10F1C000680A010000840000C408010001840000F6
:10F1D0005C0B0100028400000C09010003840000A4
:10F1E000E80801002D2D2D2D2D2D2D2D2D2D2D43FC
:10F1F000524153484C4F472D2D2D2D2D2D2D2D2D6A
:10F200002D2D2D0D0A000000290000000000000037
:10F210000000000035B2000031B2000025B200004D
:10F2200019B10000A1B0000095B00000000000007E
:10F2300034F200001C050100C80B010000000000B2
:10F24000D96F0000AC0B0100B40B010000000000FE
:10F2500055700000AC020100D40B0100000000005A
:10F26000B570000000000000000000000000000079
:10F2700000000000E80B0100F40B01002CF200007C
:10F280000000000001000000E58100000100000016
:10F29000EDDA0000000000009CF20000D80D010033
:10F2A000640D010084F2000015790000D00D01000A
:10F2B000E00C01008CF2000015790000000E010046
:10F2C000E00D010000000000ED7A0000140E0100C6
:10F2D000F00D010000000000F57A0000AC02010012
:10F2E000040E010000000000457C0000000000004A
:10F2F0000000000000000000000000001C0E0100E3
:10F30000200E010094F20000BD7800000040404053
:10F3100040404040404041414141414040404040E8
:10F320004040404040404040404040404005020294
:10F330000202020202020202020202020220202053
:10F3400020202020202020020202020202029090AF
:10F3500090909090101010101010101010101010AD
:10F360001010101010101010020202020202888801
:10F37000888888880808080808080808080808080D
:10F3800008080808080808080202020240000000F5
:10F390000DF300005072696E74204E6F72646963E1
:10F3A0002053656D69636F6E647563746F72206C52
:10F3B0006F676F2E000000006E6F7264696300005B
:10F3C0005072696E74206561636820706172616D4E
:10F3D0006574657220696E206E6577206C696E6554
:10F3E0002E0000005072696E7420616C6C20656E96
:10F3F000746572656420706172616D6574657273A5
:10F400002E000000616C6C00706172616D00000084
:10F410007072696E74000000707974686F6E00001D
:10F4200053746F70207365636F6E647320636F75C0
:10F430006E7465722E0000005265736574207365EA
:10F44000636F6E647320636F756E7465722E000057
:10F450005374617274207365636F6E647320636F9D
:10F46000756E7465722E000073746F70000000007A
:10F47000726573657400000073746172740000003B
:10F48000446973706C6179207365636F6E64732077
:10F490006F6E207465726D696E616C207363726546
:10F4A000656E0000636F756E746572004578656304
:10F4B000757465206120636F6D6D616E642E000050
:10F4C00052656D6F7665206120636F6D6D616E644E
:10F4D0002E0000004164642061206E65772064790D
:10F4E0006E616D696320636F6D6D616E642E0A4598
:10F4F00078616D706C652075736167653A205B207B
:10F5000064796E616D6963206164642074657374ED
:10F51000205D2077696C6C206164642061206479CF
:10F520006E616D696320636F6D6D616E6420277419
:10F53000657374272E0A496E207468697320657894
:10F54000616D706C652C20636F6D6D616E64206EF3
:10F55000616D65206C656E677468206973206C69E5
:10F560006D6974656420746F203332206368617242
:10F57000732E20596F752063616E2061646420755D
:10F580007020746F20323020636F6D6D616E647314
:10F590002E20436F6D6D616E647320617265206112
:10F5A00075746F6D61746963616C6C7920736F72CF
:10F5B00074656420746F20656E7375726520636F67
:10F5C000727265637420434C4920636F6D706C6583
:10F5D00074696F6E2E00000053686F7720616C6C49
:10F5E0002061646465642064796E616D6963206381
:10F5F0006F6D6D616E64732E0000000061646400C5
:10F60000657865637574650072656D6F7665000079
:10F6100073686F770000000044656D6F6E737472DD
:10F620006174652064796E616D696320636F6D6DCF
:10F63000616E642075736167652E000064796E6188
:10F640006D6963000D0A202020202020202020202A
:10F6500020202E636F3A2E202020202020202020E2
:10F660002020202020202020202027786F2C2020E0
:10F6700020202020202020200D0A202020202020B3
:10F680002020202E2C636F6C6C6C6C632C2E202041
:10F69000202020202020202020202027636B4F4F77
:10F6A0006F3A3A2C2E2E2020202020200D0A2020D8
:10F6B000202020202E3A6F6F6F6F6F6C6C6C6C6C1B
:10F6C0006C6C6C3A272E20202020202E3B644F4F5C
:10F6D0004F4F4F4F6F3A3A3A3B3B3B272E2020206B
:10F6E0000D0A202020276F6B7864646F6F6F6F6C3A
:10F6F0006C6C6C6C6C6C6C6C6C6C6C3B27636B4FE7
:10F700004F4F4F4F4F4F4F4F6F3A3A3A3B3B3B2C87
:10F710002C2C27200D0A2020204F4F4F6B78646F30
:10F720006F6F6F6C6C6C6C6C6C6C6C6C6C6C6C6C10
:10F730006C6C6C64784F4F4F4F4F4F4F6F3A3A3A63
:10F740003B3B3B2C2C2C272E0D0A2020204F4F4FCB
:10F750004F4F4F6B646F6F6C6C6C6C6C6C6C6C6C43
:10F760006C6C6C6C6C6C6C6C6C6C6C64784F4F4F2C
:10F770006F3A3A3A3B3B3B2C2C2C272E0D0A20208B
:10F78000204F4F4F4F4F4F4F4F4F6B786F6C6C6CFC
:10F790006C6C6C6C6C6C6C6C6C6C6C6C6C6C6C63B2
:10F7A00063636C646C3A3A3A3B3B3B2C2C2C272E1F
:10F7B0000D0A2020204F4F4F4F4F4F4F4F4F4F4F6D
:10F7C0004F4F78646F6C6C6C6C6C6C6C6C6C6C6CAC
:10F7D0006C6C6C63636363633A3A3A3A3B3B3B2C31
:10F7E0002C2C272E0D0A2020204F4F4F4F4F4F4FCC
:10F7F0004F4F4F4F4F4F4F4F4F6B78646C6C6C6C4B
:10F800006C6C6C6C6C6C6C63636363633A3A3A3A2D
:10F810003B3B3B2C2C2C272E0D0A2020206B4F4FDE
:10F820004F4F4F4F4F4F4F4F4F4F4F4F4F4F4F4FE8
:10F830004F6B646F6C6C6C6C6C6C6C636363636358
:10F840003A3A3A3A3B3B3B2C2C2C272E0D0A2020EF
:10F85000206B4F4F4F4F4F4F4F4F4F4F4F4F4F4FCB
:10F860004F4F4F4F4F4F4F4F4F78646C6C6C6C63E2
:10F87000636363633A3A3A3A3B3B3B2C2C2C272E8A
:10F880000D0A2020206B4F4F4F4F4F4F4F4F4F4F80
:10F890004F4F4F4F4F4F4F4F4F4F4F4F4F4F4F4F78
:10F8A0006B786F6C636363633A3A3A3A3B3B3B2C49
:10F8B0002C2C272E0D0A2020206B4F4F4F4F4F4FDF
:10F8C0004F4F4F4F4F4F4F4F4F4F4F4F4F4F4F4F48
:10F8D0004F4F4F4F4F4F4F4F6B646C633A3A3A3A2A
:10F8E0003B3B3B2C2C2C272E0D0A202020784F4F01
:10F8F0004F4F4F4F4F4F4F4F4F78646B4F4F4F4FBE
:10F900004F4F4F4F4F4F4F4F4F4F4F4F4F4F4F4F07
:10F91000786F633A3B3B3B2C2C2C272E0D0A202082
:10F9200020784F4F4F4F4F4F4F4F4F4F4F64633AD9
:10F930003A6C646B4F4F4F4F4F4F4F4F4F4F4F4F9E
:10F940004F4F4F4F4F4F4F6B64633B2C2C2C27274F
:10F950000D0A202020784F4F4F4F4F4F4F4F4F4FA2
:10F960004F64633A3A3B3B2C3B63646B4F4F4F4FC2
:10F970004F4F4F4F4F4F4F4F4F4F4F4F4F4F4F786E
:10F980006C3B27270D0A2020202E6C6B4F4F4F4FCA
:10F990004F4F4F4F4F64633A3A3B3B2C2C27272E57
:10F9A0002E3B6F4F4F4F4F4F4F4F4F4F4F4F4F4F7C
:10F9B0004F4F4F4F4F4F78270D0A202020202020F7
:10F9C0002E3B6F4F4F4F4F4F4F64633A3A3B3B2CA8
:10F9D0002E202020202020202E3A784F4F4F4F4FAE
:10F9E0004F4F4F4F4F4F4F643B2E20200D0A20208A
:10F9F00020202020202020202E3A784F4F64633A88
:10FA00002C2E2020202020202020202020202020DC
:10FA100027636B4F4F4F4F6B6C27202020202020F7
:10FA20000D0A202020202020202020202020202EF1
:10FA30006F6427202020202020202020202020202C
:10FA40002020202020202027786B2C202020202000
:10FA5000202020200D0A0D0A0000000064756D6D45
:10FA600079206F7074696F6E2068656C7020737494
:10FA700072696E67000000002D7400002D2D746502
:10FA8000737400007573625F636C693A7E242000B2
:10FA90007274745F636C693A7E2420005072696EE0
:10FAA0007420696E666F726D6174696F6E20616239
:10FAB0006F7574204D50552073746174652E00006D
:10FAC00044756D70204D505520726567697374657B
:10FAD00072732E00696E666F0000000064756D70B1
:10FAE00000000000436F6D6D616E647320666F727D
:10FAF000204D5055206D616E6167656D656E7400B7
:10FB00006D7075002D2D2F2D2D000000574257418F
:10FB10002F2D2D0057422F2D2D00000057542F2D33
:10FB20002D0000002D2D2F574257410057425741BD
:10FB30002F5742574100000057422F57425741006C
:10FB400057542F57425741002D2D2F574200000088
:10FB5000574257412F57420057422F57420000004B
:10FB600057542F57420000002D2D2F5754000000EE
:10FB7000574257412F57540057422F575400000007
:10FB800057542F57540000002E2E5C2E2E5C2E2E24
:10FB90005C2E2E5C2E2E5C2E2E5C636F6D706F6E55
:10FBA000656E74735C6C69627261726965735C74B2
:10FBB000696D65725C6578706572696D656E74619A
:10FBC0006C5C6170705F74696D6572322E630000E9
:10FBD0002E2E5C2E2E5C2E2E5C2E2E5C2E2E5C2E5F
:10FBE0002E5C636F6D706F6E656E74735C6C6962B2
:10FBF0007261726965735C757362645C6170705F79
:10FC0000757362645F636C6173735F626173652EA9
:10FC1000680000002E2E5C2E2E5C2E2E5C2E2E5C9C
:10FC20002E2E5C2E2E5C636F6D706F6E656E74731E
:10FC30005C6C69627261726965735C757362645C45
:10FC4000636C6173735C6364635C61636D5C61705E
:10FC5000705F757362645F6364635F61636D2E637D
:10FC60000000000053797374656D207265736574CC
:10FC70002E00000054726967676572206572726FAA
:10FC8000722E00005072696E74206170706C69632E
:10FC90006174696F6E2073697A652E006170705FA0
:10FCA00073697A65000000007761726E696E6700A3
:10FCB0005761726E696E67206C6F67206D65737334
:10FCC000616765207769746820706172616D657421
:10FCD000657273004572726F72206C6F67206D657C
:10FCE0007373616765207769746820706172616DF4
:10FCF00065746572730000006C6F675F6D736700F9
:10FD000054726967676572206C6F67206D657373E5
:10FD1000616765207769746820646563696D616CEB
:10FD200020617267756D656E747300002E2E5C2EF7
:10FD30002E5C2E2E5C2E2E5C2E2E5C2E2E5C636F87
:10FD40006D706F6E656E74735C6C696272617269FE
:10FD500065735C74696D65725C6578706572696DF8
:10FD6000656E74616C5C6472765F7274632E63009E
:10FD70004461746120627573206572726F7220280D
:10FD800072657475726E2061646472657373206944
:10FD90006E2074686520737461636B206672616D98
:10FDA00065206973206E6F742072656C6174656480
:10FDB00020746F2074686520696E73747275637443
:10FDC000696F6E2074686174206361757365642067
:10FDD000746865206572726F7229000044617461F5
:10FDE00020627573206572726F72202850432076EE
:10FDF000616C756520737461636B656420666F72F6
:10FE00002074686520657863657074696F6E207210
:10FE1000657475726E20706F696E747320746F20D4
:10FE200074686520696E737472756374696F6E208F
:10FE300074686174206361757365642074686520FB
:10FE40006661756C7429000043617573653A2042E0
:10FE500075734661756C74206F6E206120766563E2
:10FE6000746F72207461626C6520726561642064D5
:10FE70007572696E6720657863657074696F6E204E
:10FE800070726F63657373696E672E0054686520C6
:10FE900070726F636573736F722068617320657829
:10FEA00065637574656420616E2053444956206F04
:10FEB00072205544495620696E7374727563746973
:10FEC0006F6E207769746820612064697669736F4A
:10FED00072206F66203000005468652070726F6376
:10FEE0006573736F722068617320617474656D70DF
:10FEF00074656420746F206578656375746520612E
:10FF00006E20696E737472756374696F6E207468A5
:10FF10006174206D616B657320696C6C6567616CE1
:10FF200020757365206F66207468652045505352B4
:10FF3000000000005468652070726F636573736F12
:10FF4000722068617320617474656D7074656420DB
:10FF5000616E20696C6C6567616C206C6F616420F8
:10FF60006F66204558435F52455455524E20746F7A
:10FF7000207468652050432C2061732061207265D5
:10FF800073756C74206F6620616E20696E76616C8B
:10FF9000696420636F6E746578742C206F722061C1
:10FFA0006E20696E76616C6964204558435F5245E6
:10FFB0005455524E2076616C75650000546865207A
:10FFC00070726F636573736F7220617474656D70A6
:10FFD0007465642061206C6F6164206F722073749B
:10FFE0006F72652061742061206C6F636174696F4A
:10FFF0006E207468617420646F6573206E6F742066
:020000040001F9
:100000007065726D697420746865206F70657261C7
:1000100074696F6E0000000041204D656D4D616E8A
:10002000616765206661756C74206F6363757272B9
:10003000656420647572696E6720666C6F617469AF
:100040006E672D706F696E74206C617A792073749D
:1000500061746520707265736572766174696F6E24
:10006000000000004120627573206661756C742089
:100070006F6363757272656420647572696E672060
:10008000666C6F6174696E672D706F696E74206C39
:10009000617A79207374617465207072657365721A
:1000A000766174696F6E00005468652070726F63CA
:1000B0006573736F722068617320617474656D700D
:1000C00074656420746F206578656375746520615C
:1000D0006E20756E646566696E656420696E737402
:1000E00072756374696F6E00496E737472756374B0
:1000F000696F6E20627573206572726F7200000006
:100100005468652070726F636573736F72206861E5
:100110007320617474656D7074656420746F206100
:100120006363657373206120636F70726F636573BF
:10013000736F7200556E737461636B20666F72200B
:10014000616E20657863657074696F6E2072657486
:1001500075726E2068617320636175736564206FCA
:100160006E65206F72206D6F7265206163636573C9
:10017000732076696F6C6174696F6E7300000000A4
:10018000537461636B696E6720666F7220616E20C5
:10019000657863657074696F6E20656E747279201E
:1001A00068617320636175736564206F6E65206F8D
:1001B00072206D6F72652061636365737320766969
:1001C0006F6C6174696F6E73000000005468652085
:1001D00070726F636573736F7220686173206D61F5
:1001E000646520616E20756E616C69676E65642060
:1001F0006D656D6F727920616363657373000000D4
:10020000556E737461636B20666F7220616E20653A
:100210007863657074696F6E2072657475726E2094
:1002200068617320636175736564206F6E65206F0C
:1002300072206D6F7265204275734661756C7473C0
:1002400000000000537461636B696E6720666F7213
:1002500020616E20657863657074696F6E20656ECD
:100260007472792068617320636175736564206FAF
:100270006E65206F72206D6F7265204275734661E6
:10028000756C7473000000005072696E7420737492
:1002900061747573206F662062616C6C6F63206996
:1002A0006E7374616E6365732E0000007374617405
:1002B0007573000062616C6C6F630000436F6D6D5D
:1002C000616E647320666F722042414C4C4F432034
:1002D0006D616E6167656D656E74000025730D0A52
:1002E000092D20456C656D656E742073697A653AD9
:1002F000092564202B202564206279746573206FA2
:100300006620646562756720696E666F726D6174E0
:10031000696F6E0D0A092D2055736167653A0925CD
:1003200075252520282575206F7574206F6620257A
:100330007520656C656D656E7473290D0A092D2035
:100340004D6178696D756D3A09257525252028253B
:1003500075206F7574206F6620257520656C656D3E
:10036000656E7473290D0A0D0A000000456E616206
:100370006C6520636F6C6F7265642073796E746155
:10038000782E000044697361626C6520636F6C6F46
:100390007265642073796E7461782E006F666600F2
:1003A0006F6E000044697361626C6520434C4920A4
:1003B0006563686F2E204172726F777320616E647F
:1003C00020627574746F6E733A204261636B737050
:1003D0006163652C2044656C6574652C20456E64F2
:1003E0002C20486F6D652C20496E736572742061F6
:1003F0007265206E6F742068616E646C65642E0097
:10040000456E61626C6520434C49206563686F2EC0
:100410000000000047657420434C492073746174E8
:1004200069737469637320666F7220746865204C09
:100430006F67676572206D6F64756C652E000000D4
:10044000526573657420434C4920737461746973F9
:100450007469637320666F7220746865204C6F67DF
:10046000676572206D6F64756C652E00546F6767E9
:100470006C6520434C49206563686F2E00000000C6
:10048000434C4920737461746973746963732E00FB
:10049000546F67676C6520636F6C6F72656420735F
:1004A000796E7461782E00006563686F000000004B
:1004B000636F6C6F7273000073746174730000007B
:1004C000417373756D6520383020636861727320E5
:1004D00073637265656E20776964746820616E6409
:1004E0002073656E64207468697320736574746921
:1004F0006E6720746F20746865207465726D696E14
:10050000616C2E0064656661756C7400436C656196
:10051000722073637265656E2E000000636C656106
:100520007200000055736566756C2C206E6F742028
:10053000556E69782D6C696B6520434C4920636F5B
:100540006D6D616E64732E00636C6900436F6D6D39
:10055000616E6420686973746F72792E0000000008
:10056000686973746F727900436F6E736F6C652086
:1005700067657473207465726D696E616C20736356
:100580007265656E2073697A65206F72206173737E
:10059000756D657320383020696E20636173652046
:1005A00074686520726561646F7574206661696C3A
:1005B000732E204974206D757374206265206578F0
:1005C0006563757465642061667465722065616336
:1005D00068207465726D696E616C207769647468F7
:1005E000206368616E676520746F20656E73757235
:1005F0006520636F7272656374207465787420641B
:100600006973706C61792E00726573697A65000098
:10061000436F6D6D616E64206275666665722069F8
:100620007320746F6F2073686F727420746F20650D
:100630007870616E6420616C6C20636F6D6D616EAB
:100640006473206D61746368696E672077696C6498
:1006500063617264207061747465726E0D0A0000CB
:10066000202000002E2E5C2E2E5C2E2E5C2E2E5C6A
:100670002E2E5C2E2E5C636F6D706F6E656E7473C4
:100680005C6C69627261726965735C636C695C63FE
:1006900064635F61636D5C6E72665F636C695F6308
:1006A00064635F61636D2E630000000061646472C7
:1006B0005F69735F77697468696E5F626F756E6496
:1006C0007328705F66732C20706167655F61646476
:1006D000722C20286C656E202A20705F66732D3E78
:1006E000705F666C6173685F696E666F2D3E6572E0
:1006F0006173655F756E6974292900002E2E5C2E6A
:100700002E5C2E2E5C2E2E5C2E2E5C2E2E5C636FAD
:100710006D706F6E656E74735C6C69627261726924
:1007200065735C6578706572696D656E74616C5F28
:100730006D656D6F626A5C6E72665F6D656D6F622E
:100740006A2E63005072696E7420737461747573DD
:10075000206F6620717565756520696E7374616EB2
:100760006365732E000000007175657565000000FB
:1007700025730D0A092D20456C656D656E74207317
:10078000697A653A0925640D0A092D205573616758
:10079000653A092575252520282575206F75742053
:1007A0006F6620257520656C656D656E7473290D07
:1007B0000A092D204D6178696D756D3A09257525F9
:1007C0002520282575206F7574206F6620257520DB
:1007D000656C656D656E7473290D0A092D204D6F6A
:1007E00064653A090925730D0A0D0A004E52465FE9
:1007F0004552524F525F494E56414C49445F444125
:10080000544100004E52465F4552524F525F534F83
:1008100046544445564943455F4E4F545F454E410B
:10082000424C4544000000004E52465F4552524F34
:10083000525F464541545552455F4E4F545F454EB9
:1008400041424C45440000004E52465F4552524FD3
:10085000525F4D555445585F554E4C4F434B5F4684
:1008600041494C45440000004E52465F4552524FAC
:10087000525F4D555445585F4C4F434B5F4641497D
:100880004C4544004E52465F4552524F525F4D55C3
:100890005445585F434F4E445F494E49545F46416B
:1008A000494C4544000000004E52465F4552524FAD
:1008B000525F4D555445585F494E49545F46414932
:1008C0004C4544004E52465F4552524F525F424C97
:1008D000455F495053505F52585F504B545F5452DC
:1008E000554E4341544544004E52465F4552524F87
:1008F000525F424C455F495053505F504545525FEF
:1009000052454A4543544544000000004E52465F5C
:100910004552524F525F424C455F495053505F4CD5
:10092000494E4B5F444953434F4E4E454354454413
:10093000000000004E52465F4552524F525F4150F8
:10094000495F4E4F545F494D504C454D454E5445BF
:10095000440000004E52465F4552524F525F4E4F88
:10096000545F535550504F52544544004E52465FC9
:100970004552524F525F4D4F44554C455F4E4F5478
:100980005F494E495449414C495A454400000000D2
:100990004E52465F4552524F525F4D4F44554C4563
:1009A0005F414C52454144595F494E495449414C7D
:1009B000495A4544000000004E52465F4552524F8E
:1009C000525F4E4F545F464F554E44004E52465F65
:1009D0004552524F525F494E56414C49445F535421
:1009E000415445004E52465F4552524F525F44417A
:1009F00054415F53495A45004E52465F4552524F4B
:100A0000525F494F5F50454E44494E470000000039
:100A10004E52465F4552524F525F5356435F4841D4
:100A20004E444C45525F4D495353494E47000000D8
:100A30004E52465F4552524F525F494E56414C49C5
:100A4000445F4C454E475448000000004E52465FFC
:100A50004552524F525F4452565F5457495F455278
:100A6000525F414E41434B004E52465F4552524FFA
:100A7000525F4452565F5457495F4552525F444E4D
:100A800041434B004E52465F4552524F525F494ED2
:100A90005445524E414C00004E52465F4552524F13
:100AA000525F53544F524147455F46554C4C0000EE
:100AB0004E52465F4552524F525F4E554C4C0000CD
:100AC0004E52465F4552524F525F494E56414C4935
:100AD000445F504152414D004E52465F4552524F85
:100AE000525F4E4F5F4D454D000000004E52465F35
:100AF0004552524F525F464F5242494444454E0080
:100B00004E52465F4552524F525F4452565F5457C1
:100B1000495F4552525F4F56455252554E000000B4
:100B20004E52465F4552524F525F494E56414C49D4
:100B3000445F4144445200004E52465F4552524F7A
:100B4000525F494E56414C49445F464C4147530021
:100B50004E52465F53554343455353004E52465FF2
:100B60004552524F525F424C455F495053505F438C
:100B700048414E4E454C5F414C52454144595F45BA
:100B800058495354530000004E52465F4552524F4D
:100B9000525F54494D454F55540000004E52465F38
:100BA0004552524F525F425553590000726561647D
:100BB00000000000526561642073746F72656420E8
:100BC0006C6F67730000000052656D6F7665206C76
:100BD0006F677300466C617368206C6F6720737475
:100BE0006174757300000000666C6173686C6F67F8
:100BF00000000000436F6D6D616E647320666F725C
:100C00002072656164696E67206C6F67732073740E
:100C10006F72656420696E206E6F6E2D766F6C61E9
:100C200074696C65206D656D6F7279002E2E5C2E77
:100C30002E5C2E2E5C2E2E5C2E2E5C2E2E5C636F78
:100C40006D706F6E656E74735C6C696272617269EF
:100C500065735C6578706572696D656E74616C5FF3
:100C60006C6F675C7372635C6E72665F6C6F675FFC
:100C70006261636B656E645F666C6173682E6300AE
:100C80002E2E5C2E2E5C2E2E5C2E2E5C2E2E5C2E9E
:100C90002E5C636F6D706F6E656E74735C6C6962F1
:100CA0007261726965735C6578706572696D656E95
:100CB00074616C5F6C6F675C7372635C6E72665FAD
:100CC0006C6F675F66726F6E74656E642E63000092
:100CD0006E6F6E650000000064656275670000005D
:100CE000276C6F6720656E61626C65203C6C657671
:100CF000656C3E203C6D6F64756C655F303E202EE8
:100D00002E2E20203C6D6F64756C655F6E3E272033
:100D1000656E61626C6573206C6F677320757020FF
:100D2000746F20676976656E206C6576656C2069E6
:100D30006E20737065636966696564206D6F6475A4
:100D40006C65732028616C6C206966206E6F206D65
:100D50006F64756C6573207370656369666965643B
:100D6000292E0000276C6F672064697361626C65CF
:100D7000203C6D6F64756C655F303E202E2E203CEC
:100D80006D6F64756C655F6E3E2720646973616288
:100D90006C6573206C6F677320696E207370656378
:100DA0006966696564206D6F64756C657320286180
:100DB0006C6C206966206E6F206D6F64756C657356
:100DC00020737065636966696564292E0000000000
:100DD000656E61626C65000064697361626C6500D8
:100DE000526573756D65206C6F6767696E6700008B
:100DF00048616C74206C6F6767696E670000000063
:100E0000676F00004C6F676765722073746174755B
:100E10007300000068616C74000000006C6F670074
:100E2000436F6D6D616E647320666F7220636F6EC9
:100E300074726F6C6C696E67206C6F6767657200A7
:100E40001B5B313B33306D001B5B306D00000000DD
:100E50001B5B313B33316D001B5B313B33326D002B
:100E60001B5B313B33336D001B5B313B33346D0017
:100E70001B5B313B33356D001B5B313B33366D0003
:100E80001B5B313B33376D006170705F74696D655A
:100E9000722E6D5F74696D65725F30007175657576
:100EA000652E6D5F636C695F6364635F61636D5F33
:100EB0006C6F675F6261636B656E645F71756575AA
:100EC0006500000062616C6C6F632E6D5F636C691E
:100ED0005F6364635F61636D5F636D645F686973C3
:100EE000745F6D656D6F626A000000006170705F15
:100EF00074696D65722E6D5F636C695F7274745F87
:100F00007472616E73706F72745F74696D65720074
:100F100071756575652E6D5F636C695F7274745F62
:100F20006C6F675F6261636B656E645F7175657539
:100F30006500000062616C6C6F632E6D5F636C69AD
:100F40005F7274745F636D645F686973745F6D650D
:100F50006D6F626A000000006D5F636C695F6364BF
:100F6000635F61636D5F6C6F675F6261636B656E2A
:100F7000645F7175657565006D5F636C695F727440
:100F8000745F6C6F675F6261636B656E645F7175E0
:100F9000657565006D5F636C695F6364635F616362
:100FA0006D5F636D645F686973745F6D656D6F62BB
:100FB0006A0000006D5F636C695F7274745F636DDB
:100FC000645F686973745F6D656D6F626A000000CD
:100FD0006170705F74696D65722E6D5F6273705FB2
:100FE0006C6564735F746D72000000006170705F07
:100FF00074696D65722E6D5F6273705F616C65728E
:10100000745F746D720000006170705F74696D656B
:10101000722E6D5F6273705F627574746F6E5F7451
:101020006D7200006E72665F6D707500737461633F
:101030006B5F677561726400636C6F636B000000C7
:101040005553424400000000434C4F434B00000006
:101050004750494F54450000505253005541525497
:101060000000000055415254450000006170705F5F
:1010700074696D65722E6D5F646574656374696F04
:101080006E5F64656C61795F74696D65725F6964D8
:10109000000000006170705F74696D65720000008F
:1010A00061746669666F2E6D5F7265715F666966F1
:1010B0006F0000006170705F757362640000000073
:1010C0006364635F61636D006170705F7573626418
:1010D0005F636F7265000000686172646661756CC1
:1010E0007400000071756575652E6D5F72785F71B3
:1010F00075657565000000006D5F72785F717565DC
:1011000075650000636C695F7561727400000000B2
:101110006E72665F6673746F7261676500000000CF
:101120007077725F6D676D7400000000736F72748A
:101130006C6973740000000071756575652E6D5FD4
:10114000666C6173686C6F675F71756575650000CB
:1011500071756575652E6D5F63726173686C6F671D
:101160005F717565756500006D5F666C6173686CB5
:101170006F675F7175657565000000006D5F637274
:101180006173686C6F675F7175657565000000005D
:1011900062616C6C6F632E6C6F675F6D656D706FF5
:1011A0006F6C0000617070006C6F675F6D656D70D3
:1011B0006F6F6C005414010008000020FC04000054
:1011C0002817000078150100040500200C3B0000E2
:1011D000A021000000000000D0E800000000000096
:1011E00018E900000000000028E9000000000000ED
:1011F00080E9000000000000F0E9000000000000AD
:10120000BCEA00000000000020ED0000000000002B
:1012100030ED00000000000040ED00000000000084
:1012200088ED000000000000D0ED0000000000008C
:1012300004EF00000000000014EF000000000000B8
:1012400024EF00000000000034EF00000000000068
:10125000A8F000000000000074F200000000000090
:10126000FCF20000880E0100000004039C0E010047
:1012700000000003C40E010000000003EC0E01009A
:1012800000000403100F010000000003340F0100F0
:1012900000000003D00F010000000403EC0F010068
:1012A00000000403081001000000040324100100E2
:1012B000000000002C1001000000040438100100A0
:1012C0000000000040100100000000004810010074
:1012D0000000000050100100000000005810010044
:1012E000000000005C10010000000000641001001C
:1012F000000000006C1001000000040394100100C5
:1013000000000404A010010000000003B41001005C
:1013100000000000C010010000000000C810010023
:1013200000000000D810010000000404E4100100D7
:101330000000000304110100000000001011010072
:101340000000040420110100000000002C11010025
:1013500000000000381101000000000350110100DE
:10136000000000039011010000000003A41101001F
:1013700000000404D0000020C8000020D00000209D
:10138000040B002084030020940F010030000000B3
:10139000E0000020D8000020E0000020FC0F00202A
:1013A000A8030020B40F010030000000C00200209C
:1013B000D4170020E4170020E4170020EC040020DC
:1013C000A811010018000000F80A0020E40A00201B
:1013D000040000000400000001000000580F01009C
:1013E00078030020F00F0020DC0F00200400000034
:1013F0000400000001000000780F01009C030020A1
:10140000A816002024160020800000000100000023
:1014100000000000F81001009804002018170020B8
:10142000F416002008000000040000000100000085
:1014300068110100D4040020481700202417002060
:101440000800000004000000010000007C11010001
:10145000E004002081A314F29A200C0114136C0301
:10146000422013B80AB320172328EA231D94A3E0CF
:10147000ED041DC813015A904CCBB00F4C0A114417
:101480004C0A1DE44C01142304FB1A0C041A1C041E
:101490001A14041A24041A2C041A40041A38041AC0
:1014A00068041A70041A80041A78041A48041A503E
:1014B000041A60041A580401451510014011021164
:1014C000044B5C04FC011003264131239CEC1AA060
:1014D000041ACA041AF00403120AED12A8120163D6
:1014E000BCFF143401011A80041A1814811AE80C84
:1014F00023DCFD1A7004111302011A44049A6420BB
:1015000029401BD8FE3C2944193C01101ACC141A5E
:101510008C200B1060061C141C14011A38040114D2
:1015200013941773203F2922137C02242095521410
:10153000D00C011AF81223A8FC23D4FA1AD81029C7
:1015400004291429102920291C0114E93814480EF3
:10155000011A40041A50041A58041A60041A680444
:101560001A70041A78041A800411045490D003638A
:081570003D7403FFFF0F019B16
:00000001FF
